:020000040000FA
:200000000208540200800402003F00020008B922FFFFFF02008014FFFFFFFF0200801CFFAA
:20002000FFFFFF020080245745422D47535737323454472020204C56332E30EB7002E722F0
:2000400089828A831410E704F593E022F593E49322BB0002F722BB8000500989828A838BC1
:20006000931593F022BC000BBE0029EF8DF084FFADF022E4CCF875F008EF2FFFEE33FEEC9A
:2000800033FCEE9DEC984005FCEE9DFE0FD5F0E9E4CEFD22EDF8F5F0EE008420D21CFEADD5
:2000A000F075F008EF2FFFED33FD4007985006D5F0F222C398FD0FD5F0EA22A3F8E0C5F033
:2000C00025F0F0E582158270021583E0C838F0E822BB0006F709A7F01922BB8000500D8985
:2000E000828A838B931593F0E5F0A3F022E88FF0A4CC8BF0A42CFCE98EF0A42CFC8AF0ED79
:20010000A42CFCEA8EF0A4CDA8F08BF0A42DCC3825F0FDE98FF0A42CCD35F0FCEB8EF0A40D
:20012000FEA9F0EB8FF0A4CFC5F02ECD39FEE43CFCEAA42DCE35F0FDE43CFC22EB9FF5F0F0
:20014000EA9E42F0E99D42F0E89C45F022E8600FEFC333FFEE33FEED33FDEC33FCD8F122D5
:20016000BB0006E9F802000332BB8000500C89828A838B9315930200017B22ECF0A3EDF035
:20018000A3EEF0A3EFF022EB700C87F009E608B5F019DFF6801589828A831410E70FF59383
:2001A000E0F5F0A3E608B5F002DFF5806AF593E493F5F0A3E608B5F05EDFF4805ACB701311
:2001C00088828C838B9387F009E493A3B5F048DFF580441410E71F88848C858B9589828ACD
:2001E00083F593758620E0F5F0E493A3A3B5F024DFF4DEF2801E88848C858B9589828A83F8
:20020000F593758620E493F5F0E493A3A3B5F004DFF3DEF17586007FFFB5F0020F22400245
:200220007F012202000187809488F0EF60010E4E60F0ED60EE1410E7EECB701288828C8370
:20024000F59387F009E0A3B5F0CDDFF680C91410E71E88848C858B9589828A83F593758682
:2002600020E0F5F0E0A3A3B5F0AADFF5DEF380A488848C858B9589828A83F593758620E47F
:2002800093F5F0E0A3A3B5F08BDFF4DEF28085EB7008E709F608DFFA801B89828A831410E7
:2002A000E70AF593E0A3F608DFFA8009F593E493A3F608DFF9ECFAA9F0EDFB2288F0EF601A
:2002C000010E4E60F088F0ED60C51410E7E7CB700E88828C838B93E709F0A3DFFA80D614AF
:2002E00010E71C88848C858B9589828A83F593758620E0F0A3A3DFFADEF875860080B68875
:20030000848C858B9589828A83F593758620E493F0A3A3DFF9DEF77586008099C5F0F8A3AF
:20032000E028F0C5F0F8E582158270021583E038F022ECF608EDF608EEF608EFF62290008E
:200340007004E0F54090007005E0F541854082854183E020E7077E007F00C2D72289428A6E
:20036000435407F54512000539E02402F54450020545120003E0053AE53A7002053BE54050
:200380002544F540E541354530E604C2E6242DF5411200040090007004E540F090007005A2
:2003A000E541F0AE45AF44D2D72290007010E020E61EA3EDF0A3E9F0A3EAF0EC5407D2E6EA
:2003C00090007010F00538E53870020539D2D7227C007D00C2D72290007010E0A2E6B32247
:2003E00075F001800375F0041200040078407F06900070921200052190007090E5F0F02217
:2004000090007090E0540770F7221200046D90007008742DF0900070107508101200045861
:20042000E490007004F090007006F0742D90007005F090007007F0751D10751C10751E008B
:20044000751F2D75832D758200E4F0753800753900753A00753B0022E4A808F0A3D8FC22F2
:20046000120005171200040A120004AB22900004A175080A79707860120005287518C075CD
:2004800019A8751A00751B647510C07511A87512007513017514FF7515FF7516FF7517006E
:2004A00022000B78667788C0A800649000706AE0440CF0229000706AE054F3F02290007017
:2004C0006AE04401F0229000706AE054FEF0229000706AE04402F0229000706AE054FDF0A0
:2004E000229000706AE04440F0229000706AE054BFF02290007000E04410F0229000700045
:20050000E054EFF02290007000E04420F02290007000E05420F0229000700AF000000000F0
:2005200022E6F008A3DFFA2289A0E493A3F208B800030989A0D508F222A3E58330E6037569
:20054000832D22754300754200754100754000754508754400120003E5754308754200758E
:200560004108754000754508754400120003E51200040090000000750910750800750B00D7
:20058000750A0012000638400B9000706CE04408F0D2D722C2D7227543007542007541000E
:2005A000754000754508754400120003E5754308754200754108754000754508754400129A
:2005C0000003E51200040090000000750910750800750B00750A00120006384051754310DA
:2005E000754200754110754000754508754400120003E575431875420075411875400075D5
:200600004508754400120003E51200040090001000750910750800750B10750A00120006F2
:2006200038400B9000706CE04418F0D2D722C2D722E6F008A3DFFA22A90B89A0A80AE49397
:20064000F5F0A3E265F0701008B800030989A01200067D50E9C2D722D2D722A90B89A0A88D
:200660000AE0F5F0A3E265F0701008B800030989A01200067D50EAC2D722D2D722E50860BA
:200680000A14F50845097007D2D72215091508C2D7229000700B7418F09000700C7420F0A2
:2006A00075A06022120006927824E2E2B408157400F21200072912000721120007071200B4
:2006C000070E802E22120006927816E2E2703708E2E2B4013178281200079C5029120007F9
:2006E0003912000779120007411200078178177402F27800E2E2FC4480F208E2E2FD7918FC
:200700007A20120003AA22781AE4F208F222782680F7E2E2F5F0E3E3F2E5F0F30809DAF2BF
:20072000227A04781C792080E9790878027A0680E1E2E2F30809DAF922780879027A0680EF
:20074000F0780879227A0680E8E4F309F3227A08E480037A04E4F309DAFC22E0F3A309E013
:20076000F3227A04E0F3A309DAFA227A0280027A04E2E2F0A308DAF922900070607A068041
:20078000E3781879227A0A8089E0F5F0E2E265F0700708A3DAF3D2D722C2D7229000706605
:2007A0007A0480E59000200AE0FEA3E08E8375820075814F73220D0A205446333331465556
:2007C0003A333956463038302031364B2D626173656420426C616E6B20436865636B696E64
:2007E00067002E2E2E5B6661696C5D0A002E2E2E5B6F6B5D0A000D0A205446333331465581
:200800003A6465766963655B53535420333956463038305D000D0A20544633333146553A7F
:20082000536563746F722D62617365642832353620736563746F72732920466C61736820DD
:2008400045726173652028314D29002E2E2E5B6F6B5D2E0075C7AA75C755759D02787FE409
:20086000F6D8FD900000007F007E607D01E4F0A3DFFCDEFADDF875814F12000517D20D12DF
:200880000004B41200040A12001DD412001DF0120013EBEF7004020008A5020008B312006D
:2008A0001D36EF700EC20D120004AB1200000702000C7BD20D02008000300D040200800C16
:2008C000C0E0C0D075D00012001DACD0D0D0E0320D0A544633333146553A52657620257542
:2008E0000A54616966617465636820496E632E000D0A2849503D200025752E00257529003D
:200900000D0A284D41433D200025782E00257829000D0A54463333313A2054465450206475
:200920006F6E652E204A756D7020746F20307825782E0A000D0A436865636B204368656363
:200940006B53756D3D00307825782E2E2E4F4B21210D0A00307825782E2E2E4661696C218C
:20096000210D0A001B5B324A000D0A436865636B204D6167696320436F64652E2E2E004FE3
:200980004B2121004661696C212100496C6C6567616C206669726D77617265002E000D0A90
:2009A00020496E76616C6964206669726D776172652021000D0A20466C6173682065727204
:2009C0006F722021004387049000555574AAF090002AAA7455F09000555574A0F08F828EE5
:2009E000838D93E52EF05387FB229000262FEEF0A3EFF0E4784EF608F6D390002630E0944A
:200A0000009000262FE094005003010C7A90002620E0FF94094003010B36EF705E90002659
:200A20002FE0FEA3E0FFD39400EE94004031784EE6FC08E67B012448F974203CFA1200007A
:200A40003B643A601A90002630E024FFF09000262FE034FFF0784F06E61870C10680BEEF53
:200A60004E7003010C7A784B7601900026207401F0784F06E618704F06804C90002620E0A7
:200A8000784BF6784BE6C39409504E90002630E094009000262FE09400403E784E0806E60B
:200AA000188606700106147B012448F974203EFA1200003BFF784BE6062423F582E4342663
:200AC000F583759300EFF090002630E024FFF09000262FE034FFF080AA784BE6900026204D
:200AE000F0C394095003010C7A9000261A7426F0A37423F0120018D1EF64014E70069000A5
:200B00002620F022120018D1EF64044E7003010C2B7D027F01120018D59000261CEFF07D06
:200B2000067C007F037E00120018D990002614EEF0A3EFF0807E9000261DE0FFA3E0900043
:200B40002614CFF0A3EFF090002621E06066D390002630E094009000262FE09400405590F2
:200B600000261A7426F0A37421F0784E0806E6188606700106147B012448F974203EFA12DB
:200B800000003B90002622F090002630E024FFF09000262FE034FFF07D017C00E4FFFE12A4
:200BA0000018D912001541E490002621F09000261CE014F09000261A7420F0A37448F0A335
:200BC000E0FF784C760008A607D3784DE6940018E694004049D390002630E0940190002636
:200BE0002FE094004038784EE6FE08E6FF2401FDE43EFC120018D912001541784F74022635
:200C0000F618E436F618E6161870011690002630E024FEF09000262FE034FFF080AB784D53
:200C2000E69000261CF0E61846700890002620F00109F99000262FE07004A3E064017026D0
:200C4000784E0806E6188606700106147B012448F974203EFA1200003B90002621F0E49076
:200C600000262FF0A3F090002614E0FFA3E09000261DCFF0A3EFF00109F922900070FFE058
:200C8000784AF67E087FD0E6540FFD7C0012000E721200113C7E087FF0E4FDFC12000E72B0
:200CA000E4784AF6784AE6FDC39403501E7E087FF874042DF582E43420F583759300E0FD7D
:200CC0007C0012000E72784A0680D97E087FFC90002007E0FD7C0012000E727E097F00E458
:200CE000FDFC12000E72E4784AF6784AE6FDC39405501E7E097F0974122DF582E43420F5F8
:200D000083759300E0FD7C0012000E72784A0680D97E097F0D90002017E0FD7C0012000EE9
:200D2000727B017A2079181200033E90002608EEF0A3EFF0D39424EE940040E59000202621
:200D4000E0B4081FA3E0B4061A90002609E024F0F090002608E034FFF0120006C5784AA6D8
:200D60000780BE90002026E0B408B6A3E0B400B19000202AE0FFA3E090002608CFF0A3EFD3
:200D8000F090002034E0FCA3E0FDA3E0FEA3E0FF900020001200017BE4784AF6784AE6FF9F
:200DA0007C007B012420F9EC3420FA1200003BFE740C2FF582E43420F583759300EEF006B7
:200DC000E6B406D890002028E064456003010D219000202EE0543F6003010D2190002031E4
:200DE000E0B4010E120006A4E490002608F0A3F0805190002031E0B411499000203EE07091
:200E000004A3E06445701690002609E024E4F090002608E034FFF012000FDA802690002073
:200E20003EE064FC7004A3E064036003010D2190002609E024E4F090002608E034FFF012DA
:200E400000164D9000264DE07003010D2112001E169000200A741FF0A374FCF07E097F110D
:200E6000FD7C1F12000E72C2A9C2AF120007A4010D2190002638EEF0A3EFF0A3ECF0A3ED23
:200E8000F090002638E475F001120000BB85F082F583759300E4939000263DF07003010F09
:200EA000D9E064256003010FBA9000263C740AF090002638E475F001120000BB85F082F572
:200EC00083759300E49324DB7003010FBA800090002639E024FFF090002638E034FFF090F1
:200EE000002638E475F001120000BB85F082F583759300E4939000263DF0E0249D60142473
:200F0000EE601924FD6003010FBA9000263C7410F080099000263BE0FF010FD29000263E87
:200F2000740AF09000263AE07002A3E0605A9000263CE0FBFD7C009000263AE0FEA3E0FF2E
:200F400012000065AA059000263AE0FEA3E0FFEBFD7C00120000659000263AEEF0A3EFF0F0
:200F6000D3EA64809489EA40052457FF80032430FF9000263EE014F0244EF582E43426F540
:200F800083759300EFF0809B9000263EE0B40A047F30803E9000263EE0C3940A4003010E42
:200FA00081E0FF04F0744E2FF582E43426F583759300E0FF12001E2880DA9000263DE0FF54
:200FC00012001E289000263DE0640A6003010E817F0D12001E28010E812290002044E0FE1D
:200FE000A3E0FFEE600301113BEF24FD606404600301113B12001C509000203CE0FFA3E07D
:2010000090002643CFF0A3EFF09000203EE0FEA3E0FF90002641EEF0A3EFF090002044E419
:20102000F0A37404F0E4A3F0A3F09000203CEEF0A3EFF090002643E0FFA3E09000203ECF47
:20104000F0A3EFF090002608E4F0A37404F0020012949000203EE0FEA3E0FF90002641E0B4
:201060006E7003A3E06F60030111339000263FE0FEA3E0FF90002046E0B50608A3E0B507C8
:201080000301112F90002640E02401FF9000263FE03400FE90002046E06E7003A3E06F6002
:2010A000030111339000203CE0FFA3E090002643CFF0A3EFF07E097F9CE4FDFC12000E724F
:2010C000C390002609E09404FF90002608E09400FE120009EA9000262EE0702B90002617B6
:2010E000E0C3941450067E097F9E80047E097FB4E4FDFC12000E727F047E0012001BE4905C
:2011000000264D7401F02290002640E004F070079000263FE004F0C390002609E094049041
:20112000002608E0940250079000264D7401F002001D72E490002608F0A3F022D2A9D2AF78
:20114000E49000262FF0A3F09000262FE0FEA3E0FFC39402EE9400505BEF2404FFE43EFE42
:2011600012001A7D90002631EEF0A3EFF0E0FD90002630E025E0FB9000262FE033FA740472
:201180002BF58274203AF583759300EDF090002631E0FF74052BF58274203AF58375930053
:2011A000EFF090002630E004F0709D9000262FE004F08094E49000262FF0A3F09000262F8B
:2011C000E0FEA3E0FFC39403EE9400505412001A7D90002631EEF0A3EFF0E0FD900026307C
:2011E000E025E0FB9000262FE033FA74122BF58274203AF583759300EDF090002631E0FF04
:2012000074132BF58274203AF583759300EFF090002630E004F070A49000262FE004F08071
:201220009BE4784BF6784BE6FF2404F582E43420F583759300E0FEEF2466FDE434708D828C
:20124000F583759300EEF006E6B404D9E4784BF6784BE6FF2412F582E43420F58375930009
:20126000E0FEEF2460FDE434708D82F583759300EEF006E6B406D99000706CE054FDF0908F
:20128000007001743FF0900070007410F0900070DAE4F02290002609E02408FE900026086F
:2012A000E0340090002040F0A3CEF0E4A3F0A3F090002000E0FCA3E0FDA3E0FEA3E0FF9030
:2012C0000020381200017B90002004E0FCA3E0FDA3E0FEA3E0FF900020341200017B900013
:2012E0002609E0241CF090002608E03400F0900020287445F0E4A3F09000202E7440F0E48F
:20130000A3F0A37410F0A304F090002608E0FFA3E09000202ACFF0A3EFF090002009E004B4
:20132000F0700790002008E004F090002008E09000202CF090002009E09000202DF0E4907C
:20134000002032F0A3F0900020187490F090002609E02412F090002608E03400F0C3A3E02F
:20136000944090002608E094005006E4F0A37440F090002018E054F8FE90002608E04EFF19
:20138000A3E090002018CFF0A3EFF0E4FF740C2FF582E43420F583759300E0FEEF7C007B3C
:2013A00001241AF9EC3420FAEE120000510FEFB406DBE4FF74122FF582E43420F583759310
:2013C00000E0FE74202FF582E43420F583759300EEF00FEFB406DD900020267408F0A3E401
:2013E000F07B017A207918020003AAE4FFFEFDFC9000262F1200017BE490002633F07E0916
:201400007F64FDFC12000E727E097F69E4FDFC12000E727FFC7EFF7D0F7C00900026341284
:2014200000017B9000262FE0F8A3E0F9A3E0FAA3E0FBC000C001C002C003A3E0FFE4FDFE95
:20144000A3A3E0F9A3E0FAA3E02FFFEE3AFEED39FDE42FFFE43EFEED3481FDA907AA06AB1A
:20146000051200003BFFD003D002D001D000EB4FFFEAFEE9FDE8FC9000262F1200017B90E7
:2014800000262FE0FCA3E0FDA3E0FEA3E0FF78081200014D9000262F1200017B900026335C
:2014A000E004F0E0C3940350030114239000262FE0F8A3E0F9A3E0FAA3E0FBC000C001C01E
:2014C00002C003A3E0FFE4FDFEA3A3E0F9A3E0FAA3E02FFFEE3AFEED39FDE42FFFE43EFE1E
:2014E000ED3481FDA907AA06AB051200003BFFD003D002D001D000EB4FFFEAFEE9FDE8FCC0
:201500009000262F1200017B7F557EAA7D557CAA9000262FE0F8A3E0F9A3E0FAA3E0FBC36D
:201520001200013C700D7E097F7FFDFC12000E727F01227E097F84E4FDFC12000E727F00B5
:201540002290002618EEF0A3EFF090002614E475F001120000BBAFF090002631F0A3EFF062
:2015600090002619E0FF9000262CF090002046E07004A3E0640160030115FC90002631E07D
:20158000FCA3E0FDC39427EC9400403CD3ED943AEC9400503390002617E004F08D828C8305
:2015A000759300E4936F6006E49000262DF090002617E0B414129000262DE07004A3F0804F
:2015C000079000262E7401F090002616E0702DA3E0641470279000262EE06020E4F52F1282
:2015E0000005971200173912001810EF70069000262EF022900026167401F022900026311E
:20160000E0FEA3E04E7002052F9000262EE06401703A90002616E0640170319000262CE02E
:20162000FDF46028E52F7011C3EE9440401E90002631E0FEA3E0FF800F90002631E0FEA37B
:20164000E0FF9000262CE0FD12001B76227FD87E5A7D947C0190002054E0F8A3E0F9A3E08F
:20166000FAA3E0FBC31200013C600301173890002046E0FEA3E0FF64014E6007EF4E60031D
:20168000011738E490002052F0A3F090002050E0FEA3E0FFEE6003011738EF24FB600B24F3
:2016A000FB600924096003011738802D78127C207D017B017A2079487E007F06120002297E
:2016C000EF707590002608E4F0A37428F090002050E4F0A3740BF0800E12001CA390002080
:2016E00050E4F0A3740CF078487C207D017B017A2079127E007F06120002BC90002044E48D
:20170000F0A37402F0A3E4F0A304F09000204EE4F0A304F09000203EE0FEA3E0FF9000205B
:201720003CE0FDA3E0A3CDF0A3EDF09000203CEEF0A3EFF012001294227E077FF6E4FDFC30
:2017400012000E727E087F15E4FDFC12000E72E4F52FF523752408AE23AF24E4FCFDFB7AB7
:2017600010F9F8120000ED8F288E278D268C25A2AFE433F522C2AF4387049000555574AA83
:20178000F090002AAA7455F0900055557480F074AAF090002AAA7455F0E47FFF7EFFFDFC1B
:2017A000AB28AA27A926A825D31200013C401BE42528FFE43527FEE5263401FDA907AA0661
:2017C000AB05743012000051800C8528828527837593007430F05387FBE52224FF92AFAEDE
:2017E00023AF24E4FCFDFB7A10F9F8120000ED120019FB0524E52470020523C3E52394014F
:2018000050030117577E087F4BE4FDFC02000E727E077FB6E4FDFC12000E72E4752502F5B9
:2018200024F523F522E47F3FFEFDFCAB25AA24A923A822D31200013C40030118C3E4F52648
:20184000F527E4FF7E40FDFCAB25AA24A923A822120000ED8F2B8E2A8D298C28E4FCFDE501
:201860002B2527F52BE52A3526F52AED3529F529EC3528F528E4252BFFE4352AFEE52934C3
:2018800081FDA907AA06AB051200003BF4600D7E077FE2E4FD12000E727F00220527E527DA
:2018A00070020526C3E52694404097E5252401F525E43524F524E43523F523E43522F522CD
:2018C0000118257E077FEDE4FDFC12000E727F01227D087F077C007E0090002631ECF0A35D
:2018E000EDF0E4A3F0A3F0AD07AC06C390002632E09D90002631E09C40629000261AE0FEC0
:20190000A3E08E837593002DF582E5833CF583759300E0F990002634E0C4F8540FC868F081
:2019200090002633E0C454F048F0E9D39439500BE9C39430FFE49400FE8013C3E99441FFC2
:20194000E49400CF240ACF3400FE90002633E04EF0A3E04FF00DBD00010C808F9000263379
:20196000E0FEA3E0FF2290002635EEF0A3EFF09000265C7408F0F5C84402F0F5C87F327E3D
:201980000012001E159000265CE04404F0F5C87F647E0012001E1512001E079000265A74BA
:2019A00008F0A3E4F09000265AE0FCA3E0FD4C6043A3E054FAF090002635E0FEA3E0FFEC65
:2019C0005EFEED5F4E60089000265CE04404F09000265CE012001E0F12001E119000265CFB
:2019E000E04401F0F5C89000265AE0C313F0A3E013F080B19000265CE0FF22900026361297
:201A000000017B752901E4F52CF52D90002636A3E0FDA3E0FEA3E02400FFE43EFEED34812F
:201A2000FDA907AA06AB051200003BF52A532A40E529604090002636A3E0FDA3E0FEA3E052
:201A40002400FFE43EFEED3481FDA907AA06AB051200003BF52B532B40E52AB52B03E4F59E
:201A600029852B2A052DE52D7002052CB4FFC1E52CB4FFBCE5297F0060027F0122C2AFEE98
:201A80004408FE120019669000265CEFF0E490002633F0A3F09000265A7480F0A3E4F0902F
:201AA00000265AE07002A3E060379000265CE054FA12001E0E12001E07AFC8EF30E3149068
:201AC00000265AE0FEA3E0FF90002633E04EF0A3E04FF09000265AE0C313F0A3E013F080A1
:201AE000BE9000265CE054F8F0F5C87F907E0112001E15D2AF90002633E0FEA3E0FF2290EE
:201B000000262FEBF0A3EAF0A3E9F0E490002637F0A3F09000263574FFF5F0120000BB45F3
:201B2000F0604690002632E0FBA3E0FAA3E0F91200003BFF9000262FE0FBA3E0FAA3E0F94E
:201B400090002637E475F001120000BBFCE925F0F9EA3CFAEF1200005160B890002633E437
:201B600075F0011200031C80AA9000262FE0FBA3E0FAA3E0F92290002633EEF0A3EFF0A3DD
:201B8000EDF0AF2FE4FCFDFEFBFA7901F8120000ED8F268E258D248C2390002633E0FEA317
:201BA000E0FFE4FCFDE5262FF526E5253EF525ED3524F524EC3523F523A3E0F52EA2AFE41C
:201BC00033F522C2AFAF26AE25AD24AC23120009C5AF26AE25AD24AC23120019FBE5222489
:201BE000FF92AF22900070007429F090002044E4F0A37405F0A3EEF0A3EFF064044E7020D9
:201C0000900026327481F0A37409F0A3748BF0A3E4F0A37411F07B017A20794812001AFFC4
:201C200090002641E0FFA3E09000203CCFF0A3EFF090002643E0FFA3E09000203ECFF0A373
:201C4000EFF090002608E4F0A37415F002001294E49000263FF0A3F090002000E0FCA3E0E4
:201C6000FDA3E0FEA3E0FF900026451200017BE490002641F0A3F0A3F0A3F09000264DF064
:201C80009000262EF090002617F090002616F09000262D04F0900070007421F0900070DAC1
:201CA000E4F0227B017A20796CE475F004120000D1740229F9E43AFAE475F008120000D11F
:201CC000740229F9E43AFA90002004E0FCA3E0FDA3E0FEA3E0FF12000160740429F9E43A16
:201CE000FEC3E99444FFEE942090002608F0A3EFF0229000262FEEF0A3EFF0E4F523D3ED6E
:201D00009400EC9400402C9000262FE0FEA3E0AA06F97B811200003B2523F523ED1D700130
:201D20001C90002630E004F070D49000262FE004F080CBAF23227E097F34E4FDFC12000E5A
:201D400072E4F522FD7C80FF7E8012001CF28F22E522B4FF0E7E097F46FD7C0012000E7230
:201D60007F01227E097F54AD227C0012000E727F002290002044E4F0A37404F0900026411F
:201D8000E0FFA3E09000203CCFF0A3EFF090002643E0FFA3E09000203ECFF0A3EFF090009A
:201DA0002608E4F0A37404F002001294C0D0C2A9C2AFE5492401F549E43548F548E4354773
:201DC000F547E43546F546758C5D758A3DD2AFD2A9D0D022E58954F04401F589758C5D758D
:201DE0008A3DE4F549F548F547F546D2B9D28C227598504387805389CF438920758DF37593
:201E00008CF3D28ED299229000265CE04401F0F5C87FF47E01229000706CE054E7F022AF16
:201E200049AE48AD47AC46223099FDC2998F9922FFFFFFFFFFFFFFFFFFFFFFFFFFFFFFFF00
:201E4000FFFFFFFFFFFFFFFFFFFFFFFFFFFFFFFFFFFFFFFFFFFFFFFFFFFFFFFFFFFFFFFFA2
:201E6000FFFFFFFFFFFFFFFFFFFFFFFFFFFFFFFFFFFFFFFFFFFFFFFFFFFFFFFFFFFFFFFF82
:201E8000FFFFFFFFFFFFFFFFFFFFFFFFFFFFFFFFFFFFFFFFFFFFFFFFFFFFFFFFFFFFFFFF62
:201EA000FFFFFFFFFFFFFFFFFFFFFFFFFFFFFFFFFFFFFFFFFFFFFFFFFFFFFFFFFFFFFFFF42
:201EC000FFFFFFFFFFFFFFFFFFFFFFFFFFFFFFFFFFFFFFFFFFFFFFFFFFFFFFFFFFFFFFFF22
:201EE000FFFFFFFFFFFFFFFFFFFFFFFFFFFFFFFFFFFFFFFFFFFFFFFFFFFFFFFFFFFFFFFF02
:201F0000FFFFFFFFFFFFFFFFFFFFFFFFFFFFFFFFFFFFFFFFFFFFFFFFFFFFFFFFFFFFFFFFE1
:201F2000FFFFFFFFFFFFFFFFFFFFFFFFFFFFFFFFFFFFFFFFFFFFFFFFFFFFFFFFFFFFFFFFC1
:201F4000FFFFFFFFFFFFFFFFFFFFFFFFFFFFFFFFFFFFFFFFFFFFFFFFFFFFFFFFFFFFFFFFA1
:201F6000FFFFFFFFFFFFFFFFFFFFFFFFFFFFFFFFFFFFFFFFFFFFFFFFFFFFFFFFFFFFFFFF81
:201F8000FFFFFFFFFFFFFFFFFFFFFFFFFFFFFFFFFFFFFFFFFFFFFFFFFFFFFFFFFFFFFFFF61
:201FA00075C7AA75C755759D02787FE4F6D8FD900000007F007E607D01E4F0A3DFFCDEFA5B
:201FC000DDF875814F12000517C20D120004B41200040A12001DD412001DF0C20D120004F9
:201FE000AB02000C7BFFFFFFFFFFFFFFFFFFFFFFFFFFFFFFFFFFFFFFFFFFFFFF0200085466
:20200000020020C0C5F0F8A3E028F0C5F0F8E582158270021583E038F022EB9FF5F0EA9EC0
:2020200042F0E99D42F0E89C45F022E8600FECC313FCED13FDEE13FEEF13FFD8F122E86096
:202040000FEFC333FFEE33FEED33FDEC33FCD8F122BB0006E9F8020020B4BB8000500C89B3
:20206000828A838B9315930200206C22ECF0A3EDF0A3EEF0A3EFF022D093D083D082E4935B
:202080007012740193700DA3A393F8740193F5828883E4737402936C70127403936D700C9D
:2020A0007404936E70067405936F60DDA3A3A3A3A3A380CAECF608EDF608EEF608EFF62295
:2020C00002002FF6E490002005F0A3F0E0FF12003492E490002004F090002004E0FF04F0F7
:2020E000EFC3940A5069E47F807E80FDFC9000200F1200206C90002006E0FFC00790002094
:202100000FE0FCA3E0FDA3E0FEA3E0FF900020161200206CD0077D147C00120032D790005E
:202120002006E0FF7B017A20790F7D147C00120033E5E47F807E80FDFC9000200FE0F8A3B1
:20214000E0F9A3E0FAA3E0FBC31200201A708990002004E0B40A0280FEE47F81FEFDFC9066
:2021600000200F1200206C90002006E0FFC0079000200FE0FCA3E0FDA3E0FEA3E0FF900088
:2021800020161200206CD0077D177C00120032D7E4FF7E04FDFC9000200F1200206C90001E
:2021A0002006E0FFC0079000200FE0FCA3E0FDA3E0FEA3E0FF900020161200206CD0077D7D
:2021C000187C00120032D7E490002004F090002004E0FF245AF582E43420F583759300E0A8
:2021E000FE74092FF582E43420F583759300EEF090002004E004F0E0B406D2E4900020049C
:20220000F090002004E0FBC39403506DE0FD25E02409F582E43420F583759300E0FEED25FA
:20222000E0240AF582E43420F583759300E0FDEDFFE4FCFD9000200F1200206C90002006A8
:20224000E0FFC007EB2419FDE433FCC004C0059000200FE0FCA3E0FDA3E0FEA3E0FF900069
:2022600020161200206CD005D004D007120032D790002004E004F08088E47F747E88FDFC89
:202280009000200F1200206C90002006E0FFC0079000200FE0FCA3E0FDA3E0FEA3E0FF90D7
:2022A0000020161200206CD0077D1C7C00120032D7E47F807E19FDFC9000200F1200206C73
:2022C00090002006E0FFC0079000200FE0FCA3E0FDA3E0FEA3E0FF900020161200206CD050
:2022E000077D1D7C00120032D7E47F2C7E01FDFC9000200F1200206C90002006E0FFC007E6
:202300009000200FE0FCA3E0FDA3E0FEA3E0FF900020161200206CD0077D1E7C0012003209
:20232000D7E4FFFEFDFC9000200F1200206C90002006E0FFC0079000200FE0FCA3E0FDA375
:20234000E0FEA3E0FF900020161200206CD0077D267C00120032D7E47FFF7EFFFDFC900040
:20236000200F1200206CE490002004F090002004E0FEC39424503D90002006E0FFC007EE24
:202380002427FDE433FCC004C0059000200FE0FCA3E0FDA3E0FEA3E0FF9000201612002043
:2023A0006CD005D004D007120032D790002004E004F080B8E47FFFFEFDFC9000200F12002C
:2023C000206C90002006E0FFC0079000200FE0FCA3E0FDA3E0FEA3E0FF90002016120020FF
:2023E0006CD0077D4B7C00120032D7E47FFF7EFFFDFC9000200F1200206C90002006E0FF71
:20240000C0079000200FE0FCA3E0FDA3E0FEA3E0FF900020161200206CD0077D4C7C001245
:202420000032D7E47FFF7E01FDFC9000200F1200206C90002006E0FFC0079000200FE0FC65
:20244000A3E0FDA3E0FEA3E0FF900020161200206CD0077D4D7C00120032D7E47FFF7EFF7E
:20246000FDFC9000200F1200206C90002006E0FFC0079000200FE0FCA3E0FDA3E0FEA3E08B
:20248000FF900020161200206CD0077D4E7C00120032D7E47FA07EC0FDFC9000200F120095
:2024A000206C90002006E0FFC0079000200FE0FCA3E0FDA3E0FEA3E0FF900020161200201E
:2024C0006CD0077D687C00120032D7E47F417EFAFDFC9000200F1200206CE490002004F043
:2024E00090002004E0FEC39402503D90002006E0FFC007EE2469FDE433FCC004C005900064
:20250000200FE0FCA3E0FDA3E0FEA3E0FF900020161200206CD005D004D007120032D7909E
:20252000002004E004F080B8E47F417EFAFDFC9000200F1200206CE490002004F0900020C1
:2025400004E0FEC39402503D90002006E0FFC007EE246BFDE433FCC004C0059000200FE0A2
:20256000FCA3E0FDA3E0FEA3E0FF900020161200206CD005D004D007120032D79000200429
:20258000E004F080B8E47F107E20FDFC9000200F1200206C90002006E0FFC0079000200FAD
:2025A000E0FCA3E0FDA3E0FEA3E0FF900020161200206CD0077D6D7C00120032D7E47F0499
:2025C0007E08FDFC9000200F1200206C90002006E0FFC0079000200FE0FCA3E0FDA3E0FE27
:2025E000A3E0FF900020161200206CD0077D6E7C00120032D7E47F107E20FDFC9000200FD3
:202600001200206C90002006E0FFC0079000200FE0FCA3E0FDA3E0FEA3E0FF9000201612CA
:2026200000206CD0077D6F7C00120032D7E47F047E08FDFC9000200F1200206C90002006BB
:20264000E0FFC0079000200FE0FCA3E0FDA3E0FEA3E0FF900020161200206CD0077D707C12
:2026600000120032D7E490002004F090002004E0FBC39404400301271DE47FFF7E01FDFC6B
:202680009000200F1200206CEB75F002A42471FDE435F0FCC004C00590002006E0FFC0076B
:2026A0009000200FE0FCA3E0FDA3E0FEA3E0FF900020161200206CD007D005D004120032D4
:2026C000D7E47FFF7EFFFDFC9000200F1200206C90002004E075F002A42471FFE435F0CFE3
:2026E0002401FDE43FFCC004C00590002006E0FFC0079000200FE0FCA3E0FDA3E0FEA3E095
:20270000FF900020161200206CD007D005D004120032D790002004E004F001266BE47F0836
:202720007E08FDFC9000200F1200206C90002006E0FFC0079000200FE0FCA3E0FDA3E0FEC5
:20274000A3E0FF900020161200206CD0077D797C00120032D7E47F1E7E14FDFC9000200F64
:202760001200206C90002006E0FFC0079000200FE0FCA3E0FDA3E0FEA3E0FF900020161269
:2027800000206CD0077D7A7C00120032D7E4FFFEFDFC9000200F1200206C90002006E0FF7C
:2027A000C0079000200FE0FCA3E0FDA3E0FEA3E0FF900020161200206CD0077D7B7C001273
:2027C0000032D7E47F207E40FDFC9000200F1200206C90002006E0FFC0079000200FE0FC62
:2027E000A3E0FDA3E0FEA3E0FF900020161200206CD0077D817C00120032D7E47F507EFA5B
:20280000FDFC9000200F1200206C90002006E0FFC0079000200FE0FCA3E0FDA3E0FEA3E0E7
:20282000FF900020161200206CD0077D827C00120032D7E4FF7E40FDFC9000200F1200203D
:202840006C90002006E0FFC0079000200FE0FCA3E0FDA3E0FEA3E0FF900020161200206C2E
:20286000D0077D8C7C00120032D7E47F11FEFDFC9000200F1200206C90002006E0FFC007BD
:202880009000200FE0FCA3E0FDA3E0FEA3E0FF900020161200206CD0077D957C001200320D
:2028A000D7E47F337E22FDFC9000200F1200206C90002006E0FFC0079000200FE0FCA3E03B
:2028C000FDA3E0FEA3E0FF900020161200206CD0077D967C00120032D7E47F557E44FDFCA0
:2028E0009000200F1200206C90002006E0FFC0079000200FE0FCA3E0FDA3E0FEA3E0FF9071
:202900000020161200206CD0077D977C00120032D7E490002007F0A3F090002007E0FAA30F
:20292000E0FBC39419EA648094804003012BF9E47F837E04FDFC9000200F1200206C9000B4
:202940002006E0FFC007EBAE027803C333CE33CED8F92400FDEE3401FCC004C00590002086
:202960000FE0FCA3E0FDA3E0FEA3E0FF900020161200206CD005D004D007120032D790005A
:202980002007E0FAA3E0FB64184A6003012A547F817E16FDFC9000200F1200206C90002076
:2029A00006E0FFC007EBAE027803C333CE33CED8F92402FDEE3401FCC004C0059000200F35
:2029C000E0FCA3E0FDA3E0FEA3E0FF900020161200206CD005D004D007120032D7E47F80B6
:2029E0007E36FDFC9000200F1200206C90002006E0FFC007A3E0FEA3E07803C333CE33CE2D
:202A0000D8F92401FDEE3401FCC004C0059000200FE0FCA3E0FDA3E0FEA3E0FF9000201637
:202A20001200206CD005D004D007120032D7E4FFFEFDFC9000200F1200206C90002006E090
:202A4000FFC007A3E0FEA3E07803C333CE33CED8F9012B1AE47FF17E17FDFC9000200F12A2
:202A600000206C90002006E0FFC007A3E0FEA3E07803C333CE33CED8F92402FDEE3401FC17
:202A8000C004C0059000200FE0FCA3E0FDA3E0FEA3E0FF900020161200206CD005D004D0B2
:202AA00007120032D7E47F807ED6FDFC9000200F1200206C90002006E0FFC007A3E0FEA3E7
:202AC000E07803C333CE33CED8F92401FDEE3401FCC004C0059000200FE0FCA3E0FDA3E09D
:202AE000FEA3E0FF900020161200206CD005D004D007120032D7E47F01FEFDFC9000200F3D
:202B00001200206C90002006E0FFC007A3E0FEA3E07803C333CE33CED8F92403FDEE34015F
:202B2000FCC004C0059000200FE0FCA3E0FDA3E0FEA3E0FF900020161200206CD005D004E5
:202B4000D007120032D7E4FFFEFDFC9000200F1200206C90002006E0FFC007A3E0FEA3E0EC
:202B60007803C333CE33CED8F92404FDEE3401FCC004C0059000200FE0FCA3E0FDA3E0FEDB
:202B8000A3E0FF900020161200206CD005D004D007120032D7E47F017E10FDFC9000200F0A
:202BA0001200206C90002006E0FFC007A3E0FEA3E07803C333CE33CED8F92405FDEE3401BD
:202BC000FCC004C0059000200FE0FCA3E0FDA3E0FEA3E0FF900020161200206CD005D00445
:202BE000D007120032D790002008E004F0700790002007E004F0012919229000201EEFF043
:202C00007B017A2079427D107C0012002EEB90002042A3A3A3E05480FFEF60037F0022909E
:202C200000201FA3A3A3E05407FFE4FEFDFC120020782C91000000012C420000000500007C
:202C40002C8E9000204EE0FCA3E0FDA3E0FEA3E0FF9000202D1200206C9000201EE0FF7DB8
:202C6000037C001200339E9000204AE0FCA3E0FDA3E0FEA3E0FF9000202D1200206C90008E
:202C8000201EE0FF7D027C001200339E80037F002290002023E0FCA3E0FDA3E0FEA3E0FFE3
:202CA0009000202D1200206C9000201EE0FF7D017C001200339E9000201FE0FCA3E0FDA341
:202CC000E0FEA3E0FF9000202D1200206C9000201EE0FFE4FDFC1200339E9000201EE0FFFF
:202CE0007B017A2079427D107C0012002EEB90002042A3A3A3E05480FFEF70DE9000201F35
:202D0000A3A3A3E05478FFE4FEFDFC78031200202B120020782D43000000002D57000000CE
:202D2000012D6B000000032D6B000000042D6B000000052D6B000000062D6B000000070081
:202D4000002D819000201EE0FF7B017A2079527D047C0012002EEB9000201EE0FF7B017A6C
:202D600020794E7D037C0012002EEB9000201EE0FF7B017A20794A7D027C0012002EEB8019
:202D8000037F00227F012290002021EFF07B017A2079427D107C0012002EEB90002042A3A3
:202DA000A3A3E05480FFEF60037F002290002022A3A3A3E05407FFE4FEFDFC120020782D80
:202DC000D8000000022DD8000000042DD80000000600002DD57F002290002022A3A3A3E0C7
:202DE0005478FFE4FEFDFC78031200202B120020782E19000000002E36000000012E53007E
:202E00000000032E53000000042E53000000062E530000000700002E7A90002052E0FCA3F2
:202E2000E0FDA3E0FEA3E0FF9000202D1200206C7D04120033969000204EE0FCA3E0FDA3DE
:202E4000E0FEA3E0FF9000202D1200206C7D03120033969000204AE0FCA3E0FDA3E0FEA3C2
:202E6000E0FF9000202D1200206C90002021E0FF7D027C001200339E80037F002290002096
:202E800026E0FCA3E0FDA3E0FEA3E0FF9000202D1200206C90002021E0FF7D017C00120076
:202EA000339E90002022E0FCA3E0FDA3E0FEA3E0FF9000202D1200206C90002021E0FFE401
:202EC000FDFC1200339E90002021E0FF7B017A2079427D107C0012002EEB90002042A3A329
:202EE000A3E05480FFEF70DE7F01229000202AEFF0A3ECF0A3EDF0A3EBF0A3EAF0A3E9F06E
:202F0000E4A3F0A3F0E4FFFEFDFC9000203E1200206C9000202BE0FCA3E0FD9000202AE050
:202F2000FF120031F29000202AE0FFE4FD1200348CE0FF0D120034DFE0FF120032CAE0FF14
:202F4000E4FD120034DFE4FFFEFC900020371200206CE490002032F0120034AC12003267B6
:202F600090002032E004F0E0C3942040EB90002037E0FCA3E0FDA3E0FEA3E0FF9000202DF6
:202F8000E0FBA3E0FAA3E0F912002051E4FFFEFDFC900020371200206CE490002032F012B3
:202FA0000034AC1200326790002032E004F0E0C3940940EB90002037A3A3E0FEA3E0FBEEEE
:202FC000FAE4F9F89000202BE0FEA3E0FFE4FCFDC31200201A601E90002030E475F0011241
:202FE000002004FED3741E95F0EE6480F87480984003012F0522E490002000F0A3F090002E
:203000002000E0FEA3E0FFC39402EE9400505BEF2404FFE43EFE1200317090002002EEF031
:20302000A3EFF0E0FD90002001E025E0FB90002000E033FA74562BF58274203AF583759329
:2030400000EDF090002002E0FF74572BF58274203AF583759300EFF090002001E004F07073
:203060009D90002000E004F08094E490002000F0A3F090002000E0FEA3E0FFC39403EE9418
:203080000050541200317090002002EEF0A3EFF0E0FD90002001E025E0FB90002000E03396
:2030A000FA745A2BF58274203AF583759300EDF090002002E0FF745B2BF58274203AF58333
:2030C000759300EFF090002001E004F070A490002000E004F0809B020020C490002006EE47
:2030E000F0A3EFF0900020647408F0F5C84402F0F5C87F327E00120034D290002064E044AF
:2031000004F0F5C87F647E00120034D2120034C4900020627408F0A3E4F090002062E0FC98
:20312000A3E0FD4C6043A3E054FAF090002006E0FEA3E0FFEC5EFEED5F4E600890002064EB
:20314000E04404F090002064E0120034CC120034CE90002064E04401F0F5C890002062E065
:20316000C313F0A3E013F080B190002064E0FF22C2AFEE4408FE120030DB90002064EFF004
:20318000E490002004F0A3F0900020627480F0A3E4F090002062E07002A3E0603790002079
:2031A00064E054FA120034CB120034C4AFC8EF30E31490002062E0FEA3E0FF90002004E0CF
:2031C0004EF0A3E04FF090002062E0C313F0A3E013F080BE90002064E054F8F0F5C87F9077
:2031E0007E01120034D2D2AF90002004E0FEA3E0FF229000203CECF0A3EDF0AB07E4FA1297
:20320000003477120032CA9000203EE0FCA3E0FDA3E0FEA3E0FF78011200202B9000203EE4
:203220001200206C0AEAB420D69000203CE0FEA3E0FFE4FCFDA31200206CE4FA120034774D
:20324000120032CA9000203EE0FCA3E0FDA3E0FEA3E0FF78011200202B9000203E1200201D
:203260006C0AEAB409D622E4FCFDFE900020331200206C90002033E0FCA3E0FDA3E0FEA37A
:20328000E0FF90002032E0F9F81200203EA31200206C90002037E0FCA3E0FDA3E0FEA3E0A4
:2032A000FF90002033E0F8A3E0F9A3E0FAA3E0FBEF4BFFEE4AFEED49FDEC48FC9000203724
:2032C0001200206C9000202AE0FFAE077D01120034D91D020034D990002013EFF0A3ECF0F8
:2032E000A3EDF0C3EC94015027A3E0FCA3E0FDA3E0FEA3E0FF9000202D1200206C90002066
:2033000014E0FCA3E0FD90002013E0FF0200339E90002016E0FCA3E0FDA3E0FEA3E0FF9013
:2033200000201D1200206C90002014E0FCA3E0FD90002013E0FF120034332290002019ECA0
:20334000F0A3EDF0A3EBF0A3EAF0A3E9F0C007E47F21FEFDFC9000201F1200206C90002027
:2033600019E0FEA3E0FFE4FCFD900020231200206CD00712002BFA9000204AE0FCA3E0FD22
:20338000A3E0FEA3E0FF9000201BE0FBA3E0FAA3E0F90200205190002021E0FF7C0090005C
:2033A000202AEFF0C007C004C0059000202DE0FCA3E0FDA3E0FEA3E0FF9000203E12002038
:2033C0006CD005D004D007120031F29000202AE0FFE4FD1200348CE0FF0D120034E5E0FF6A
:2033E0001D020034E590002013EFF090002016EBF0A3EAF0A3E9F090002014ECF0A3EDF039
:20340000C3EC940190002013E0FF5013A3E0FCA3E0FDA3E0FBA3E0FAA3E0F902002EEBA32F
:20342000E0FCA3E0FDA3E0FBA3E0FAA3E0F91200333B22AB05AA04A9079000201DE0FCA3BD
:20344000E0FDA3E0FEA3E0FF9000204A1200206CAF01C007E47F22FEFDFC9000202212001D
:20346000206CAE02AF03E4FCFD900020261200206CD00702002D879000203EE0FCA3A3E090
:20348000FEA3E05401FFA907AF03AD01ED24FF929122AE07E4FD1200348C0D120034D31D47
:2034A000120034D9120034DF020034E59000202AE0FFA290E4339000203BF09000203BE005
:2034C0005401FF2290002064E04401F0F5C87FF47E0122ED24FF929022ED24FF929222EDE5
:2034E00024FF929522ED24FF929322FFFFFFFFFFFFFFFFFFFFFFFFFFFFFFFFFFFFFFFFFF1E
:20350000FFFFFFFFFFFFFFFFFFFFFFFFFFFFFFFFFFFFFFFFFFFFFFFFFFFFFFFFFFFFFFFFCB
:20352000FFFFFFFFFFFFFFFFFFFFFFFFFFFFFFFFFFFFFFFFFFFFFFFFFFFFFFFFFFFFFFFFAB
:20354000FFFFFFFFFFFFFFFFFFFFFFFFFFFFFFFFFFFFFFFFFFFFFFFFFFFFFFFFFFFFFFFF8B
:20356000FFFFFFFFFFFFFFFFFFFFFFFFFFFFFFFFFFFFFFFFFFFFFFFFFFFFFFFFFFFFFFFF6B
:203F0000120020C022FFFFFFFFFFFFFFFFFFFFFFFFFFFFFFFFFFFFFFFFFFFFFFFFFFFFFFA8
:203F2000FFFFFFFFFFFFFFFFFFFFFFFFFFFFFFFFFFFFFFFFFFFFFFFFFFFFFFFFFFFFFFFFA1
:203F4000FFFFFFFFFFFFFFFFFFFFFFFFFFFFFFFFFFFFFFFFFFFFFFFFFFFFFFFFFFFFFFFF81
:203F6000FFFFFFFFFFFFFFFFFFFFFFFFFFFFFFFFFFFFFFFFFFFFFFFFFFFFFFFFFFFFFFFF61
:203F8000FFFFFFFFFFFFFFFFFFFFFFFFFFFFFFFFFFFFFFFFFFFFFFFFFFFFFFFFFFFFFFFF41
:208000000200A12CE4FFEF24FF9291220201C25C02000000020239593098FDAF99C2987EB9
:208020000022322202008022EB7008E709F608DFFA801B89828A831410E70AF593E0A3F633
:2080400008DFFA8009F593E493A3F608DFF9ECFAA9F0EDFB2288F0EF60010E4E60F088F0C9
:20806000ED60C51410E7E7CB700E88828C838B93E709F0A3DFFA80D61410E72A89828A837D
:20808000F593ECFAE0A3C8C582C8CCC583CCCBC593CBF0A3C8C582C8CCC583CCCBC593CB12
:2080A000DFE2DEE080AA89828A83F593ECFAE493A3C8C582C8CCC583CCCBC593CBF0A3C877
:2080C000C582C8CCC583CCCBC593CBDFE1DEDF02008050EB7002E72289828A831410E704E7
:2080E000F593E022F593E49322F8EB7006E7C828F3E82289828A831410E708F593E0C82825
:20810000F0E822F593E49322BB000327F722F8EB89828A831410E706F593E028F022F59310
:20812000E4932822BB0002F722BB8000500989828A838B931593F022EF8DF0A4A8F0CF8C21
:20814000F0A428CE8DF0A42EFE22C2D5EC30E709B2D5E4C39DFDE49CFCEE30E716B2D5E4B9
:20816000C39FFFE49EFE12008878C3E49DFDE49CFC80041200887830D507C3E49FFFE49EE6
:20818000FE22C5F0F8A3E028F0C5F0F8E582158270021583E038F022A3F8E0C5F025F0F063
:2081A000E582158270021583E0C838F0E822EB7007E7F5F009E7192289828A831410E70859
:2081C000F593E0F5F0A3E022F593E493F5F074019322F8EB700C09E5F027C7F5F019E83757
:2081E000C72289828A831410E707F593E802008198F593E4740193F5F0E49322BB000B0920
:20820000C5F027F7C5F01937F722F8EB89828A831410E707F593E802008182F5937401935B
:2082200025F0F5F0E4933822BB0006F709A7F01922BB8000500D89828A838B931593F0E595
:20824000F0A3F022E88FF0A4CC8BF0A42CFCE98EF0A42CFC8AF0EDA42CFCEA8EF0A4CDA874
:20826000F08BF0A42DCC3825F0FDE98FF0A42CCD35F0FCEB8EF0A4FEA9F0EB8FF0A4CFC540
:20828000F02ECD39FEE43CFCEAA42DCE35F0FDE43CFC2275F008758200EF2FFFEE33FECD4A
:2082A00033CDCC33CCC58233C5829BED9AEC99E58298400CF582EE9BFEED9AFDEC99FC0F2E
:2082C000D5F0D6E4CEFBE4CDFAE4CCF9A88222B800C1B90059BA002DEC8BF084CFCECDFCF3
:2082E000E5F0CBF97818EF2FFFEE33FEED33FDEC33FCEB33FB10D703994004EB99FB0FD89B
:20830000E5E4F9FA227818EF2FFFEE33FEED33FDEC33FCC933C910D7059BE99A4007EC9BDE
:20832000FCE99AF90FD8E0E4C9FAE4CCFB2275F010EF2FFFEE33FEED33FDCC33CCC833C82E
:2083400010D7079BEC9AE899400AED9BFDEC9AFCE899F80FD5F0DAE4CDFBE4CCFAE4C8F91A
:2083600022CFF4CFCEF4CECDF4CDCCF4CC22EB9FF5F0EA9E42F0E99D42F0E89C45F022E8D9
:20838000600FECC313FCED13FDEE13FEEF13FFD8F122E8600FEFC333FFEE33FEED33FDEC65
:2083A00033FCD8F122EB7006E9F8020088DC89828A831410E706F593020088E8F59302004E
:2083C00088F4BB0006E9F80200892DBB8000500C89828A838B9315930200842F22EB70061A
:2083E000E9F80200890489828A831410E706F59302008911F5930200891D7401FF3395E074
:20840000FEFDFCA3A3A3E02FFFF0E582158270021583E03EFEF0E582158270021583E03D45
:20842000FDF0E582158270021583E03CFCF022ECF0A3EDF0A3EEF0A3EFF022A42582F582DA
:20844000E5F03583F58322EB7006E9F80200893989828A831410E706F5930200894BF593E0
:208460000200898BBB001CD093D0F0D0E0F8D0E0C9FBD0E0FAD0E0CBC8C0E0C0F0C093023E
:20848000008942BB80005022D093D0F0D0E0F8D0E0C9F582D0E0CAF583D0E0CB14C8C0E0C0
:2084A000C0F0C093889302008982D093D083D082D0E0D0E0D0E0E473D093D083D082F8E43E
:2084C000937012740193700DA3A393F8740193F5828883E4737402936860EFA3A3A380DF48
:2084E000D093D083D082F8E4937012740193700DA3A393F8740193F5828883E47374029343
:20850000B5F0067403936860E9A3A3A3A380D88B938A838982159353937FE473EB700C8789
:20852000F009E608B5F041603F80F489828A831410E70FF593E0F5F0A3E608B5F02A6028F4
:2085400080F3F593E493F5F0A3E608B5F01A601880F2CB701588828C838B9387F009E4930C
:20856000A3B5F004600280F380611410E72E89828A83F593ECFAE0F5F0A3C8C582C8CCC56A
:2085800083CCCBC593CBE493A3C8C582C8CCC583CCCBC593CBB5F033603180DA89828A8304
:2085A000F593ECFAE493F5F0A3C8C582C8CCC583CCCBC593CBE493A3C8C582C8CCC583CCD8
:2085C000CBC593CBB5F004600280D97F00F845F0600EE863F0806480D395F01F40027F0157
:2085E000220200851C02008552ED60F51410E7F5CB701488828C83F59387F009E0A3B5F003
:20860000CA60C880F480C41410E72D89828A83F593ECFAE0F5F0A3C8C582C8CCC583CCCB08
:20862000C593CBE0A3C8C582C8CCC583CCCBC593CBB5F097609580DB89828A83F593ECFADD
:20864000E493F5F0A3C8C582C8CCC583CCCBC593CBE0A3C8C582C8CCC583CCCBC593CBB599
:20866000F0A360A180DAEB7008E709F60870FA801B89828A831410E70AF593E0A3F6087010
:20868000FA8009F593E493A3F60870F9ECFAA9F0EDFB2288F0ED60CE1410E7F0CB700E8866
:2086A000828C83F593E709F0A370FA80DF1410E72889828A83F593ECFAE0A3C8C582C8CC76
:2086C000C583CCCBC593CBF0A3C8C582C8CCC583CCCBC593CB70E280B589828A83F593EC4D
:2086E000FAE493A3C8C582C8CCC583CCCBC593CBF0A3C8C582C8CCC583CCCBC593CB70E138
:20870000808CEB700C87F009E608B5F019DFF6801589828A831410E711F593E0F5F0A3E646
:2087200008B5F002DFF5020087B3F593E493F5F0A3E608B5F07DDFF48079CB701388828C33
:20874000838B9387F009E493A3B5F067DFF580631410E73089828A83F593ECFAE0F5F0A3F2
:20876000C8C582C8CCC583CCCBC593CBE493A3C8C582C8CCC583CCCBC593CBB5F035DFDC00
:20878000DEDA802F89828A83F593ECFAE493F5F0A3C8C582C8CCC583CCCBC593CBE493A32E
:2087A000C8C582C8CCC583CCCBC593CBB5F004DFDBDED97FFFB5F0020F2240027F012202BE
:2087C0000087020200873A88F0EF60010E4E60EEED60EC1410E7ECCB701288828C83F593BD
:2087E00087F009E0A3B5F0CBDFF680C71410E72F89828A83F593ECFAE0F5F0A3C8C582C8EB
:20880000CCC583CCCBC593CBE0A3C8C582C8CCC583CCCBC593CBB5F09ADFDDDEDB80948911
:20882000828A83F593ECFAE493F5F0A3C8C582C8CCC583CCCBC593CBE0A3C8C582C8CCC5AC
:2088400083CCCBC593CBB5F004DFDCDEDA020087B3EF4E6022EF60010EEDBB0007F709DFD8
:20886000FCA9F022BB8000500E89828A838B931593F0A3DFFCDEFA22BC000BBE0029EF8D38
:20888000F084FFADF022E4CCF875F008EF2FFFEE33FEEC33FCEE9DEC984005FCEE9DFE0F52
:2088A000D5F0E9E4CEFD22EDF8F5F0EE008420D21CFEADF075F008EF2FFFED33FD400798CE
:2088C0005006D5F0F222C398FD0FD5F0EA22C3E49FFFE49EFEE49DFDE49CFC22E6FC08E680
:2088E000FD08E6FE08E6FF22E0FCA3E0FDA3E0FEA3E0FF22E493FC740193FD740293FE740C
:208900000393FF22E6FB08E6F908E6FA08E6CBF822E0F8A3E0F9A3E0FAA3E0FB22E493F83D
:20892000740193F9740293FA740393FB22ECF608EDF608EEF608EFF622E6FB08E6FA08E68D
:20894000F922EBF608EAF608E9F622E0FBA3E0FAA3E0F922F8E0FBA3A3E0F925F0F0E582D6
:20896000158270021583E0FA38F022F8E0FBA3A3E025F0F9F0E582158270021583E038FA21
:20898000F022EBF0A3EAF0A3E9F022E493FB740193FA740293F922706F72743D00706F72E4
:2089A000743D253032640073706565643D0073706565643D2564007365745F666C6F773D56
:2089C000007365745F666C6F773D2564007365745F716F733D007365745F716F733D25646F
:2089E000006367695F736574706F72743D256400506F72742053657474696E67004D656455
:208A000069612074797065206973206368616E6765642E3C62723E43757272656E742073D2
:208A2000706565642073657474696E67206973206E6F74207375697461626C652E00766C84
:208A4000616E5F69643D00766C616E5F69643D256400646573633D0026006367695F766CC5
:208A6000616E00564C414E2053657474696E6700564C414E206465736372697074696F6E03
:208A8000206D75737420626520756E6971756500564C414E206E616D65206D7573742062F2
:208AA0006520302D25642063686172616374657273007663623D007663623D253032640030
:208AC0006367695F736574766C616E3D256400496620616E7920706F727420696E206120AD
:208AE000564C414E2047726F75702062656C6F6E677320746F2061207472756E6B2C207476
:208B0000686520564C414E2047726F7570206D75737420696E636C75646520616C6C207034
:208B20006F72747320696E2074686174207472756E6B2E006E756D3D006E756D3D25640080
:208B40007663623D2564006367695F64656C766C616E0076747970653D0076747970653DB2
:208B600025640044656661756C74007379733D006C6F633D006C6F67696E3D005379737487
:208B8000656D206E616D65206D75737420626520302D25642063686172616374657273002C
:208BA00053797374656D2053657474696E67006367695F737973004C6F636174696F6E20E8
:208BC0006E616D65206D75737420626520302D2564206368617261637465727300496E76B1
:208BE000616C6964206C6F67696E2074696D656F75742076616C75650069703D00496E76FB
:208C0000616C69642049502041646472657373006D6B3D00496E76616C6964205375626E87
:208C20006574204D61736B0067773D00496E76616C696420476174657761792049500049D9
:208C400050207375626E6574206D75737420626520657175616C20746F206761746577616F
:208C600079207375626E65742E006F6C645F706173733D006E65775F706173733D00726596
:208C80006E65775F706173733D004368616E67652050617373776F72640050617373776F01
:208CA0007264206C656E6774682063616E2774206265207A65726F2E006367695F70617384
:208CC000730050617373776F7264206D75737420626520302D25642063686172616374659D
:208CE0007273004F6C642070617373776F72642069732077726F6E672E004E65772070614B
:208D00007373776F726420697320696E636F6E73697374656E742E007425643D0025303285
:208D200064005472756E6B2053657474696E6700416C6C20706F72747320696E20746865F4
:208D4000207472756E6B206D7573742062656C6F6E6720746F207468652073616D6520569F
:208D60004C414E2873292E006367695F7472756E6B006D6F64653D006D6F64653D25303215
:208D80006400736E69666665723D00736E69666665723D2530326400736F757263653D0062
:208DA000736F757263653D2530326400547261702053657474696E6700496E76616C69649E
:208DC0002054726170204950006367695F74726170006669623D00636F703D00257325250B
:208DE0006400647669643D00505649442053657474696E6700496E76616C69642056494430
:208E00002076616C7565006367695F7076696400647072693D00496E76616C69642050723B
:208E2000696F726974792076616C7565005649442025303264206973206E6F742065786994
:208E400073742C206F7220506F72742025303264206973206E6F7420746865206D656D629F
:208E60006572206F662056494420253032642E00276367695F7076696427007669643D00D7
:208E80005649442053657474696E67005649442076616C7565206D7573742062652062651A
:208EA000747765656E203220616E642034303934006367695F6164647669640054686520BA
:208EC000564944207461626C65206861732066696C6C65640054686520564944206973205B
:208EE000657869737420696E20564944207461626C65007025643D002564007461675F6960
:208F0000643D007461675F69643D2564005468652064656661756C7420564944206F662044
:208F2000706F727420253032642069732025642C20736F2069742063616E206E6F7420624C
:208F40006520756E73656C65637465642E00276367695F7365747669643D25642700546841
:208F60006520564944206973207468652064656661756C7420564944206F6620706F72744A
:208F800020253032642C20736F2069742063616E206E6F742062652064656C657465642ECC
:208FA000006367695F7365747669643D25640052656D6F766520564C414E007061737377DD
:208FC000643D00716F73747970653D00716F73747970653D25640070253032643D001021FA
:208FE0000D12008018BF0D027F0A0200A39690082BCCE0FF2290082BCCEFF0D22122FFFF17
:209000000180C200000F3C74723E3C746820636F6C7370616E3D343E25730A3C74723E0ABB
:20902000203C74643E3C623E42797465730A203C746420636F6C7370616E3D333E256C75D9
:209040000A0A003C74723E0A203C74643E3C623E25730A203C74643E256C750A203C7464EC
:209060003E3C623E25730A203C74643E256C750A0A008383FB8384038384068384097663A7
:209080006200203C74643E0A203C73656C656374206E616D653D25733E0A203C6F70746920
:2090A0006F6E2076616C75653D25643E25730A000A3C7472206865696768743D33303E0A43
:2090C000203C746420616C69676E3D63656E7465723E3C623E25730A203C74643E3C623E69
:2090E0000A0083A7F283A80083A80E83A82183A83583A84C20203C696E707574207479709A
:20910000653D636865636B626F78206E616D653D25732076616C75653D25642025733E20B7
:2091200025733C62723E0A004825810102040810204080412BBB01422523000A42252B0004
:209140000042251F0000422521000042251B000042252D0000422525FFFF42251D8000421B
:209160002515000042251700004225190000C11F421FBD0000421FBF000042246F00005272
:2091800026A7837FCC837FD8837FE9837FFB837FE9837FFB4C27FF838AE1838AE9838AEC3B
:2091A000838AEF603022A083A2CB83A2D283A2DF83A2DF83A2E183A2E883A2F583A2F583A8
:2091C000A2F783A2FE83A30B83A30B83A30B83A30B83A30B83A30B58236983606983607129
:2091E00083607B83608583608E83609783609C8360A446235D83609C8360A9462363836038
:20920000B08360B44623578360B78360BE6040218300081018202830380A121A220C141C54
:20922000240E161E262E01020304050607090B0D0F11131517191B1D1F21232527292A2B5A
:209240002C2D2F31323334353637393A3B3C3D3E3F4C263C83AA7783AA7E83AA8283AA8914
:2092600049263383AA8E83AA9983AAAB462A8D83AF5083AF5749298283971F839727839763
:209280002C4320FD0000006256040A833EA86367695F64756D7900000000000000000000C2
:2092A000000082A5206367695F6C6F67696E00000000000000000000008305636367695F3F
:2092C000706F727400000000000000000000000081E3786367695F736574706F727400004A
:2092E000000000000000008303A56367695F766C616E0000000000000000000000008297E7
:20930000096367695F736574766C616E0000000000000000008260DA6367695F64656C76BC
:209320006C616E00000000000000000082F8F96367695F707669640000000000000000003A
:209340000000008200076367695F76696400000000000000000000000000825A256367697B
:209360005F6164647669640000000000000000000081D18E6367695F646576696365000040
:20938000000000000000000081C3BA6367695F64657461696C000000000000000000008248
:2093A0003C4F6367695F737461746973740000000000000000008282186367695F7472757B
:2093C0006E6B00000000000000000000008218536367695F6D6972726F720000000000009A
:2093E00000000000829E476367695F7061737300000000000000000000000081F1B96367C8
:20940000695F73797300000000000000000000000000820C8E6367695F74726170000000C0
:20942000000000000000000000832F896367695F6261636B757000000000000000000000E9
:2094400082CC3A6367695F62616B5F646174610000000000000000832FD66367695F7265DA
:209460007365740000000000000000000000833B936367695F716F7300000000000000006A
:20948000000000000082FEFF6367695F7170626173650000000000000000000082FD0D6350
:2094A00067695F716473637000000000000000000000008300F96367695F71317000000042
:2094C00000000000000000000000000000000000000000000000000000000000000000008C
:2094E00000422B5400004215DA00004214C000004614BA819FD1819FDF5215C281A007818E
:20950000A01E81A03481A04A81A06281A07E4615D481A09B81A0B84213B000004219820005
:209520000100E52524FFF582E43423F583759308E0052522900823FC301704900823FFE4F7
:2095400075F00112008954020080D32010E57F2ED2108018EF540F2490D43440D4FF3014C0
:209560000BEF24BFB41A0050032461FFE526600215260529E52970020528301711900823D3
:20958000FCE475F00112008954EF020081240200A3967403D2178003E4C217F52590082350
:2095A000FC12008982E4F526F528F529E52660087F201200956C80F47527FFC211C210C2BD
:2095C00012C213C215C216C21812009534FF700E3017067F001200957DAF29AE2822B4252A
:2095E00063C2D5C21412009534FF24D0B40A00501A75F00A782630D50508B6FF0106C6A460
:2096000026F620D5047002D21380D824CFB41A00EF5004C2E5D214020097AAD21180C4D2B9
:209620001080BED21280BAD2D580B8D21580B27F201200956C2012077401B5260040F01249
:20964000009522FF1200956C020095ACD218D216808F12009522FB12009522FA12009522CD
:20966000F94A4B700679817A987B8120123DE52660397E00E9C0E02EF9EAC0E03400FA12D3
:209680000080D3F9D0E0FAD0E0C960060EEE652770E2C2D5EBC0E0EAC0E0E9C0E0EE1200E6
:2096A00097F2D0E0F9D0E0FAD0E0FB120080D3FF6096EBC0E0EAC0E0E9C0E01200956CD048
:2096C000E02401F9D0E03400FAD0E0FBE5270460DAD527D7020096487BFF7A9779EED21230
:2096E0008089791080027908C216C2188008D2D5790A8004790AC2D5E527047002F527E451
:20970000FAFDFEFF12009522FC7B0820111612009522FD7B1030100C12009522FE120095BB
:2097200022FF7B20EC3382D592D55013C3E43010069FFFE49EFEE42011039DFDE49CFCE410
:20974000CBF8C211EC700CCFCECDCCE824F8F870F38017C3EF33FFEE33FEED33FDEC33FCA4
:20976000EB33FB994002FB0FD8E9EB301105F8D0E0C448B211C0E00AEC4D4E4F78207B00EF
:2097800070C2EAB5270040BCC0E0120097F4D0F0D0E0201104C4C0E0C4B211C0F0120095B1
:2097A00055D0F0D5F0EA020095AC120084B896525396E258961F4C961B4296E64F96EE44C2
:2097C00096EE4996354396F45596D84696D84596D847989E5096232D96272E964E2B962B8C
:2097E00023964C20988A2A95E148000096443F3F3F00790AA2D5201314301509B910020445
:2098000004B9080104A2D520160250010420126D9212B526005036C0E07F2030131A7F308B
:20982000A2127216721550101200984DC212C216C215C2187F308010301503E9C0E012008F
:20984000956C301503D0E0F9D0E0B526CA3015197F30B9100D1200956C7F583014077F78B2
:209860008003B908041200956C3012067F2D0200956C7F202018F77F2B2016F222921280B0
:20988000CC286E756C6C2900D211120095223011F7C211782630D50108F6020095E112000D
:2098A00095227F4960087F4310E7027F5814C0E0EF1200955D743A1200955DD0E0600DC0F9
:2098C000E0C412009555D0E012009555D213752604020096E2E52A301C0104F82328240176
:2098E000F582E43423F58375930822900822FE301C0490082301E475F0011200895402000D
:2099000080D360E6C52E7002152D14C52E201C05FF02008FF5900822FE74FFF5F00200899F
:209920006BFF02023C34E52B6006D52B037F0022201C1012008FDEEF6008052EE52E700255
:20994000052D22900822FE1200894B120080D3FF60E5900822FEE475F0011200895480D724
:2099600012009930EFC0E012009921D0E040F18091D21C8002C21C900822FE12008982E4B8
:20998000F52CF52AF52DF52E752B00C21BC219C21AC21D120098EBFF7005AF2C7E0022B4F7
:2099A0002532120098EBFF24D0B40A00500C75F00AC52BA4252BF52B80E824CFB41A00EF23
:2099C0005002C2E502009C0BD21A80D6D21980D2D21D80CEEF12009921500912009960EF1B
:2099E000600F80A4EFC0E012009930D0E06F6098EF700402009A7B12009902809D12009964
:209A000030EF6077E52B7008052B800412009930EF6017201D11120098D5E475F0011200AA
:209A20008954EF12008124D52BE2201D04052A052C80AF12009926EFC0E012009921D0E015
:209A4000500512009902E4FF201D11120098D5E475F00112008954EF12008124EF70D42022
:209A60001D04052A052C020099E2E52B6002052B1200996012009926EF70BD301C05E41207
:209A8000009902E52C60030200999A7EFF7FFF22201D1474FFFCFDFEFF120098D512008991
:209AA0004B120083C2052A02009988D0E080CC7900800A7910800679088002790AD21EE549
:209AC0002B6002052BE9C0E012009960EF60DC12009930BF2D04D21B8003BF2B0B1200992F
:209AE00060EF60C712009926D0E0B40A028034B40802802FBF302870027408C21EC0E012F7
:209B0000009926D0E0BF78028003BF5816052BD52B028007D52B04D21E800B7410801B7026
:209B200002740ABF000BEFF8E4FCFDFEFF02009BB3C0E0EF12009902D0E0F9E4FCFDFEFF0B
:209B4000E9C0E0ECC0E0EDC0E0EEC0E0EFC0E012009926EFF8D0E0FFD0E0FED0E0FDD0E0D4
:209B6000FCD0F0E8604DB461004007B47B005002C2E524D0503DFA24F6500724F95034245F
:209B80000AFAEAB5F000502BCFA9F0A42FFF92D5E9C5F0CEA4A2D53EFE92D5E9C5F0CDA4DD
:209BA000A2D53DFD92D5E9C5F0CCA4A2D53CFCC21E808DE8C0E0201D30201E09052C301B2B
:209BC00004120088CE120098D51200894B052A20190C201A0FEE8FF012008228800B120031
:209BE00083C28005EF12008124D0E01200990202009988201D13120098D51200894B052A91
:209C0000E52D852EF01200822880E4120084B89A6A539AB35899CC4C99C84299A2489AB7FD
:209C20004F9ABB4499FD439AAF499ABB559A90469A90459A904799D02A9BF34E000099D4FB
:209C400090007004E0F54090007005E0F541854082854183E020E7077E007F00C2D7228911
:209C6000428A435407F54512009E3BE02402F5445002054512009CE2053AE53A7002053BDA
:209C8000E5402544F540E541354530E604C2E62418F54112009D0290007004E540F09000D3
:209CA0007005E541F0AE45AF44D2D72290007010E020E61EA3EDF0A3E9F0A3EAF0EC540794
:209CC000D2E690007010F00538E53870020539D2D7227C007D00C2D72290007010E0A2E6CB
:209CE000B32275F001800375F00412009D0278407F069000709212009E2390007090E5F085
:209D0000F02290007090E0540770F72212009D6F900070087418F09000701075081012008C
:209D20009D5AE490007004F090007006F0741890007005F090007007F0751D10751C10752E
:209D40001E00751F18758318758200E4F0753800753900753A00753B0022E4A808F0A3D883
:209D6000FC2212009E1912009D0C12009DAD2290009DA375080A7970786012009E2A751844
:209D8000C07519A8751A00751B647510C07511A87512007513017514FF7515FF7516FF75B7
:209DA000170022000B78667788C0A800649000706AE0440CF0229000706AE054F3F02290D7
:209DC00000706AE04401F0229000706AE054FEF0229000706AE04402F0229000706AE05484
:209DE000FDF0229000706AE04440F0229000706AE054BFF02290007000E04410F02290002F
:209E00007000E054EFF02290007000E04420F02290007000E05420F0229000700AF00000E7
:209E2000000022E6F008A3DFFA2289A0E493A3F208B800030989A0D508F222A3E58330E648
:209E400003758318224745542000696E6465782E68746D00706F73745F75726C3D002E005B
:209E60006367695F6C6F676F757400636F6E6669672E62696E006367695F62616B5F6461F5
:209E80007461006367695F006367695F6C6F67696E004C6F67696E004F6E6C79206F6E65B3
:209EA00020757365722063616E206C6F67696E006367695F6465766963650077726F6E6709
:209EC0002070617373776F7264006C6F67696E2074696D656F7574006367695F706F727458
:209EE000006367695F716F73006367695F717062617365006367695F713170006367695F39
:209F00007164736370006367695F64656C766C616E006367695F766C616E006367695F7465
:209F200072756E6B006367695F6D6972726F72006367695F737973006367695F70617373FA
:209F4000006367695F74726170006367695F7365747674797065006367695F70766964005D
:209F60006367695F736574766964006367695F766964006367695F61646476696400636723
:209F8000695F64656C766964006367695F7265736574006367695F636C72737461740063DA
:209FA00067695F73746174697374006367695F616464766C616E006367695F736574766C3A
:209FC000616E006367695F7365747669643D25640053797374656D20626F6F747570004C41
:209FE0006F67696E20696E76616C69642070617373776F72642066726F6D2025642E2564E6
:20A000002E25642E256400506F727420256420666962657220696E73657274656400506F1F
:20A0200072742025642066696265722072656D6F76656400506F7274202564206669626553
:20A0400072206C696E6B20757000506F7274202564206669626572206C696E6B20646F770D
:20A060006E00506F72742025642066696265722072656365697665206572726F7200506FF0
:20A080007274202564206669626572207472616E736D6974206572726F7200506F72742068
:20A0A000256420636F707065722072656365697665206572726F7200506F727420256420B3
:20A0C000636F70706572207472616E736D6974206572726F72005553526F626F746963732E
:20A0E0002031302F3130302F31303030204D6270732032342D506F727420536D61727420DE
:20A1000053776974636820202020202020202020202020202020202020202020202020208D
:20A1200020202020202000282564290075C7AA75C755759D0275C7AA75C75575C600787F51
:20A14000E4F6D8FD75814FD20D0200A1770201A0A5E493A3F85407240CC8C333C4540F4404
:20A1600020C8834004F456800146F6DFE4800C010204081020408090009128E47E0193603C
:20A18000CCA3FF543F30E509541FFEE493A360010ECF54E0B4E026E493FBA3E493FAA3E4DC
:20A1A00093F9A3E493C083C08212008124D082D083A309E970010ADFEADEE880BE54C02502
:20A1C000E0602B408CE493A3FAE493A3F8E493A3C8C582C8CAC583CA759308F0759300A3AA
:20A1E000C8C582C8CAC583CADFE3DEE1808DE493A3F8E493A34003F68001F208DFF4020069
:20A20000A17B68656C6C6F3F3F3F0068696869232323006D616320777269746500676F20D4
:20A220006C6F6164657200636C6F7365746D006D61632072656164002573006D6163006D8D
:20A240006F64656C2072656164006D6F64656C3A00555352393937373234006677766572E9
:20A2600020726561640066777665723A00322E30302E30385F3131303900726263686B0034
:20A280004661696C004F6B005553526F626F746963732031302F3130302F31303030204DFD
:20A2A0006270732032342D506F727420536D61727420537769746368202020202020202048
:20A2C000202020202020202020202020202020202020202020202020000012233445FE25AD
:20A2E00073005553526F626F746963732031302F3130302F31303030204D62707320323495
:20A300002D506F727420536D617274205377697463682020202020202020202020202020F2
:20A3200020202020202020202020202020202020202000696E6465782E68746D006C656617
:20A34000742E68746D00746F702E68746D0062756C6C65742E67696600666F726D2E6373A4
:20A3600073006C6F676F2E676966000A454550524F4D2052656D61696E65642053697A6583
:20A380003A2025640A00496E69742066696E69736865642E0A00EFB40A08740D1200A3A20D
:20A3A000740A309811A899B8130CC2983098FDA899C298B811F63099FDC299F59922E4FF01
:20A3C000FE120080D3600C0FEF70010E09E970F10A80EE2244656661756C740061646D69E4
:20A3E0006E00EF6402600301A59390081A69F0A3F090081A66E0FBA3E0FAA3E02415F9E457
:20A400003AFA120080D3FFB4073090081A66A3E0FAA3E02416F9E43AFA740112008108D373
:20A420009405500301B54490081A66A3E0FAA3E02415F9E43AFAE401B540EFB40522900898
:20A440001A66E0FBA3E0FAA3E02416F9E43AFA740112008108D39405500301B54401A58C5B
:20A4600090081A66E0FBA3E0FAA3E02415F9E43AFA120080D3FF700301B54420E40301A521
:20A480003890081A66A3E0FAA3E02416F9E43AFA74FF12008108600301B54412020B2B90DC
:20A4A000081A66E0FBA3E0FAA3E02417F9E43AFA7401120080E9B4052090081A66E0FBA38E
:20A4C000E0FAA3E02415F9E43AFAE412008124900819847480F001B0C890081A66E0FBA312
:20A4E000E0FAA3E02415F9E43AFA120080D3540F14700301AC2824FE603014700301B0396E
:20A5000024FE700301B03924FE700301B0392406600301B54490081979E0FBA3E0FAA3E0B1
:20A52000240DF9E43AFAE401AC3B900819847404F0120233C601B1DB90081A66E0FBA3E060
:20A54000FAA3E02415F9E43AFA120080D3540F6403600301B54490081A66A3E0FAA3E0246C
:20A5600016F9E43AFA74FF12008108600301B54490081A66A3E0FAA3E02417F9E43AFA7471
:20A5800001120080E96405600301B54412020B2B01A4B99008248FE0FBA3E0FAA3E0F99022
:20A5A000081A69E0FEA3E0FFE92FF9EA3EFAE41200812490081A667409F0A37419F0A37426
:20A5C0008FF09008248FE0FBA3E0FAA3E0F990081973EBF0A3EAF0A3E9F0240EF9E43AFAA2
:20A5E0009008197FEBF0A3EAF0A3E9F090081973E0FBA3E0FAA3E0240CF9E43AFA12008184
:20A60000AEFFAEF0BE0807BF06040201C40B90081973E0FBA3E0FAA3E0240CF9E43AFA1235
:20A620000081AE7004E5F06408600301AD989008197FE0FBA3E0FAA3E02402F9E43AFA1239
:20A640000081AEFFAEF090081A69EEF0A3EFF0D394DCEE9405400301AD989008197FE0FB55
:20A66000A3E0FAA3E0F9120080D3B44511E92406F9E43AFA120081AEE5F0543F600301AD94
:20A680009812023CB19008197FE0FBA3E0FAA3E02410F9E43AFA120083DDC31200836E6039
:20A6A000259008197FE0FBA3E0FAA3E02410F9E43AFA120083A574FFFBFAF9F8C31200833A
:20A6C0006E600301AD981201D3D6EFF47002EEF4600301AD989008197FE0FBA3E0FAA3E0BC
:20A6E000240CF9E43AFA120083A590081973E0FBA3E0FAA3E02406F9E43AFA1201BEE09064
:20A7000008197FE0FBA3E0FAA3E02409F9E43AFA120080D3B40149120080D3FF90081A66A1
:20A72000E0FBA3E0FAA3E02414F9E43AFAEF120081249008197FE0FBA3E0FAA3E0240CF91B
:20A74000E43AFA120083A590081A66E0FBA3E0FAA3E02404F9E43AFA120083C20202278178
:20A760009008197FE0FBA3E0FAA3E02409F9E43AFA120080D36411600301A8689008197F12
:20A78000A3E0FAA3E02414F9E43AFA9008197CEBF0A3EAF0A3E9F09008248FE0FBA3E0FACC
:20A7A000A3E0F9120223509008197FE0FBA3E0FAA3E02409F9E43AFA120080D3FF90081A37
:20A7C00066E0FBA3E0FAA3E02414F9E43AFAEF120081249008197CE0FBA3E0FAA3E024021B
:20A7E000F9E43AFA120081AEFF90081A66E0FBA3E0FAA3E0F9E5F08FF0120082289008195B
:20A800007CE0FBA3E0FAA3E0F9120081AEFF90081A66E0FBA3E0FAA3E02402F9E43AFAE599
:20A82000F08FF0120082289008197FE0FBA3E0FAA3E0240CF9E43AFA120083A590081A664F
:20A84000E0FBA3E0FAA3E02404F9E43AFA120083C290081A66E0FBA3E0FAA3E0F91200810E
:20A86000AEFFAEF002023AA69008197FE0FBA3E0FAA3E02409F9E43AFA120080D364066031
:20A880000301AD989008197FE0FBA3E0FAA3E02414F9E43AFA90081979EBF0A3EAF0A3E90D
:20A8A000F012023DAB90081979E0FBA3E0FAA3E02402F9E43AFA120081AE6F7003EE65F00A
:20A8C000600301AD9890082AEEE4F0A304F090082AEEE0FEA3E0FFC39405EE940040030182
:20A8E000A9AC7C007D2B12008138748F2FF974193EFA7B0990081A66EBF0A3EAF0A3E9F0B4
:20A900002415F9E43AFA120080D3700301A99990081979E0FBA3E0FAA3E02402F9E43AFA96
:20A92000120081AEFFAEF090081A66E0FBA3E0FAA3E0F9120081AE6F7003EE65F0705AE934
:20A940002402F9E43AFA120081AEFFAEF090081979E0FBA3E0FAA3E0F9120081AEB50739AE
:20A96000E5F0B5063490081A66E0FBA3E0FAA3E02404F9E43AFA120083A59008197FE0FBA2
:20A98000A3E0FAA3E0240CF9E43AFA120083DDC31200836E700301AD3E90082AEFE004F05A
:20A9A000700790082AEEE004F001A8CE90081979E0FBA3E0FAA3E0240DF9E43AFA1200804C
:20A9C000D36402600301AD9890082AEEE4F0A304F090082AEEE0FEA3E0FFC39405EE94008C
:20A9E000502D900819A475F02BEF1200843BEE75F02BA42583F583759308E0605E90082A83
:20AA0000EFE004F070CB90082AEEE004F080C290082AEEE4F0A304F090082AEEE0FEA3E046
:20AA2000FFC39405EE9400502F900819A475F02BEF1200843BEE75F02BA42583F5837593CB
:20AA400008E06407601590082AEFE004F070C990082AEEE004F080C001AD9890082AEEE0D6
:20AA6000FEA3E0FF7C007D2B12008138748F2FF974193EFA90081A667409F0A3EAF0A3E9E9
:20AA8000F09008197FE0FBA3E0FAA3E02409F9E43AFA120080D3FF90081A66E0FBA3E0FAA9
:20AAA000A3E02414F9E43AFAEF1200812490081A66E0FBA3E0FAA3E02416F9E43AFA740270
:20AAC0001200812490081A66E0FBA3E0FAA3E02417F9E43AFAE41200812490081979E0FBE0
:20AAE000A3E0FAA3E02402F9E43AFA120081AEFF90081A66E0FBA3E0FAA3E0F9E5F08FF09F
:20AB00001200822890081979E0FBA3E0FAA3E0F9120081AEFF90081A66E0FBA3E0FAA3E048
:20AB20002402F9E43AFAE5F08FF0120082289008197FE0FBA3E0FAA3E0240CF9E43AFA1270
:20AB40000083A590081A66E0FBA3E0FAA3E02404F9E43AFA120083C290081A66E0FBA3E0D4
:20AB6000FAA3E02415F9E43AFA7411120081249008198BE0FCA3E0FDA3E0FEA3E0FF90089F
:20AB80001A66E0FBA3E0FAA3E0240CF9E43AFA120083C2EF2401FFE43EFEE43DFDE43CFC55
:20ABA00090081A66E0FBA3E0FAA3E02410F9E43AFA120083C290081979E0FBA3E0FAA3E001
:20ABC0002404F9E43AFA120083A5EF2401FFE43EFEE43DFDE43CFC90081A66E0FBA3E0FA25
:20ABE000A3E02408F9E43AFA120083C290081A66E0FBA3E0FAA3E02422F9E43AFAC003C071
:20AC000002C00190081A66A3E0FAA3E02420F9E43AFA90082A60EBF0A3EAF0A3E9F0D0013D
:20AC2000D002D00312022C4890081979E0FBA3E0FAA3E0240DF9E43AFA74101200812490D5
:20AC4000081979E0FBA3E0FAA3E0240DF9E43AFA120080D344021200812490081979E0FBD6
:20AC6000A3E0FAA3E02414F9E43AFA90082AF0EBF0A3EAF0A3E9F074021200812490082A16
:20AC8000F0E0FBA3E0FAA3E02401F9E43AFA74041200812490082AF0E0FBA3E0FAA3E024D3
:20ACA00002F9E43AFA74051200812490082AF0E0FBA3E0FAA3E02403F9E43AFA747812008E
:20ACC000812490082AF0E0FBA3E0FAA3E02404F9E43AFA74011200812490082AF0E0FBA3AD
:20ACE000E0FAA3E02405F9E43AFA74011200812490082AF0E0FBA3E0FAA3E02406F9E43AC3
:20AD0000FA74041200812490082AF0E0FBA3E0FAA3E02407F9E43AFA74021200812490087C
:20AD20001A69E4F0A37430F090081979E0FBA3E0FAA3E0240CF9E43AFA747001B45FE490D3
:20AD4000081984F090081979E0FBA3E0FAA3E0240DF9E43AFA120080D330E22490081A6664
:20AD6000E0FBA3E0FAA3E02415F9E43AFAE412008124900819847420F0120233C601B32178
:20AD800090081979E0FBA3E0FAA3E0240DF9E43AFA120080D320E40301B32190081979E021
:20ADA000FBA3E0FAA3E0240CF9E43AFA120080D3C4540F75F004A4FFAEF090082AEEEEF093
:20ADC000A3EFF02414FFE43EFEC390081A6AE09FFF90081A69E09EFEF0A3EFF0D39400EEDF
:20ADE0009400403490081A66E0FBA3E0FAA3E02408F9E43AFA120083A590081979E0FBA339
:20AE0000E0FAA3E02404F9E43AFA120083DDC31200836E600301B42B90081A66E0FBA3E0AB
:20AE2000FAA3E02410F9E43AFA120083A590081979E0FBA3E0FAA3E02408F9E43AFA1200C2
:20AE400083DDC31200836E706690081A66E0FBA3E0FAA3E02410F9E43AFA120083A59008EC
:20AE60001A66A3E0FAA3E0240CF9E43AFA120083C290081A66E0FBA3E0FAA3E02415F9E4B1
:20AE80003AFA120080D3FF30E425900819847401F0EF54EF1200812490081A66E0FBA3E0E8
:20AEA000FAA3E02416F9E43AFA74021200812490081A66E0FBA3E0FAA3E02415F9E43AFA60
:20AEC000120080D3540F14B40800400301B4279000AEDE75F004A4C58325F0C58373020078
:20AEE000AEFE0200AF1A0200AF9D0200B23C0200B3240200B3F20200B42B0200B2219008CF
:20AF00001984E030E011740312008124900819847440F0120233C601B32190081984E03065
:20AF2000E07890081979E0FBA3E0FAA3E0240DF9E43AFA120080D36412705F90081A66E0D0
:20AF4000FBA3E0FAA3E02415F9E43AFA74031200812490081979E0FBA3E0FAA3E02404F958
:20AF6000E43AFA120083A590081A66E0FBA3E0FAA3E02408F9E43AFA120083C2120083A5BE
:20AF8000EF2401FFE43EFEE43DFDE43CFC120083C27442120233B901B0A901B32190081957
:20AFA00079E0FBA3E0FAA3E0240DF9E43AFA120080D320E00301B03C90081A6AE02401FF86
:20AFC00090081A69E03400FEE4FCFD90081A66E0FBA3E0FAA3E02408F9E43AFA120083C2E0
:20AFE0007410120233B990081A66E0FBA3E0FAA3E02410F9E43AFA120083A5EF2401FFE464
:20B000003EFEE43DFDE43CFC120083C290081A66E0FBA3E0FAA3E02415F9E43AFA74181288
:20B0200000812490081A66E0FBA3E0FAA3E02417F9E43AFAE41200812401B135D390081A25
:20B040006AE0940090081A69E09400404590081984E04402F090081A66E0FBA3E0FAA3E0C0
:20B060002408F9E43AFAC003C002C001120083DD90081A69E0FEA3E0FFE4FCFDEB2FFFEA80
:20B080003EFEED39FDEC38FCD001D002D003120083C290081984E05403700301B21E1202A0
:20B0A00033C6EF4E700301B42B90081984E0FF30E52C90081A66E0FBA3E0FAA3E02415F98D
:20B0C000E43AFAE41200812490081979E0FBA3E0FAA3E0240DF9E43AFA741401B43EEF30DC
:20B0E000E46990081A66E0FBA3E0FAA3E02410F9E43AFA120083A5EF2401FFE43EFEE43D3D
:20B10000FDE43CFC120083C290081A66E0FBA3E0FAA3E02415F9E43AFA74141200812490B3
:20B12000081A66E0FBA3E0FAA3E02417F9E43AFAE41200812490081979E0FBA3E0FAA3E0C0
:20B14000240DF9E43AFA741101B43ED390081A6AE0940090081A69E09400407790081A6674
:20B16000E0FBA3E0FAA3E02415F9E43AFA120080D320E45F120080D34410120081249008DA
:20B180001A66E0FBA3E0FAA3E02417F9E43AFAE41200812490081A66E0FBA3E0FAA3E02456
:20B1A00010F9E43AFAC003C002C001120083DD90081A69E0FEA3E0FFE4FCFDEB2FFFEA3E1D
:20B1C000FEED39FDEC38FCD001D002D003120083C28008E490081A69F0A3F0D390081A6A68
:20B1E000E0940090081A69E09400500890081984E030E12A90081A6AE02428F090081A6951
:20B20000E03400F090081979E0FBA3E0FAA3E0240DF9E43AFA74181200812401B44C01B3EB
:20B220002190081984E020E00301B42790081A66E0FBA3E0FAA3E0241501B41ED390081A75
:20B240006AE0940090081A69E09400403D90081A66E0FBA3E0FAA3E02408F9E43AFAC00311
:20B26000C002C001120083DD90081A69E0FEA3E0FFE4FCFDEB2FFFEA3EFEED39FDEC38FCFF
:20B28000D001D002D003120083C290081979E0FBA3E0FAA3E0240DF9E43AFA120080D33005
:20B2A000E04990081984E090081A6630E027E0FBA3E0FAA3E02415F9E43AFA7407120081CE
:20B2C0002490081A66E0FBA3E0FAA3E02416F9E43AFAE4800FE0FBA3E0FAA3E02415F9E4A8
:20B2E0003AFA74161200812401B3B790081984E030E01A90081A66E0FBA3E0FAA3E0241503
:20B30000F9E43AFA74051200812401B427D390081A6AE0940090081A69E09400400301B426
:20B320002B01B427D390081A6AE0940090081A69E09400403D90081A66E0FBA3E0FAA3E0A4
:20B340002408F9E43AFAC003C002C001120083DD90081A69E0FEA3E0FFE4FCFDEB2FFFEA9D
:20B360003EFEED39FDEC38FCD001D002D003120083C290081979E0FBA3E0FAA3E0240DF952
:20B38000E43AFA120080D330E05590081A66E0FBA3E0FAA3E02415F9E43AFA740712008180
:20B3A0002490081A66E0FBA3E0FAA3E02416F9E43AFAE41200812490081A66E0FBA3E0FA20
:20B3C000A3E02408F9E43AFA120083A5EF2401FFE43EFEE43DFDE43CFC120083C2804CD310
:20B3E00090081A6AE0940090081A69E09400503B803590081984E030E02D90081A66E0FBA9
:20B40000A3E0FAA3E02415F9E43AFA74071200812490081A66E0FBA3E0FAA3E02416F9E4A6
:20B420003AFAE4120081240200802390081979E0FBA3E0FAA3E0240DF9E43AFA74101200BB
:20B44000812490081A69E4F0A37428F090081979E0FBA3E0FAA3E0240CF9E43AFA7450120D
:20B4600000812490081A66E0FBA3E0FAA3E02408F9E43AFA120083A590081979E0FBA3E035
:20B48000FAA3E02408F9E43AFA120083C290081A66E0FBA3E0FAA3E0240CF9E43AFA120055
:20B4A00083A590081979E0FBA3E0FAA3E02404F9E43AFA120083C290081A66E0FBA3E0FA5F
:20B4C000A3E0F9120081AEFF90081979E0FBA3E0FAA3E0F9E5F08FF01200822890081A668A
:20B4E000E0FBA3E0FAA3E02402F9E43AFA120081AEFF90081979E0FBA3E0FAA3E02402F9D6
:20B50000E43AFAE5F08FF01200822890081979E0FBA3E0FAA3E0240EF9E43AFA740575F0DD
:20B5200078120082287F027E001201272590081A66E0FBA3E0FAA3E02416F9E43AFA7402C5
:20B54000120081242290081979E0FBA3E0FAA3E02414F9E43AFA90081976EBF0A3EAF0A3A2
:20B56000E9F090081A66E0FBA3E0FAA3E02424F9E43AFA9008066EEBF0A3EAF0A3E9F09036
:20B58000081A66A3E0FAA3E02423F9E43AFA90080403EBF0A3EAF0A3E9F090081A66A3E0BD
:20B5A000FAA3E02418F9E43AFA90080660EBF0A3EAF0A3E9F090081A66A3E0FAA3E0241A99
:20B5C000F9E43AFA90080400EBF0A3EAF0A3E9F090081A66A3E0FAA3E0241CF9E43AFA90F1
:20B5E00008066BEBF0A3EAF0A3E9F090081A66A3E0FAA3E0241EF9E43AFA90080663EBF0B7
:20B60000A3EAF0A3E9F090081984E0FD30E6549008066EE0FBA3E0FAA3E0F9E4120081243A
:20B620009008066EE0FBA3E0FAA3E02402F9E43AFAE4F5F01200822890080660E0FBA3E00B
:20B64000FAA3E0F9E475F001120082289008066BE0FBA3E0FAA3E0F9E475F001120082288B
:20B6600001C3B5ED30E70301C3B590081984E020E10301C1C49008066EE0FBA3E0FAA3E04B
:20B68000F9120080D3600301C1C4900829F17481F0A3749EF0A37445F0A3E4F0A37404F059
:20B6A00090081976E0FBA3E0FAA3E0F9120221CFEF600301B73D900823AFF090081976E0E3
:20B6C000FBA3E0FAA3E02405F9E43AFA900823AFE0FF7C0029F9EC3AFAA3EBF0A3EAF0A390
:20B6E000E9F0120080D3FE64206004EEB43F1174B32FF582E43423F583759308E4F0801937
:20B70000900823AFE0FF04F074B32FF582E43423F583759308EEF080A27B097A2379B312FD
:20B7200000A3BEEF4E600301B7FF78B37C237D097B817A9E794A1200869301B7FF90082888
:20B74000327481F0A3749EF0A37454F090081976E0FBA3E0FAA3E0F9120207F5900823B05C
:20B76000EBF0A3EAF0A3E9F0900823B0E0FBA3E0FAA3E04A4B703F90080666E064037003AD
:20B7800001BB7190081A69E0FEA3E0FF7D0090081976E0FBA3E0FAA3E0F912008851E4902A
:20B7A000081A69F0A3F090081976E0FBA3E0FAA3E0F9020148249008264B7481F0A3749E6E
:20B7C000F0A37454F0A37481F0A3749EF0A3745EF0A37409F0A37423F0A374B3F0900823DD
:20B7E000B0E0FBA3E0FAA3E0F91201E0B49008066EE0FBA3E0FAA3E0F97401120081249082
:20B800000829F17481F0A3749EF0A37460F0A3E4F0A3740AF07B097A2379B3120221CFEF4D
:20B82000704990081A66E0FBA3E0FAA3E02404F9E43AFA120083A590080667E0F8A3E0F990
:20B84000A3E0FAA3E0FBC31200836E700301B8E1E4FFFEFDFC90080667E0F8A3A3A3E0C3D7
:20B860001200836E600301B9D88076900829F17481F0A3749EF0A3746BF0A3E4F0A3740A94
:20B88000F07B097A2379B3120221CFEF701078B37C237D097B817A9E7976120086939008E2
:20B8A00029F17481F0A3749EF0A37483F0A3E4F0A37404F07B097A2379B3120221CFEF7028
:20B8C0000301B997900829977409F0A37423F0A374AAF07B097A2379B312020484EF4E70DE
:20B8E0002078B37C237D097B817A9E798812008693900806667401F0E4FFFEFDFCA301BBF6
:20B900001F9008066EE0FBA3E0FAA3E0F9740212008124900823AAE0FBA3E0FAA3E0F9C002
:20B9200003C002C0019008066EE0FBA3E0FAA3E02404F9E43AFA12008464900823ADE0FE21
:20B94000A3E0FF9008066EE0FBA3E0FAA3E02402F9E43AFAEE8FF01200822812023CA1C06D
:20B9600004C005C006C00712023DE7E4FCFD7B587A02F9F812008244D003D002D001D000FE
:20B98000EB2FFFEA3EFEE93DFDE83CFC900804061200842F01C2E890081A66E0FBA3E0FAA3
:20B9A000A3E02404F9E43AFA120083A590080667E0F8A3E0F9A3E0FAA3E0FBC31200836E77
:20B9C000603EE4FFFEFDFC90080667E0F8A3A3A3E0C31200836E60289008296A7481F0A348
:20B9E000749EF0A37498F0A37481F0A3749EF0A37488F07B817A9E79921202157801C3B5B1
:20BA00009008066EE0FBA3E0FAA3E0F9120080D36401600301BB26900829F17481F0A37489
:20BA20009EF0A374B0F0A3E4F0A3740AF07B097A2379B3120221CFEF600301BB2690081903
:20BA400076E0FBA3E0FAA3E0F912021917EF4E707512023CE1E4FBFAF9F8C31200836E6015
:20BA60003D12023CF1EF5402FFE4FEFDFC7B02FAF9F8C31200836E702590081A66E0FBA3D0
:20BA8000E0FAA3E02404F9E43AFA120083A590082AB31200842F7FEA7E0312020CA7900853
:20BAA000296A7481F0A3749EF0A374BBF0A37481F0A3749EF0A37488F07B817A9E799212BA
:20BAC00002157801C3B590081A66E0FBA3E0FAA3E02404F9E43AFA120083A59008066712E1
:20BAE00000842F900806667402F012023CA1C004C005C006C00712023DE7E4FCFD7B587AC0
:20BB000002F9F812008244D003D002D001D000EB2FFFEA3EFEE93DFDE83CFC9008040612DE
:20BB200000842F01C025900829F17481F0A3749EF0A37488F0A3E4F0A37409F07B097A23F9
:20BB400079B3120221CFEF70099008066604F001C02590080666E0B4010F78B37C237D0977
:20BB60007B817A9E798801BFEA90080666E0B403399008296A7481F0A3749EF0A374CAF0AC
:20BB8000A37481F0A3749EF0A37488F07B817A9E799212021578900806667401F0E4FFFEDF
:20BBA000FDFCA31200842F01C3B59008066EE0FBA3E0FAA3E0F9120080D36401600301C0DD
:20BBC00025900829F17481F0A3749EF0A374D8F0A3E4F0A37408F07B097A2379B31202211D
:20BBE000CFEF701A90081976E0FBA3E0FAA3E0F912019497EF4E600301C02501BFDA90080C
:20BC000029F17481F0A3749EF0A374E1F0A3E4F0A37407F07B097A2379B3120221CFEF7063
:20BC20001390081976E0FBA3E0FAA3E0F91202302301C025900829F17481F0A3749EF0A3CA
:20BC400074E9F0A3E4F0A3740AF07B097A2379B3120221CFEF701390081976E0FBA3E0FACD
:20BC6000A3E0F91201EF0401C025900829F17481F0A3749EF0A374F4F0A3E4F0A37407F0A0
:20BC80007B097A2379B3120221CFEF701390081976E0FBA3E0FAA3E0F91201FB0F01C025E3
:20BCA000900829F17481F0A3749EF0A374FCF0A3E4F0A37409F07B097A2379B3120221CF6D
:20BCC000EF701390081976E0FBA3E0FAA3E0F91201F15E01C025900829F17481F0A3749F62
:20BCE000F0A37406F0A3E4F0A3740BF07B097A2379B3120221CFEF702690081976E0FBA343
:20BD0000E0FAA3E0F91201C09FEF4E700301BFDA78B37C237D097B817A9F791201BFEA90E7
:20BD20000829F17481F0A3749FF0A37412F0A3E4F0A37408F07B097A2379B3120221CFEF77
:20BD4000701A90081976E0FBA3E0FAA3E0F912016D79EF4E600301C02501BFDA900829F193
:20BD60007481F0A3749FF0A3741BF0A3E4F0A37409F07B097A2379B3120221CFEF701A9035
:20BD8000081976E0FBA3E0FAA3E0F91201D98FEF4E600301C02501BFDA900829F17481F006
:20BDA000A3749FF0A37425F0A3E4F0A3740AF07B097A2379B3120221CFEF701A9008197638
:20BDC000E0FBA3E0FAA3E0F91201CF57EF4E600301C02501BFDA900829F17481F0A3749FE9
:20BDE000F0A37430F0A3E4F0A37407F07B097A2379B3120221CFEF701A90081976E0FBA328
:20BE0000E0FAA3E0F912011271EF4E600301C02501BFDA900829F17481F0A3749FF0A374C2
:20BE200038F0A3E4F0A37408F07B097A2379B3120221CFEF701A90081976E0FBA3E0FAA368
:20BE4000E0F91201A975EF4E600301C02501BFDA900829F17481F0A3749FF0A37441F0A390
:20BE6000E4F0A37408F07B097A2379B3120221CFEF701A90081976E0FBA3E0FAA3E0F91208
:20BE8000014FA4EF4E600301C02501BFDA900829F17481F0A3749FF0A3744AF0A3E4F0A3E6
:20BEA000740CF07B097A2379B3120221CFEF702690081976E0FBA3E0FAA3E0F91201EDCC75
:20BEC000EF4E700301BFDA78B37C237D097B817A9F791201BFEA900829F17481F0A3749F31
:20BEE000F0A37457F0A3E4F0A37408F07B097A2379B3120221CFEF701A90081976E0FBA3FF
:20BF0000E0FAA3E0F912017C5BEF4E600301C02501BFDA900829F17481F0A3749FF0A3746D
:20BF200060F0A3E4F0A3740AF07B097A2379B3120221CFEF702690081976E0FBA3E0FAA331
:20BF4000E0F912017690EF4E700301BFDA78B37C237D097B817A9F796B01BFEA900829F100
:20BF60007481F0A3749FF0A37473F0A3E4F0A3740AF07B097A2379B3120221CFEF702490D0
:20BF8000081976E0FBA3E0FAA3E0F912016412EF4E7002804578B37C237D097B817A9F795B
:20BFA0006B8047900829F17481F0A3749FF0A3747EF0A3E4F0A3740AF07B097A2379B312A6
:20BFC0000221CFEF702A90081976E0FBA3E0FAA3E0F91201BD16EF4E7004FE7F012278B389
:20BFE0007C237D097B817A9F796B120086938035900829F17481F0A3749FF0A37489F0A3D3
:20C00000E4F0A37409F07B097A2379B3120221CFEF701290082473F0A304F090081984741B
:20C0200010F001C3B5E4900823AFF0900829F17481F0A3749FF0A37493F0A3E4F0A3740BD9
:20C04000F07B097A2379B3120221CFEF7014120222D278B37C237D097B817A9F799F120095
:20C060008693900829F17481F0A3749FF0A374ABF0A3E4F0A3740BF07B097A2379B31202CE
:20C0800021CFEF701A90082B4EF0A304F078B37C237D097B817A9F79B7120086938008E473
:20C0A00090082B4EF0A3F0E490082BB0F0A3F0900829F17481F0A3749FF0A37460F0A3E4E7
:20C0C000F0A3740AF07B097A2379B3120221CFEF7045900823017481F0A3749FF0A374C349
:20C0E000F0A37409F0A3742BF0A374B0F07B097A2379B31200997178B37C237D097B817A28
:20C100009F796B1200869390082BB1E024FFF090082BB0E034FFF0900823AFE0FD75F017D1
:20C12000A4240AF582E5F03404F583759308E0FBA3E0FAA3E04A4B700A900819847410F08E
:20C1400001C3B5ED75F017A4240DF9740435F0FA7B091200A3BE900829F4EEF0A3EFF090FC
:20C160000823AFE075F017A4240DF9740435F0FA900829F17409F0A3EAF0A3E9F07B097A0E
:20C180002379B3120221CFEF70309008066EE0FBA3E0FAA3E0F9740312008124900823AF45
:20C1A000E0FF9008066EE0FBA3E0FAA3E02401F9E43AFAEF12008124800A900823AFE00405
:20C1C000F001C1179008066EE0FBA3E0FAA3E0F9120080D36403600301C2E890081A69F0D1
:20C1E000A3F090081984E0B4043C90080400E0FBA3E0FAA3E0F9120081AEFF90080660E015
:20C20000FBA3E0FAA3E0F9E5F08FF01200822890080663E0FBA3E0FAA3E0F9120081AEFF05
:20C220009008066B803A90080660E0FBA3E0FAA3E0F9120081AEFF90080400E0FBA3E0FA35
:20C24000A3E0F9E5F08FF0120082289008066BE0FBA3E0FAA3E0F9120081AEFF9008066334
:20C26000E0FBA3E0FAA3E0F9E5F08FF0120082289008066EE0FBA3E0FAA3E02401F9E43AB7
:20C28000FA120080D375F017A4240AF582E5F03404F583759308E0FBA3E0FAA3E0F91200FF
:20C2A000850FEF6007900819847410F012023CA1C004C005C006C00712023DE7E4FCFD7B54
:20C2C000587A02F9F812008244D003D002D001D000EB2FFFEA3EFEE93DFDE83CFC9008045D
:20C2E000061200842F01C3B590081984E030E07A9008066EE0FBA3E0FAA3E02402F9E43A37
:20C30000FA120081AEC39478E5F09405402A74FA75F088120081FC9008066EE0FBA3E0FAED
:20C32000A3E02404F9E43AFA09E970010A740575F078120081FC80329008066EE0FBA3E0D3
:20C34000FAA3E02402F9E43AFAE4F5F0120082289008066EE0FBA3E0FAA3E0F9120080D35F
:20C36000B40207900819847410F09008066EE0FBA3E0FAA3E02402F9E43AFA120081AEFFF9
:20C38000AEF0D39478EE940590081A6940097405F0A37478F08005EEF0A3EFF09008066E5C
:20C3A000E0FBA3E0FAA3E02404F9E43AFA12008447120239107E007F012290080660E0FB36
:20C3C000A3E0FAA3E0F9E475F001120081D2AFF0FE600301D188EF24FE700301C4C11470CD
:20C3E0000301C83A14700301CB1D14700301CE8B2404600301D188900828327483F0A37411
:20C4000093F0A374A3F090081976E0FBA3E0FAA3E0F9120207F590081BBDEBF0A3EAF0A379
:20C42000E9F090081BBDE0FBA3E0FAA3E04A4B70037F0122900823017483F0A37493F0A34E
:20C4400074ABF0A37409F0A3741BF0A374C0F090081BBDE0FBA3E0FAA3E0F91200997190E4
:20C460000823FF7483F0A37493F0A374B5F090081BC0E0FEA3E0FF90082402EEF0A3EFF064
:20C480002401FFE43EA3F0A3EFF090081976E0FBA3E0FAA3E0F91200959290081A69EEF014
:20C4A000A3EFF090081BC0E0F9A3E0FF9008066BE0FBA3E0FAA3E0C98FF01200822801D172
:20C4C0008B9008066BE0FBA3E0FAA3E0F9120081AEFF12023BF4EF64044E701B9008066B38
:20C4E000E0FBA3E0FAA3E0F9120081AEFF120236D9EF4E700280349008066BE0FBA3E0FA41
:20C50000A3E0F9120081AEFF12023BF4EF64054E702A9008066BE0FBA3E0FAA3E0F91200ED
:20C5200081AEFF120236D9EF4E7011FE7F9CFD7B097A1B79211200885101C5D47E007F9C05
:20C540007D007B097A1B7921120088519008066BE0FBA3E0FAA3E0F9120081AEFF7B097AA5
:20C560001B792190082ACA7401F012023D5F9008066BE0FBA3E0FAA3E0F9120081AEFF7BCD
:20C58000097A1B792190082ACA7403F012023D5F9008066BE0FBA3E0FAA3E0F9120081AEA2
:20C5A000FF7B097A1B792190082ACA7405F012023D5F9008066BE0FBA3E0FAA3E0F9120035
:20C5C00081AEFF7B097A1B792190082ACA7406F012023D5F900823FF7481F0A37490F0A3FB
:20C5E0007406F0A37483F0A37495F0A3741EF090081B99E0FCA3E0FDA3E0FEA3E0FF900843
:20C6000024051200842F90081976E0FBA3E0FAA3E0F91200959290081A69EEF0A3EFF090ED
:20C62000081976E0FBA3E0FAA3E0F990081A69E0FEA3E0FFE92FF9EA3EFAC003900823FF64
:20C640007483F0A37495F0A37421F090081B3DE0FCA3E0FDA3E0FEA3E0FF90082402120010
:20C66000842F90081BA9E0FCA3E0FDA3E0FEA3E0FF900824061200842FD003120095929029
:20C68000081A6AE02FF090081A69E03EF090081BC0E4F0A304F090081BC0E0FEA3E0FFD362
:20C6A0009403EE64809480400301D18BEE600301C783EF24FE604514607D2402600301C7C9
:20C6C0008390081BC27483F0A37495F0A3748CF090081B45E0FCA3E0FDA3E0FEA3E0FF9065
:20C6E000081BC81200842F90081BC57483F0A37495F0A3749AF090081B79807490081BC259
:20C700007483F0A37495F0A374A6F090081B41E0FCA3E0FDA3E0FEA3E0FF90081BC8120009
:20C72000842F90081BC57483F0A37495F0A374B4F090081B7D803990081BC27483F0A37434
:20C7400095F0A374C7F090081B49E0FCA3E0FDA3E0FEA3E0FF90081BC81200842F90081B38
:20C76000C57483F0A37495F0A374DCF090081B81E0FCA3E0FDA3E0FEA3E0FF90081BCC126A
:20C7800000842F90081976E0FBA3E0FAA3E0F990081A69E0FEA3E0FFE92FF9EA3EFAC0037A
:20C7A000C002C001900823FF7481F0A37490F0A37443F090081BC2E0F9A3E0FAA3E0900890
:20C7C0002402C9F0A3EAF0A3E9F090081BC8E0FCA3E0FDA3E0FEA3E0FF9008240512008450
:20C7E0002F90081BC5E0F9A3E0FAA3E090082409C9F0A3EAF0A3E9F090081BCCE0FCA3E064
:20C80000FDA3E0FEA3E0FF9008240C1200842FD001D002D0031200959290081A6AE02FF0C1
:20C8200090081A69E03EF090081BC1E004F0700790081BC0E004F001C6969008066BE0FB88
:20C84000A3E0FAA3E0F9120081AEFF12023BF4EF64044E701B9008066BE0FBA3E0FAA3E048
:20C86000F9120081AEFF120236D9EF4E700280349008066BE0FBA3E0FAA3E0F9120081AEDB
:20C88000FF12023BF4EF64054E70299008066BE0FBA3E0FAA3E0F9120081AEFF120236D9D7
:20C8A000EF4E7010FE7F9CFD7B097A1B79211200885180547E007F9C7D007B097A1B79216A
:20C8C000120088519008066BE0FBA3E0FAA3E0F9120081AEFF7B097A1B792190082ACA749D
:20C8E00003F012023D5F9008066BE0FBA3E0FAA3E0F9120081AEFF7B097A1B792190082A03
:20C90000CA7406F012023D5F90081BC0E4F0A304F090081BC0E0FEA3E0FFD39404EE648045
:20C920009480400301D18BEE600301CA66EF24FE604E14700301C9BB14700301CA0124037C
:20C94000600301CA6690081BC27483F0A37495F0A374F0F090081BADE0FCA3E0FDA3E0FE17
:20C96000A3E0FF90081BC81200842F90081BC57483F0A37496F0A37400F090081B858074C6
:20C9800090081BC27483F0A37496F0A37414F090081BB1E0FCA3E0FDA3E0FEA3E0FF900828
:20C9A0001BC81200842F90081BC57483F0A37496F0A37428F090081B89803990081BC274C6
:20C9C00083F0A37496F0A3743DF090081BB5E0FCA3E0FDA3E0FEA3E0FF90081BC81200842B
:20C9E0002F90081BC57483F0A37496F0A37450F090081B8DE0FCA3E0FDA3E0FEA3E0FF8096
:20CA00005D90081BC27483F0A37496F0A37466F090081BB9E0FCA3E0FDA3E0FEA3E0FF90F8
:20CA2000081BC81200842F90081BC57483F0A37496F0A37474F090081B95E0FCA3E0FDA388
:20CA4000E0FEA3E0FF90081B91E0F8A3E0F9A3E0FAA3E02FFFEA3EFEE93DFDE83CFC9008AF
:20CA60001BCC1200842F90081976E0FBA3E0FAA3E0F990081A69E0FEA3E0FFE92FF9EA3E5B
:20CA8000FAC003C002C001900823FF7481F0A37490F0A37443F090081BC2E0F9A3E0FAA368
:20CAA000E090082402C9F0A3EAF0A3E9F090081BC8E0FCA3E0FDA3E0FEA3E0FF900824058B
:20CAC0001200842F90081BC5E0F9A3E0FAA3E090082409C9F0A3EAF0A3E9F090081BCCE06A
:20CAE000FCA3E0FDA3E0FEA3E0FF9008240C1200842FD001D002D0031200959290081A6A5F
:20CB0000E02FF090081A69E03EF090081BC1E004F0700790081BC0E004F001C9119008066E
:20CB20006BE0FBA3E0FAA3E0F9120081AEFF12023BF4EF64044E701B9008066BE0FBA3E09C
:20CB4000FAA3E0F9120081AEFF120236D9EF4E700280349008066BE0FBA3E0FAA3E0F912AA
:20CB60000081AEFF12023BF4EF64054E70299008066BE0FBA3E0FAA3E0F9120081AEFF12D6
:20CB80000236D9EF4E7010FE7F9CFD7B097A1B79211200885180757E007F9C7D007B097A0A
:20CBA0001B7921120088519008066BE0FBA3E0FAA3E0F9120081AEFF7B097A1B7921E49091
:20CBC000082ACAF012023D5F9008066BE0FBA3E0FAA3E0F9120081AEFF7B097A1B79219059
:20CBE000082ACA7402F012023D5F9008066BE0FBA3E0FAA3E0F9120081AEFF7B097A1B7974
:20CC00002190082ACA7405F012023D5F900823FF7481F0A37490F0A37406F0A37483F0A3DE
:20CC20007496F0A37489F090081BA1E0FCA3E0FDA3E0FEA3E0FF900824051200842F900899
:20CC40001976E0FBA3E0FAA3E0F91200959290081A69EEF0A3EFF090081BC0E4F0A304F0DF
:20CC600090081BC0E0FEA3E0FFD39405EE64809480400301D18BEE600301CDD4EF24FE608B
:20CC80005514700301CD1214700301CD4D14700301CD882404600301CDD490081BC27483C0
:20CCA000F0A37496F0A3748CF090081B21E0FCA3E0FDA3E0FEA3E0FF90081BC81200842FE1
:20CCC00090081BC57483F0A37496F0A37498F090081B7101CDC190081BC27483F0A37495FE
:20CCE000F0A3748CF090081B29E0FCA3E0FDA3E0FEA3E0FF90081BC81200842F90081BC5BE
:20CD00007483F0A37496F0A374A8F090081B7501CDC190081BC27483F0A37495F0A374A674
:20CD2000F090081B25E0FCA3E0FDA3E0FEA3E0FF90081BC81200842F90081BC57483F0A38A
:20CD40007495F0A3749AF090081B4D807490081BC27483F0A37495F0A374C7F090081B2D9F
:20CD6000E0FCA3E0FDA3E0FEA3E0FF90081BC81200842F90081BC57483F0A37495F0A37402
:20CD8000B4F090081B51803990081BC27483F0A37496F0A374B7F090081B69E0FCA3E0FD03
:20CDA000A3E0FEA3E0FF90081BC81200842F90081BC57483F0A37495F0A374DCF090081B9F
:20CDC00055E0FCA3E0FDA3E0FEA3E0FF90081BCC1200842F90081976E0FBA3E0FAA3E0F960
:20CDE00090081A69E0FEA3E0FFE92FF9EA3EFAC003C002C001900823FF7481F0A37490F009
:20CE0000A37443F090081BC2E0F9A3E0FAA3E090082402C9F0A3EAF0A3E9F090081BC8E0AF
:20CE2000FCA3E0FDA3E0FEA3E0FF900824051200842F90081BC5E0F9A3E0FAA3E0900824E0
:20CE400009C9F0A3EAF0A3E9F090081BCCE0FCA3E0FDA3E0FEA3E0FF9008240C1200842FAC
:20CE6000D001D002D0031200959290081A6AE02FF090081A69E03EF090081BC1E004F07007
:20CE80000790081BC0E004F001CC609008066BE0FBA3E0FAA3E0F9120081AEFF12023BF4B7
:20CEA000EF64044E701B9008066BE0FBA3E0FAA3E0F9120081AEFF120236D9EF4E700280D3
:20CEC000349008066BE0FBA3E0FAA3E0F9120081AEFF12023BF4EF64054E70299008066B76
:20CEE000E0FBA3E0FAA3E0F9120081AEFF120236D9EF4E7010FE7F9CFD7B097A1B79211263
:20CF000000885180537E007F9C7D007B097A1B7921120088519008066BE0FBA3E0FAA3E0CD
:20CF2000F9120081AEFF7B097A1B7921E490082ACAF012023D5F9008066BE0FBA3E0FAA3F1
:20CF4000E0F9120081AEFF7B097A1B792190082ACA7402F012023D5F90081BC0E4F0A30475
:20CF6000F090081BC0E0FEA3E0FFD39404EE64809480400301D14AEE600301D093EF24FE78
:20CF8000604F14700301D00C14700301D0472403600301D09390081BC27483F0A37496F0F8
:20CFA000A374C5F090081B6DE0FCA3E0FDA3E0FEA3E0FF90081BC81200842F90081BC574FA
:20CFC00083F0A37496F0A37400F090081B5901D08090081BC27483F0A37496F0A374D2F00B
:20CFE00090081B31E0FCA3E0FDA3E0FEA3E0FF90081BC81200842F90081BC57483F0A37438
:20D0000096F0A37428F090081B5D807490081BC27483F0A37496F0A374DCF090081B35E0B3
:20D02000FCA3E0FDA3E0FEA3E0FF90081BC81200842F90081BC57483F0A37496F0A37450CE
:20D04000F090081B61803990081BC27483F0A37496F0A374ECF090081B39E0FCA3E0FDA33C
:20D06000E0FEA3E0FF90081BC81200842F90081BC57483F0A37496F0A374F9F090081B65FC
:20D08000E0FCA3E0FDA3E0FEA3E0FF90081BCC1200842F90081976E0FBA3E0FAA3E0F99062
:20D0A000081A69E0FEA3E0FFE92FF9EA3EFAC003C002C001900823FF7481F0A37490F0A333
:20D0C0007443F090081BC2E0F9A3E0FAA3E090082402C9F0A3EAF0A3E9F090081BC8E0FC94
:20D0E000A3E0FDA3E0FEA3E0FF900824051200842F90081BC5E0F9A3E0FAA3E09008240911
:20D10000C9F0A3EAF0A3E9F090081BCCE0FCA3E0FDA3E0FEA3E0FF9008240C1200842FD022
:20D1200001D002D0031200959290081A6AE02FF090081A69E03EF090081BC1E004F070070D
:20D1400090081BC0E004F001CF6190081976E0FBA3E0FAA3E0F990081A69E0FEA3E0FFE9F8
:20D160002FF9EA3EFA900823FF7483F0A37497F0A3740EF01200959290081A6AE02FF0902D
:20D18000081A69E03EF080037F01227F002290080660E0FBA3E0FAA3E0F9120081AEFFAE70
:20D1A000F0E5F0600301DC06EF120084B8D1E101D60502D66C03D68D07D6F808D70509D756
:20D1C000090DD7590ED9030FDAD710DAD712DB4313DB5016DBA817DBB518DBB51A0000DC52
:20D1E00006900823FF7483F0A37480F0A37434F090081976E0FBA3E0FAA3E0F91200959292
:20D2000090081A69EEF0A3EFF0E490081E9DF0A3F090081E9DE475F00112008182AFF0FE8A
:20D22000600301D4E1EF14B40D00400301D4E19000D23E75F004A4C58325F0C58373020051
:20D24000D2720200D2900200D2AE0200D2E10200D2F10200D3060200D31B0200D330020058
:20D26000D34E0200D3E40200D3FF0200D41F0200D44C90081EA77483F0A37481F0A3746E98
:20D28000F078AA7C1E7D097B837A81797B01D41890081EA77483F0A37481F0A374CCF0786B
:20D2A000AA7C1E7D097B837A8179DD01D41890081EA77483F0A37481F0A374EAF0900823F0
:20D2C000FF7483F0A37481F0A374FBF0A3E4F0A37402F0A3E4F0A304F0A3E4F0A30401D55C
:20D2E0007290081E9EE004F0700790081E9DE004F090081EA77483F0A37482F0A37408F01A
:20D3000012023CB1803D90081EA77483F0A37482F0A37413F012023CC1802890081EA774DE
:20D3200083F0A37482F0A3741FF012023CD1801390081EA77483F0A37482F0A3742FF01202
:20D34000023CE190081EFA1200842F01D4F490081EA77483F0A37482F0A37437F07B097A67
:20D360001E79AA12023847900823FF7483F0A37482F0A37443F090081EAAE0FF3395E090EE
:20D38000082402E4F0A3EFF090081EABE0FF3395E090082404E4F0A3EFF090081EACE0FFCA
:20D3A0003395E090082406E4F0A3EFF090081EADE0FF3395E090082408E4F0A3EFF0900811
:20D3C0001EAEE0FF3395E09008240AE4F0A3EFF090081EAFE0FF3395E09008240CE4F0A3B3
:20D3E000EF01D57290081EA77483F0A37482F0A37461F012023E7378AA7C1E7D0980199091
:20D40000081EA77483F0A37482F0A3746DF012023E7A78AA7C1E7D091200869301D57D903F
:20D42000081EA77483F0A37482F0A3747BF012023DE790082402EEF0A3EFF0900823FF74A9
:20D4400083F0A37482F0A3749301D57290081EA77483F0A37482F0A37496F0900827F6744B
:20D4600009F0A3741FF0A37400F0A37409F0A3741FF0A37402F0A37409F0A3741FF0A374FA
:20D4800004F07B097A1E79FE12022B8B900823FF7483F0A37482F0A374A4F090081EFEE0D2
:20D4A000FFA3E090082402CFF0A3EFF090081F00E0FFA3E090082404CFF0A3EFF090081F1A
:20D4C00002E0FFA3E090082406CFF0A3EFF090081F04E0FFA3E090082408CFF0A3EF01D5DD
:20D4E0007290080660E0FBA3E0FAA3E0F9E475F00201D794900823FF7483F0A37482F0A364
:20D5000074C8F090081EFAE0FCA3E0FDA3E0FEA3E0FF78181200837FE490082402F0A3EF08
:20D52000F090081EFAE0FCA3E0FDA3E0FEA3E0FF78101200837FE490082404F0A3EFF090AA
:20D54000081EFAE0FCA3E0FDA3E0FEA3E0FF78081200837FE490082406F0A3EFF090081EEA
:20D56000FAE0FCA3E0FDA3A3E0FEE490082408F0A3CEF07B097A1E79AA120095927B097AC2
:20D580001E79AA1200A3BEEF4E701078AA7C1E7D097B837A8279D41200869390081976E05F
:20D5A000FBA3E0FAA3E0F990081A69E0FEA3E0FFE92FF9EA3EFAC002C001900823FF748395
:20D5C000F0A37482F0A374DBF090081EA7E0F9A3E0FAA3E090082402C9F0A3EAF0A3E9F04A
:20D5E000A37409F0A3741EF0A374AAF0D001D0021200959290081A6AE02FF090081A69E053
:20D600003EF001D21190081976E0FBA3E0FAA3E0F990081A69E0FEA3E0FFE92FF9EA3EFA4F
:20D62000900823FF7483F0A37482F0A374F5F01200959290081A6AE02FF090081A69E03E37
:20D64000F01201E36890080660E0FBA3E0FAA3E0F9E475F003120082289008066BE0FBA31B
:20D66000E0FAA3E0F9E475F00101D794E4FFFE1201226AEF4E7002FF2290080660E0FBA3D2
:20D68000E0FAA3E0F9E475F0071200822812023DF0EF4E607090081976E0FBA3E0FAA3E0D8
:20D6A000F990081A69E0FEA3E0FFE92FF9EA3EFA900823FF7483F0A37483F0A3741CF01263
:20D6C00000959290081A6AE02FF090081A69E03EF090080660E0FBA3E0FAA3E0F9E475F0C4
:20D6E00008120082289008066BE0FBA3E0FAA3E0F9E4F5F012008228E4FFFE120173A0EF0E
:20D700004E7002FF2212023DF0900823FF7483F0A37483F0A37451F090081976E0FBA3E0DF
:20D72000FAA3E0F91200959290081A69EEF0A3EFF09008066BE0FBA3E0FAA3E0F9E475F099
:20D74000011200822890080660E0FBA3E0FAA3E0F9E475F00E120082289008066BE0FBA3A0
:20D76000E0FAA3E0F9120081AEC39401FFE5F09400FE90081EA1F0A3EFF0C39403EE64805F
:20D780009480401790080660E0FBA3E0FAA3E0F9E475F00F120082287F002290081EA2E05F
:20D7A000FF7B097A1E79A312023436E490081E9DF0A3F090081E9DE0FCA3E0FDC39402EC06
:20D7C00064809480400301D85E90081EA1E0FEA3E07802C333CE33CED8F92DFFEC3E900821
:20D7E0001E9FF0A3EFF090081E9FE0FEA3E07802C333CE33CED8F924C3F974213EFA7B0903
:20D8000078A37C1E7D097E007F04120087C7EF703A90081E9FE0FEA3E0900822A075F0035B
:20D820001200843BEE75F003A42583F583759308E0FBA3E0FAA3E02401F9E43AFA90081E26
:20D84000A7EBF0A3EAF0A3E9F0801390081E9EE004F0700790081E9DE004F001D7B39008D1
:20D860001E9DE07004A3E06402700F90081EA77483F0A37483F0A374CAF090081976E0FB90
:20D88000A3E0FAA3E0F990081A69E0FEA3E0FFE92FF9EA3EFAC002C001900823FF7483F0BD
:20D8A000A37483F0A374D2F090081EA2E02401FE90081EA1E0340090082402F0A3CEF090A0
:20D8C000081EA7E0F9A3E0FAA3E090082404C9F0A3EAF0A3E9F0D001D002120095929008BC
:20D8E0001A6AE02FF090081A69E03EF09008066BE0FBA3E0FAA3E0F9E475F001120081FCC6
:20D9000001D75978FD7C1E7D097B817A9079727E007F0C12008055900828D57409F0A37447
:20D920001EF0A374FCF0A37409F0A3741EF0A374FAF07B097A1E79FBE4FF12022B2A90082C
:20D940001976E0FBA3E0FAA3E0F990081A69E0FEA3E0FFE92FF9EA3EFAC002C00190082378
:20D96000FF7483F0A37484F0A3740EF090081EFAE075F003A424FDF582E4341EF583759337
:20D9800008E0F9A3E0FAA3E090082402C9F0A3EAF0A3E9F0D001D0021200959290081A6A3E
:20D9A000E02FF090081A69E03EF090081EFAE0701278AA7C1E7D097B837A8279D41200860C
:20D9C00093802A900823FF7483F0A37484F0A374C0F090081EFBE004FFF090082402E4F001
:20D9E000A3EFF07B097A1E79AA1200959290081976E0FBA3E0FAA3E0F990081A69E0FEA396
:20DA0000E0FFE92FF9EA3EFA900823FF7483F0A37484F0A374C5F0A37409F0A3741EF0A324
:20DA200074AAF01200959290081A6AE02FF090081A69E03EF090081EFAE0701278AA7C1E8D
:20DA40007D097B837A8279D412008693802A900823FF7483F0A37484F0A374C0F090081E7B
:20DA6000FCE004FFF090082402E4F0A3EFF07B097A1E79AA1200959290081976E0FBA3E0C6
:20DA8000FAA3E0F990081A69E0FEA3E0FFE92FF9EA3EFA900823FF7483F0A37484F0A3741F
:20DAA000F6F0A37409F0A3741EF0A374AAF01200959290081A6AE02FF090081A69E03EF01D
:20DAC00090080660E0FBA3E0FAA3E0F9E475F001120081FC01DC0912023E50EF64017070DF
:20DAE00090081976E0FBA3E0FAA3E0F990081A69E0FEA3E0FFE92FF9EA3EFA900823FF744F
:20DB000083F0A37485F0A37426F01200959290081A6AE02FF090081A69E03EF09008066B53
:20DB2000E0FBA3E0FAA3E0F9E4F5F01200822890080660E0FBA3E0FAA3E0F9E475F013124C
:20DB4000008228E4FFFE1201AFADEF4E7067FF2212023E50EF6402705C900823FF7483F032
:20DB6000A37485F0A37459F090081976E0FBA3E0FAA3E0F91200959290081A69EEF0A3EFFA
:20DB8000F09008066BE0FBA3E0FAA3E0F9E4F5F01200822890080660E0FBA3E0FAA3E0F961
:20DBA000E475F01712008228E4FFFE1200EADCEF4E7002FF2290081976E0FBA3E0FAA3E0BE
:20DBC000F990081A69E0FEA3E0FFE92FF9EA3EFA900823FF7483F0A37485F0A3748EF012CA
:20DBE00000959290081A6AE02FF090081A69E03EF090080660E0FBA3E0FAA3E0F9E4F5F01F
:20DC00001200822880037F01227F002290082956EBF0A3EAF0A3E9F07E00900829B3740928
:20DC2000F0A37429F0A3745CF07B097A29795A1202285D90082959E0FF14700301DD9B14C1
:20DC4000700301DE5614700301E05A24FE700301E1D114700301E28C2406600301E37790A4
:20DC600008295DE0FD90082956E0F9A3E0FAA3E090082A78C9F0A3EAF0A3E9F0E4FB12026A
:20DC800033F890082959E0FF9008295DE0FD90082956E0FBA3E0FAA3E02404F9E43AFA90AA
:20DCA000082A78EBF0A3EAF0A3E9F07B01120233F890082959E0FF9008295DE0FD90082976
:20DCC00056E0FBA3E0FAA3E02408F9E43AFA90082A78EBF0A3EAF0A3E9F07B02120233F80C
:20DCE00090082959E0FF9008295DE0FD90082956E0FBA3E0FAA3E0240CF9E43AFA90082A3B
:20DD000078EBF0A3EAF0A3E9F07B03120233F890082959E0FF9008295DE0FD90082956E00F
:20DD2000FBA3E0FAA3E02410F9E43AFA90082A78EBF0A3EAF0A3E9F07B04120233F890083F
:20DD40002959E0FF9008295DE0FD90082956E0FBA3E0FAA3E02414F9E43AFA90082A78EB07
:20DD6000F0A3EAF0A3E9F07B05120233F890082959E0FF9008295DE0FD90082956E0FBA372
:20DD8000E0FAA3E02418F9E43AFA90082A78EBF0A3EAF0A3E9F07B0601E37390082959E0F9
:20DDA000FF9008295DE0FD90082956E0FBA3E0FAA3E0241CF9E43AFA90082A78EBF0A3EA84
:20DDC000F0A3E9F0E4FB120233F890082959E0FF9008295DE0FD90082956E0FBA3E0FAA3B3
:20DDE000E02420F9E43AFA90082A78EBF0A3EAF0A3E9F07B01120233F890082959E0FF909C
:20DE000008295DE0FD90082956E0FBA3E0FAA3E02424F9E43AFA90082A78EBF0A3EAF0A317
:20DE2000E9F07B02120233F890082959E0FF9008295DE0FD90082956E0FBA3E0FAA3E02443
:20DE400028F9E43AFA90082A78EBF0A3EAF0A3E9F07B0301E37390082959E0FF9008295D8F
:20DE6000E0FD90082956E0FBA3E0FAA3E0242CF9E43AFA90082A78EBF0A3EAF0A3E9F0E480
:20DE8000FB120233F890082959E0FF9008295DE0FD90082956E0FBA3E0FAA3E02430F9E431
:20DEA0003AFA90082A78EBF0A3EAF0A3E9F07B01120233F890082959E0FF9008295DE0FD71
:20DEC00090082956E0FBA3E0FAA3E02434F9E43AFA90082A78EBF0A3EAF0A3E9F07B02124A
:20DEE0000233F890082959E0FF9008295DE0FD90082956E0FBA3E0FAA3E02438F9E43AFAA2
:20DF000090082A78EBF0A3EAF0A3E9F07B03120233F890082959E0FF9008295DE0FD9008AA
:20DF20002956E0FBA3E0FAA3E0243CF9E43AFA90082A78EBF0A3EAF0A3E9F07B0412023342
:20DF4000F890082959E0FF9008295DE0FD90082956E0FBA3E0FAA3E02440F9E43AFA9008D6
:20DF60002A78EBF0A3EAF0A3E9F07B05120233F890082959E0FF9008295DE0FD9008295661
:20DF8000E0FBA3E0FAA3E02444F9E43AFA90082A78EBF0A3EAF0A3E9F07B07120233F890CE
:20DFA000082959E0FF9008295DE0FD90082956E0FBA3E0FAA3E02448F9E43AFA90082A7854
:20DFC000EBF0A3EAF0A3E9F07B08120233F890082959E0FF9008295DE0FD90082956E0FBC5
:20DFE000A3E0FAA3E0244CF9E43AFA90082A78EBF0A3EAF0A3E9F07B09120233F89008290E
:20E0000059E0FF9008295DE0FD90082956E0FBA3E0FAA3E02450F9E43AFA90082A78EBF041
:20E02000A3EAF0A3E9F07B0A120233F890082959E0FF9008295DE0FD90082956E0FBA3E0BA
:20E04000FAA3E02454F9E43AFA90082A78EBF0A3EAF0A3E9F07B0B01E37390082959E0FFD6
:20E060009008295DE0FD90082956E0FBA3E0FAA3E02458F9E43AFA90082A78EBF0A3EAF094
:20E08000A3E9F0E4FB120233F890082959E0FF9008295DE0FD90082956E0FBA3E0FAA3E000
:20E0A000245CF9E43AFA90082A78EBF0A3EAF0A3E9F07B01120233F890082959E0FF900875
:20E0C000295DE0FD90082956E0FBA3E0FAA3E02460F9E43AFA90082A78EBF0A3EAF0A3E938
:20E0E000F07B02120233F890082959E0FF9008295DE0FD90082956E0FBA3E0FAA3E0246406
:20E10000F9E43AFA90082A78EBF0A3EAF0A3E9F07B03120233F890082959E0FF9008295D0C
:20E12000E0FD90082956E0FBA3E0FAA3E02468F9E43AFA90082A78EBF0A3EAF0A3E9F07BEA
:20E1400004120233F890082959E0FF9008295DE0FD90082956E0FBA3E0FAA3E0246CF9E429
:20E160003AFA90082A78EBF0A3EAF0A3E9F07B05120233F890082959E0FF9008295DE0FDAA
:20E1800090082956E0FBA3E0FAA3E02470F9E43AFA90082A78EBF0A3EAF0A3E9F07B061247
:20E1A0000233F890082959E0FF9008295DE0FD90082956E0FBA3E0FAA3E02474F9E43AFAA3
:20E1C00090082A78EBF0A3EAF0A3E9F07B0701E37390082959E0FF9008295DE0FD900829A3
:20E1E00056E0FBA3E0FAA3E02478F9E43AFA90082A78EBF0A3EAF0A3E9F0E4FB120233F815
:20E2000090082959E0FF9008295DE0FD90082956E0FBA3E0FAA3E0247CF9E43AFA90082AA5
:20E2200078EBF0A3EAF0A3E9F07B01120233F890082959E0FF9008295DE0FD90082956E0EC
:20E24000FBA3E0FAA3E02480F9E43AFA90082A78EBF0A3EAF0A3E9F07B02120233F89008AC
:20E260002959E0FF9008295DE0FD90082956E0FBA3E0FAA3E02484F9E43AFA90082A78EB72
:20E28000F0A3EAF0A3E9F07B0301E37390082959E0FF9008295DE0FD90082956E0FBA3E057
:20E2A000FAA3E02488F9E43AFA90082A78EBF0A3EAF0A3E9F0E4FB120233F890082959E0FE
:20E2C000FF9008295DE0FD90082956E0FBA3E0FAA3E0248CF9E43AFA90082A78EBF0A3EAEF
:20E2E000F0A3E9F07B01120233F890082959E0FF9008295DE0FD90082956E0FBA3E0FAA3F1
:20E30000E02490F9E43AFA90082A78EBF0A3EAF0A3E9F07B02120233F890082959E0FF9005
:20E3200008295DE0FD90082956E0FBA3E0FAA3E02494F9E43AFA90082A78EBF0A3EAF0A382
:20E34000E9F07B03120233F890082959E0FF9008295DE0FD90082956E0FBA3E0FAA3E0241D
:20E3600098F9E43AFA90082A78EBF0A3EAF0A3E9F07B04120233F82290080660E0FBA3E0AA
:20E38000FAA3E0F9E475F001120081D2AFF0FE600301EAD6EF24FE700301E9C114700301E0
:20E3A000EA3D2402600301EAD6900828327483F0A37463F0A374CDF090081976E0FBA3E050
:20E3C000FAA3E0F9120207F5900820BAEBF0A3EAF0A3E9F0900823017483F0A37463F0A3C1
:20E3E00074D6F0A37409F0A37420F0A374BDF012009971900820BFE4F0A374F0F0E0246422
:20E40000F0900820BFE03400F0900823FF7483F0A37463F0A374E1F0900820BDE0FEA3E0C8
:20E42000FF90082402EEF0A3EFF0900820BFE0FDA3E090082404CDF0A3EDF0EF2401FFE4F4
:20E440003EA3F0A3EFF090081976E0FBA3E0FAA3E0F91200959290081A69EEF0A3EFF0902A
:20E460000820BDE0F9A3E0FF9008066BE0FBA3E0FAA3E0C98FF012008228900820BEE0FF1F
:20E4800012023BF4900820C1EEF0A3EFF0900820BEE0FF7B097A2079D91201F03B7B097A5F
:20E4A0002079DD120237C9900820C1E07004A3E06404600301E59290081976E0FBA3E0FAC0
:20E4C000A3E0F990081A69E0FEA3E0FFE92FF9EA3EFA900823FF7483F0A37466F0A37411DC
:20E4E000F01200959290081A6AE02FF090081A69E03EF0900820BEE0FF120236D9EF4E708A
:20E50000087B837A66793A8031900820D9E0C4F854F0C8A3E0C4540F48540F90082369758A
:20E52000F0031200843BE475F003A42583F583759308E0FBA3E0FAA3E0F9900820BAEBF0D6
:20E54000A3EAF0A3E9F090081976E0FBA3E0FAA3E0F990081A69E0FEA3E0FFE92FF9EA3E13
:20E56000FAC002C001900823FF7483F0A37466F0A37447F0900820BAE0F9A3E0FAA3E090E7
:20E58000082402C9F0A3EAF0A3E9F0D001D00201E78C90081976E0FBA3E0FAA3E0F99008F1
:20E5A0001A69E0FEA3E0FFE92FF9EA3EFA900823FF7483F0A37466F0A3744FF012009592A8
:20E5C00090081A6AE02FF090081A69E03EF0900820C1E0FEA3E0FF64024E7003A38071EF74
:20E5E00064034E6006EF64054E706C90081976E0FBA3E0FAA3E0F990081A69E0FEA3E0FF08
:20E60000E92FF9EA3EFAC002C001900823FF7483F0A37466F0A37485F0E4A3F0A3F0900808
:20E620002369E0F9A3E0FAA3E090082404C9F0A3EAF0A3E9F0D001D0021200959290081A75
:20E640006AE02FF090081A69E03EF0900820C3E4F0A37405F08009900820C3E4F0A304F05E
:20E66000900820C3E0FFA3E0900820B8CFF0A3EFF0900820B8E0FEA3E0FFD39406EE6480FD
:20E680009480400301E7627C00900820DAE0540FFDEFB5050CECB506087B837A66799A80B6
:20E6A000067B837A6679A3900820BAEBF0A3EAF0A3E9F090081976E0FBA3E0FAA3E0F99089
:20E6C000081A69E0FEA3E0FFE92FF9EA3EFAC003C002C001900823FF7483F0A37466F0A325
:20E6E00074A4F0900820B8E0FEA3E0FF90082402EEF0A3EFF0900820BAE0F9A3E0FAA3E0D9
:20E7000090082404C9F0A3EAF0A3E9F09008236975F003EF1200843BEE75F003A42583F5A4
:20E7200083759308E0F9A3E0FAA3E090082407C9F0A3EAF0A3E9F0D001D002D003120095DB
:20E740009290081A6AE02FF090081A69E03EF0900820B9E004F07007900820B8E004F001E2
:20E76000E67190081976E0FBA3E0FAA3E0F990081A69E0FEA3E0FFE92FF9EA3EFA900823DE
:20E78000FF7483F0A37466F0A374BDF01200959290081A6AE02FF090081A69E03EF078C5A8
:20E7A0007C207D097B837A6679C912008693900820DAE0540F64056019900829A07483F0ED
:20E7C000A37466F0A374CEF07B097A2079C51202253D90081976E0FBA3E0FAA3E0F9900892
:20E7E0001A69E0FEA3E0FFE92FF9EA3EFAC002C001900823FF7481F0A37490F0A37482F0C1
:20E80000A37409F0A37420F0A374C5F0E4A3F0A3F09008235DE0F9A3E0FAA3E09008240737
:20E82000C9F0A3EAF0A3E9F0D001D0021200959290081A6AE02FF090081A69E03EF090086E
:20E8400020D9E030E0087B837A66799A80067B837A6679A3900820BAEBF0A3EAF0A3E9F010
:20E8600090081976E0FBA3E0FAA3E0F990081A69E0FEA3E0FFE92FF9EA3EFAC002C00190DC
:20E880000823FF7483F0A37466F0A374D8F0A3E4F0A304F0900820BAE0F9A3E0FAA3E09032
:20E8A000082404C9F0A3EAF0A3E9F090082360E0F9A3E0FAA3E090082407C9F0A3EAF0A3E6
:20E8C000E9F0D001D0021200959290081A6AE02FF090081A69E03EF090081976E0FBA3E0BA
:20E8E000FAA3E0F990081A69E0FEA3E0FFE92FF9EA3EFA900823FF7483F0A37466F0A374CF
:20E90000FCF01200959290081A6AE02FF090081A69E03EF0900820BEE024DDF582E4342088
:20E92000F583759308E0B401087B837A66799A80067B837A6679A3900820BAEBF0A3EAF077
:20E94000A3E9F090081976E0FBA3E0FAA3E0F990081A69E0FEA3E0FFE92FF9EA3EFAC003CF
:20E96000C002C001900823FF7483F0A37467F0A37416F090082357E0F9A3E0FAA3E0900865
:20E980002402C9F0A3EAF0A3E9F0900820BAE0F9A3E0FAA3E090082405C9F0A3EAF0A3E9D1
:20E9A000F09008235AE0F9A3E0FAA3E090082408C9F0A3EAF0A3E9F0D001D002D00301EAA2
:20E9C000C29008066BE0FBA3E0FAA3E0F9120081AEFF900820BDE5F0F0A3EFF0A3E4F0A382
:20E9E00074F0F0E02464F0900820BFE03400F0900820BEE0FF7B097A2079D91201F03B905D
:20EA0000081976E0FBA3E0FAA3E0F990081A69E0FEA3E0FFE92FF9EA3EFA900823FF74832C
:20EA2000F0A37467F0A37450F0900820BFE0FFA3E090082402CFF0A3EFF001EAC2900823E1
:20EA4000FF7483F0A37468F0A3743DF0A3E4F0A37406F09008066BE0FBA3E0FAA3E0F912AA
:20EA60000081AE2401FEE435F090082404F0A3CEF0E4A3F0A3F0A3F0A37405F0900819765A
:20EA8000E0FBA3E0FAA3E0F91200959290081A69EEF0A3EFF090081976E0FBA3E0FAA3E0EC
:20EAA0002FF9EA3EFA900823FF7483F0A3746AF0A374C2F0A3E4F0A37406F0A3E4F0A3741F
:20EAC00005F01200959290081A6AE02FF090081A69E03EF080037F01227F002290081FC186
:20EAE000EEF0A3EFF09008066BE0FBA3E0FAA3E0F9120081AE45F0600301EBB69008197637
:20EB0000E0FBA3E0FAA3E0F990081A69E0FEA3E0FFE92FF9EA3EFA900823FF7483F0A374BB
:20EB20009AF0A37438F01200959290081A6AE02FF090081A69E03EF0E490081FC3F0A3F0AE
:20EB400090081976E0FBA3E0FAA3E0F990081A69E0FEA3E0FFE92FF9EA3EFA900823FF74DE
:20EB600083F0A3749AF0A37466F01200959290081A6AE02FF090081A69E03EF090081FC41C
:20EB8000E004F0700790081FC3E004F0C390081FC4E0940490081FC3E06480948040A19063
:20EBA00008066BE0FBA3E0FAA3E0F9E475F0011200822801F1B59008066BE0FBA3E0FAA357
:20EBC000E0F9120081AEFFAEF0D39408EE9400400301ED3AEF64014E703C90081976E0FBD2
:20EBE000A3E0FAA3E0F990081A69E0FEA3E0FFE92FF9EA3EFA900823FF7483F0A3749AF02C
:20EC0000A37480F01200959290081A6AE02FF090081A69E03EF07B097A1F79D51202381D1C
:20EC200090081976E0FBA3E0FAA3E0F990081A69E0FEA3E0FFE92FF9EA3EFA900823FF74FD
:20EC400083F0A3749AF0A374B7F01200959290081A6AE02FF090081A69E03EF0E490081FCA
:20EC6000C3F0A3F012020BEA90081976E0FBA3E0FAA3E0F990081A69E0FEA3E0FFE92FF9BE
:20EC8000EA3EFAC003C002C001900823FF7483F0A3749AF0A374CBF09008066BE0FBA3E091
:20ECA000FAA3E0F9120081AEFF90082402E5F0F0A3EFF0A37409F0A3741FF0A374C9F0D0C3
:20ECC00001D002D0031200959290081A6AE02FF090081A69E03EF090081FC7E0FEA3E0FF33
:20ECE00024D5F582E4341FF583759308E0FD7C0090081FC1E0FAA3E0FB1201B973900806DF
:20ED00006BE0FBA3E0FAA3E0F9E475F001120081FC90081FC4E004F0700790081FC3E004B7
:20ED2000F0D390081FC4E0940390081FC3E064809480500301EC6401F1B59008066BE0FB9D
:20ED4000A3E0FAA3E0F9120081AEFFAEF0D39414EE9400400301EEE4EF64094E703C9008DB
:20ED60001976E0FBA3E0FAA3E0F990081A69E0FEA3E0FFE92FF9EA3EFA900823FF7483F0E1
:20ED8000A3749AF0A374E8F01200959290081A6AE02FF090081A69E03EF07B097A1F79D5FB
:20EDA0001202381D90081976E0FBA3E0FAA3E0F990081A69E0FEA3E0FFE92FF9EA3EFA90B1
:20EDC0000823FF7483F0A3749AF0A374B7F01200959290081A6AE02FF090081A69E03EF046
:20EDE0009008066BE0FBA3E0FAA3E0F9120081AEC39405FFE5F09400FEEF7802CEC313CE58
:20EE000013D8F9FF90081FC3EEF0A3EFF0A3E4F0A304F012020BEA90081976E0FBA3E0FA9F
:20EE2000A3E0F990081A69E0FEA3E0FFE92FF9EA3EFA900823FF7483F0A3749BF0A374232B
:20EE4000F090081FC5E0FFA3E090082402CFF0A3EFF090081FC3E0FFA3E090082404CFF08A
:20EE6000A3EFF0A37409F0A3741FF0A374C9F01200959290081A6AE02FF090081A69E03E7D
:20EE8000F090081FC7E0FEA3E0FF24D5F582E4341FF583759308E0FD7C0090081FC1E0FACA
:20EEA000A3E0FB1201B9739008066BE0FBA3E0FAA3E0F9E475F001120081FC90081FC6E082
:20EEC00004F0700790081FC5E004F0D390081FC6E0940490081FC5E064809480500301EE19
:20EEE0001301F1B59008066BE0FBA3E0FAA3E0F9120081AE641545F0600301EFCC7B097A6F
:20EF00001F79D51202381D12020BEA90081976E0FBA3E0FAA3E0F990081A69E0FEA3E0FF9C
:20EF2000E92FF9EA3EFA900823FF7483F0A3749BF0A37442F0A37409F0A3741FF0A374C9FC
:20EF4000F01200959290081A6AE02FF090081A69E03EF090081FC7E0FEA3E0FF24D5F582F6
:20EF6000E4341FF583759308E0FD7C0090081FC1E0FAA3E0FB1201B97390081976E0FBA3C5
:20EF8000E0FAA3E0F990081A69E0FEA3E0FFE92FF9EA3EFA900823FF7483F0A3749BF0A387
:20EFA00074BEF01200959290081A6AE02FF090081A69E03EF09008066BE0FBA3E0FAA3E0CE
:20EFC000F9E475F001120081FC01F1B59008066BE0FBA3E0FAA3E0F9120081AEFFAEF0C33A
:20EFE0009440EE9400400301F1B0EF64164E703C90081976E0FBA3E0FAA3E0F990081A695D
:20F00000E0FEA3E0FFE92FF9EA3EFA900823FF7483F0A3749BF0A374D6F01200959290086C
:20F020001A6AE02FF090081A69E03EF07B097A1F79D51202381D90081976E0FBA3E0FAA32E
:20F04000E0F990081A69E0FEA3E0FFE92FF9EA3EFA900823FF7483F0A3749AF0A374B7F029
:20F060001200959290081A6AE02FF090081A69E03EF090081FC5E4F0A304F012020BEA9093
:20F08000081976E0FBA3E0FAA3E0F990081A69E0FEA3E0FFE92FF9EA3EFA900823FF7483A6
:20F0A000F0A3749CF0A37420F090081FC7E0FFA3E090082402CFF0A3EFF0A37409F0A37490
:20F0C0001FF0A374C9F01200959290081A6AE02FF090081A69E03EF090081FC7E0FEA3E0F5
:20F0E000FF24D5F582E4341FF583759308E0FD7C0090081FC1E0FAA3E0FB1201B9739008E2
:20F10000066BE0FBA3E0FAA3E0F9E475F001120081FC9008066BE0FBA3E0FAA3E0F91200E2
:20F1200081AED39440E5F09400405D90081976E0FBA3E0FAA3E0F990081A69E0FEA3E0FF7D
:20F14000E92FF9EA3EFA900823FF7483F0A3749CF0A3743AF090081FC5E0FEA3E0FFC374E4
:20F16000049FFFE49EFEEF25E0FFEE3390082402F0A3EFF01200959290081A6AE02FF09045
:20F18000081A69E03EF0802D90081FC6E004F0700790081FC5E004F0D390081FC6E0940449
:20F1A00090081FC5E064809480500301F07B80057E007F0122E4FEFF2290080660E0FBA318
:20F1C000E0FAA3E0F9120081AEFFAEF0E5F0600301F85CEF24FE700301F44714700301F432
:20F1E0004714700301F6C014700301F81F2404600301F85C900823FF7483F0A37476F0A34A
:20F20000748BF090081976E0FBA3E0FAA3E0F91200959290081A69EEF0A3EFF0900822375F
:20F22000E4F0A304F090082237E0FEA3E0FFD39403EE64809480400301F3F8EE600301F34E
:20F2400052EF14605914700301F2CC14700301F3042403600301F35290082235E4F0A37431
:20F2600005F0900822327483F0A37477F0A37452F09008222F7483F0A37477F0A37462F038
:20F2800012023DAB90082402EEF0A3EFF0900823FF7483F0A37477F0A3746601F3479008E5
:20F2A0002235E4F0A37414F0900822327483F0A37477F0A37469F09008222F7483F0A37460
:20F2C00077F0A37475F012023E73802C90082235E4F0A37414F0900822327483F0A374779B
:20F2E000F0A37479F09008222F7483F0A37477F0A37487F012023E7A78077C227D09120041
:20F300008693804E90082235E4F0A37402F0900822327483F0A37477F0A3748BF09008229D
:20F320002F7483F0A37477F0A374B4F012023DE790082402EEF0A3EFF0900823FF7483F087
:20F34000A37477F0A374BAF07B097A2279071200959290081976E0FBA3E0FAA3E0F9900802
:20F360001A69E0FEA3E0FFE92FF9EA3EFAC003C002C001900823FF7483F0A37477F0A374FB
:20F38000BDF090082232E0F9A3E0FAA3E090082402C9F0A3EAF0A3E9F09008222FE0F9A326
:20F3A000E0FAA3E090082405C9F0A3EAF0A3E9F0A37409F0A37422F0A37407F09008223547
:20F3C000E0FFA3E09008240BCFF0A3EFF0D001D002D0031200959290081A6AE02FF0900861
:20F3E0001A69E03EF090082238E004F0700790082237E004F001F22590081976E0FBA3E0DD
:20F40000FAA3E0F990081A69E0FEA3E0FFE92FF9EA3EFA900823FF7483F0A37478F0A37491
:20F4200019F01200959290081A6AE02FF090081A69E03EF090080660E0FBA3E0FAA3E0F974
:20F44000E475F00201F85690082239E4F0A304F090082239E0FEA3E0FFD39403EE64809491
:20F4600080400301F671EE707EEF24FE602B14604C24027072900822327483F0A37478F0CF
:20F48000A37441F09008222F7483F0A37478F0A3744CF012023CB18046900822327483F0E8
:20F4A000A37478F0A3744FF09008222F7483F0A37478F0A3745BF012023CC1802290082259
:20F4C000327483F0A37478F0A3745EF09008222F7483F0A37478F0A37466F012023CD190C2
:20F4E0000822031200842F90081976E0FBA3E0FAA3E0F990081A69E0FEA3E0FFE92FF9EAA9
:20F500003EFAC002C001900823FF7483F0A37478F0A37469F090082232E0F9A3E0FAA3E0DB
:20F5200090082402C9F0A3EAF0A3E9F0D001D0021200959290081A6AE02FF090081A69E069
:20F540003EF090082237E4F0A304F012023DF9EF64014E900819767047E0FBA3E0FAA3E07C
:20F56000F990081A69E0FEA3E0FFE92FF9EA3EFAC002C001900823FF7483F0A37478F0A39E
:20F580007486F09008222FE0F9A3E0FAA3E090082402C9F0A3EAF0A3E9F0D001D0028076B6
:20F5A000E0FBA3E0FAA3E0F990081A69E0FEA3E0FFE92FF9EA3EFAC003C002C001900823C8
:20F5C000FF7483F0A37478F0A374B7F09008222FE0F9A3E0FAA3E090082402C9F0A3EAF052
:20F5E000A3E9F090082238E075F008A4FFC374209FF990082203E0FCA3E0FDA3E0FEA3E0A1
:20F60000FFA8011200837FE490082405F0A3EFF0D001D002D0031200959290081A6AE02F3D
:20F62000F090081A69E03EF090082238E004F0700790082237E004F0D390082238E0940472
:20F6400090082237E064809480500301F54B90081A6AE024FEF090081A69E034FFF0900889
:20F66000223AE004F0700790082239E004F001F45090081976E0FBA3E0FAA3E0F990081A2A
:20F6800069E0FEA3E0FFE92FF9EA3EFA900823FF7483F0A37478F0A374F1F012009592908D
:20F6A000081A6AE02FF090081A69E03EF090080660E0FBA3E0FAA3E0F9E475F00401F85628
:20F6C00012023CB1900822031200842F900823FF7483F0A37479F0A3749AF090082203E048
:20F6E000FCA3E0FDA3E0FEA3E0FF78181200837FE490082402F0A3EFF090082203E0FCA397
:20F70000E0FDA3E0FEA3E0FF78101200837FE490082404F0A3EFF090082203E0FCA3E0FD3E
:20F72000A3E0FEA3E0FF78081200837FE490082406F0A3EFF090082203E0FCA3E0FDA3A3BB
:20F74000E0FEE490082408F0A3CEF090081976E0FBA3E0FAA3E0F91200959290081A69EE95
:20F76000F0A3EFF090081976E0FBA3E0FAA3E02FF9EA3EFA900823FF7483F0A37479F0A307
:20F7800074D4F01200959290081A6AE02FF090081A69E03EF090081976E0FBA3E0FAA3E0B2
:20F7A000F990081A69E0FEA3E0FFE92FF9EA3EFA900823FF7483F0A3747AF0A374AEF012B9
:20F7C00000959290081A6AE02FF090081A69E03EF090081976E0FBA3E0FAA3E0F990081A11
:20F7E00069E0FEA3E0FFE92FF9EA3EFA900823FF7483F0A3747BF0A37451F01200959290C9
:20F80000081A6AE02FF090081A69E03EF090080660E0FBA3E0FAA3E0F9E475F005803790CD
:20F820000823FF7483F0A3747CF0A374C2F090081976E0FBA3E0FAA3E0F91200959290089F
:20F840001A69EEF0A3EFF090080660E0FBA3E0FAA3E0F9E4F5F01200822880037F01227FCA
:20F860000022E4900828EFF0900828EFE0FF04F0EFC3940A5059E47F807E80FDFC900828CE
:20F88000F51200842F900828F5E0FCA3E0FDA3E0FEA3E0FF90082A711200842F7F147E0091
:20F8A00012022DA97B097A2879F57F147E00120232F5E47F807E80FDFC900828F5E0F8A374
:20F8C000E0F9A3E0FAA3E0FBC31200836E7099900828EFE0B40A0412023AE4E47F81FEFD23
:20F8E000FC900828F51200842F900828F5E0FCA3E0FDA3E0FEA3E0FF90082A711200842F86
:20F900007F177E0012022DA9E4FF7E04FDFC900828F51200842F900828F5E0FCA3E0FDA35D
:20F92000E0FEA3E0FF90082A711200842F7F187E0012022DA9E47F747E88FDFC900828F5E5
:20F940001200842F900828F5E0FCA3E0FDA3E0FEA3E0FF90082A711200842F7F1C7E0012AB
:20F96000022DA9E47F807E11FDFC900828F51200842F900828F5E0FCA3E0FDA3E0FEA3E0B5
:20F98000FF90082A711200842F7F1D7E0012022DA9E47F2C7E01FDFC900828F51200842FEB
:20F9A000900828F5E0FCA3E0FDA3E0FEA3E0FF90082A711200842F7F1E7E0012022DA9E452
:20F9C000FFFEFDFC900828F51200842F900828F5E0FCA3E0FDA3E0FEA3E0FF90082A71125E
:20F9E00000842F7F267E0012022DA9E47FA07EFCFDFC900828F51200842F900828F5E0FCC6
:20FA0000A3E0FDA3E0FEA3E0FF90082A711200842F7F687E0012022DA9E47F417EFAFDFC07
:20FA2000900828F51200842FE4900828EFF0900828EFE0FFC394025033EF2469FFE433FECF
:20FA4000C006C007900828F5E0FCA3E0FDA3E0FEA3E0FF90082A711200842FD007D006124E
:20FA6000022DA9900828EFE004F080C2E47F417EFAFDFC900828F51200842FE4900828EFC7
:20FA8000F0900828EFE0FFC394025033EF246BFFE433FEC006C007900828F5E0FCA3E0FDDC
:20FAA000A3E0FEA3E0FF90082A711200842FD007D00612022DA9900828EFE004F080C2E40B
:20FAC0007F107E20FDFC900828F51200842F900828F5E0FCA3E0FDA3E0FEA3E0FF90082AB0
:20FAE000711200842F7F6D7E0012022DA9E47F047E08FDFC900828F51200842F900828F567
:20FB0000E0FCA3E0FDA3E0FEA3E0FF90082A711200842F7F6E7E0012022DA9E47F087E1040
:20FB2000FDFC900828F51200842F900828F5E0FCA3E0FDA3E0FEA3E0FF90082A7112008475
:20FB40002F7F6F7E0012022DA9E47F027E04FDFC900828F51200842F900828F5E0FCA3E0B2
:20FB6000FDA3E0FEA3E0FF90082A711200842F7F707E0012022DA9E4900828EFF0900828F3
:20FB8000EFE0FBC39404400301FC18E4FF7E01FDFC900828F51200842FEB75F002A4247188
:20FBA000FFE435F0FEC006C007900828F5E0FCA3E0FDA3E0FEA3E0FF90082A711200842FA6
:20FBC000D007D00612022DA9E4FFFEFDFC900828F51200842F900828EFE075F002A424710B
:20FBE000FFE435F0CF2401CF3400FEC006C007900828F5E0FCA3E0FDA3E0FEA3E0FF9008CF
:20FC00002A711200842FD007D00612022DA9900828EFE004F001FB7DE47F087E08FDFC9077
:20FC20000828F51200842F900828F5E0FCA3E0FDA3E0FEA3E0FF90082A711200842F7F79D6
:20FC40007E0012022DA9E47F1E7E14FDFC900828F51200842F900828F5E0FCA3E0FDA3E022
:20FC6000FEA3E0FF90082A711200842F7F7A7E0012022DA9E4FFFEFDFC900828F512008486
:20FC80002F900828F5E0FCA3E0FDA3E0FEA3E0FF90082A711200842F7F7B7E0012022DA9C7
:20FCA000E47F207E40FDFC900828F51200842F900828F5E0FCA3E0FDA3E0FEA3E0FF9008E4
:20FCC0002A711200842F7F817E0012022DA9E4FF7E40FDFC900828F51200842F900828F593
:20FCE000E0FCA3E0FDA3E0FEA3E0FF90082A711200842F7F8C7E0012022DA9E47F11FEFDCB
:20FD0000FC900828F51200842F900828F5E0FCA3E0FDA3E0FEA3E0FF90082A711200842F61
:20FD20007F957E0012022DA9E47F337E22FDFC900828F51200842F900828F5E0FCA3E0FD8D
:20FD4000A3E0FEA3E0FF90082A711200842F7F967E0012022DA9E47F557E44FDFC900828F8
:20FD6000F51200842F900828F5E0FCA3E0FDA3E0FEA3E0FF90082A711200842F7F977E0029
:20FD800012022DA9E4900828F0F0900828F0E0FF7E00D390082484E09F7480F8900824832B
:20FDA000E0648098500301FECC900829B37409F0A37428F0A374F3F07B097A2879F112021B
:20FDC000285D900828F3E0FAA3E0FB64184A7017FFFEFDFCA31200842FEBAE027803C333DC
:20FDE000CE33CED8F9801FE47F01FEFDFC900828F51200842F900828F3E0FEA3E07803C39D
:20FE000033CE33CED8F92403FFEE3401FEC006C007900828F5E0FCA3E0FDA3E0FEA3E0FF27
:20FE200090082A711200842FD007D00612022DA9E4FFFEFDFC900828F51200842F9008281F
:20FE4000F3E0FEA3E07803C333CE33CED8F92404FFEE3401FEC006C007900828F5E0FCA334
:20FE6000E0FDA3E0FEA3E0FF90082A711200842FD007D00612022DA9E47F017E10FDFC9098
:20FE80000828F51200842F900828F3E0FEA3E07803C333CE33CED8F92405FFEE3401FEC04A
:20FEA00006C007900828F5E0FCA3E0FDA3E0FEA3E0FF90082A711200842FD007D0061202A8
:20FEC0002DA9900828F0E004F001FD8A229008290DEFF0A3EBF0A3EAF0A3E9F012023DF0B9
:20FEE000EF4E9008290D6070E025E025E02471F582E43406F583759308E0FF9008290EE0FD
:20FF0000F9A3E0FAA3E09008277EC9F0A3EAF0A3E9F0A3E4F0A304F0A3E4F0A304F07B0959
:20FF20007A29791412021D0F90082913EFF0FE9008290DE0FFA3E0FBA3E0FAA3E0F9EEFD91
:20FF400090082699E4F0A3EDF0A3E4F0A304F0A3E4F0A304F001FFF6E0FF7E007B097A2960
:20FF60007911120234749008290DE025E025E02471F582E43406F583759308E0FFC007909B
:20FF800008290EE0F9A3E0FAA3E09008277EC9F0A3EAF0A3E9F090082911E0540FFFA3E0C3
:20FFA00090082781CFF0A3EFF0E4A3F0A3F07B097A297914D00712021D0F90082913EFF038
:20FFC000FE9008290EE0FBA3E0FAA3E0F9EEFD90082699E4F0A3EDF090082911E0540FFFD6
:20FFE000A3E09008269BCFF0A3EFF0E4A3F0A3F09008290DE0FF120214D3220202071EFFE8
:020000040001F9
:20000000E490082BBCF02290080660E0FBA3E0FAA3E0F9120081AEFFAEF0E5F0600321065C
:2000200064EF24FE603714607014700321021D14700321033F1470032105E82405600321DD
:2000400006647F017E0012020D5D90080660E0FBA3E0FAA3E0F9E475F00221065D9008235E
:20006000FF7483F0A3746FF0A37452F090081976E0FBA3E0FAA3E0F91200959290081A697C
:20008000EEF0A3EFF090080660E0FBA3E0FAA3E0F9E475F003120082289008066BE0FBA39F
:2000A000E0FAA3E0F9120081AEC39401FFE5F09400FE7B097A2579F5120228C5EF4E702B81
:2000C00090080660E0FBA3E0FAA3E0F9E475F00412008228D390081A6AE0940090081A69C7
:2000E000E09400500321021D7F00229008066BE0FBA3E0FAA3E0F9120081AEC39401FFE5FE
:20010000F09400FE90082BB0E0B50616A3E0B50711900825FF7483F0A3746FF0A374FDF0CC
:20012000800F900825FF7483F0A37470F0A37406F0900825F5E0FEA3E0FF64014E90082686
:2001400002700D7483F0A37470F0A37407F0800B7483F0A37470F0A37406F090081976E0B7
:20016000FBA3E0FAA3E0F990081A69E0FCA3E0FDE92DF9EA3CFAC003C002C001900823FFE5
:200180007483F0A37470F0A37417F09008066BE0FBA3E0FAA3E0F9120081AEFD900824020A
:2001A000E5F0F0A3EDF0900825FFE0F9A3E0FAA3E090082404C9F0A3EAF0A3E9F0A3EEF072
:2001C000A3EFF090082602E0F9A3E0FAA3E090082409C9F0A3EAF0A3E9F0D001D002D00317
:2001E0001200959290081A6AE02FF090081A69E03EF09008066BE0FBA3E0FAA3E0F9E4754C
:20020000F001120081FCC390081A6AE094B090081A69E0940450032100997F002290081969
:2002200076E0FBA3E0FAA3E0F990081A69E0FEA3E0FFE92FF9EA3EFA900823FF7483F0A382
:200240007470F0A37433F01200959290081A6AE02FF090081A69E03EF0900825F1E4F0A3EE
:2002600004F0C390082484E09401FF90082483E09400FE900825F1E0FCA3E0FDD39FEE6494
:2002800080F8EC648098505490081976E0FBA3E0FAA3E0F990081A69E0FEA3E0FFE92FF953
:2002A000EA3EFA900823FF7483F0A37470F0A374F1F0A3ECF0A3EDF01200959290081A6AB8
:2002C000E02FF090081A69E03EF0900825F2E004F0708F900825F1E004F0808690081976C5
:2002E000E0FBA3E0FAA3E0F990081A69E0FEA3E0FFE92FF9EA3EFA900823FF7483F0A374C4
:2003000070F0A374FFF01200959290081A6AE02FF090081A69E03EF09008066BE0FBA3E093
:20032000FAA3E0F9E475F0011200822890080660E0FBA3E0FAA3E0F9E475F00521065D900D
:20034000082BB0E0FEA3E0FF7B097A2579F5120228C5EF4E700EFE7F0AFD7B097A2579F5F8
:20036000120088519008066BE0FBA3E0FAA3E0F9120081AEFFC390082484E09401FD900868
:200380002483E09400FCD3EF9DE5F09C402B90080660E0FBA3E0FAA3E0F9E475F0061200D8
:2003A0008228D390081A6AE0940090081A69E0940050032105E87F00229008066BE0FBA318
:2003C000E0FAA3E0F9120081AEC39401FEE5F09400900825F3F0A3CEF0E490082605F0A38C
:2003E000F0900825F3E0FEA3E07803CEA2E713CE13D8F824F7F58274253EF583759308E095
:20040000FD7C00900825F4E05407F974017E00A801088005C333CE33CED8F9FBAA06EA5CCE
:20042000FEEB5D4E601090082606E004F0700790082605E004F0900825F3E0FEA3E0780386
:20044000CEA2E713CE13D8F824FBF58274253EF583759308E0FFEB5F601090082606E0044B
:20046000F0700790082605E004F090081976E0FBA3E0FAA3E0F990081A69E0FEA3E0FFE91F
:200480002FF9EA3EFA900823FF7483F0A37471F0A37447F01200959290081A6AE02FF090C7
:2004A000081A69E03EF0900825F1E4F0A37402F0900825F1E0FEA3E0FFC3EE648094805011
:2004C000032105BD90082605E0FCA3E0FDEFB50515EEB50411900825FF7483F0A37471F086
:2004E000A3744FF0800F900825FF7483F0A37470F0A37406F0900825F1E0FEA3E0FF4E9004
:20050000082602600D7483F0A37471F0A37457F0800B7483F0A37470F0A37406F0900819DA
:2005200076E0FBA3E0FAA3E0F990081A69E0FCA3E0FDE92DF9EA3CFAC003C002C0019008ED
:2005400023FF7483F0A37471F0A3745CF0900825F3E0FDA3E090082402CDF0A3EDF0A3EE1B
:20056000F0A3EFF0900825FFE0F9A3E0FAA3E090082406C9F0A3EAF0A3E9F090082602E060
:20058000F9A3E0FAA3E090082409C9F0A3EAF0A3E9F0D001D002D0031200959290081A6A20
:2005A000E02FF090081A69E03EF0900825F2E024FFF0900825F1E034FFF02104B09008064D
:2005C0006BE0FBA3E0FAA3E0F9E475F001120081FCC390081A6AE094B090081A69E094046D
:2005E00050032103647F002290082BB0E07002A3E0900825FF700D7483F0A37471F0A37488
:2006000088F0800B7483F0A37470F0A37406F0900823FF7483F0A37471F0A37491F0900823
:2006200025FFE0F9A3E0FAA3E090082402C9F0A3EAF0A3E9F090081976E0FBA3E0FAA3E04B
:20064000F91200959290081A69EEF0A3EFF090080660E0FBA3E0FAA3E0F9E4F5F0120082BE
:20066000287F00227F01229008274FEBF0A3EAF0A3E9F09008274EEFF07E00900829B374DB
:2006800009F0A37427F0A37454F07B097A2779521202285D90082755E0049008275CF090BC
:2006A00008274FE0FBA3E0FAA3E0F9120081AE540F640660032107897F807E04FDFC9008B4
:2006C00027561200842F90082754E0FEA3E07803C333CE33CED8F92400FFEE3401FEC00649
:2006E000C00790082756E0FCA3E0FDA3E0FEA3E0FF90082A711200842FD007D00612022DD9
:20070000A99008274EE0FF25E025E02474F582E43406F583759308E064017051EF25E02566
:20072000E02473F582E43406F583759308E06405703B9008274EE07D0112021BF7900827E1
:200740005A7408F0A3E4F0A3E0FF9008275AE0FAA3E0FBE4FD1202376F9008274EE0FF7D65
:200760000512021BF79008275A740880069008275A741AF0A3E4F0A3E0FF9008275AE0FAB0
:20078000A3E0FBE4FD0202376FE47F837E04FDFC900827561200842F90082754E0FEA3E0A1
:2007A0007803C333CE33CED8F92400FFEE3401FEC006C00790082756E0FCA3E0FDA3E0FE65
:2007C000A3E0FF90082A711200842FD007D00612022DA99008274FE0FBA3E0FAA3E0F91214
:2007E0000081AE540F6405600321097A90082754E07004A3E0641870032108BF9008274E29
:20080000E025E025E02474F582E43406F583759308E0B401249008275A7408F0A3E4F0A3E1
:20082000E0FF9008275AE0FAA3E0FBE4FD1202376F7F017E00120231059008274EE025E093
:2008400025E02473F582E43406F583759308E064019008275A70337405F0A374E1F0A3E00A
:20086000FF9008275AE0FAA3E0FB7D041202376F9008275A7402F0A3E4F0A3E0FF90082796
:200880005AE0FAA3E0FB7D098014E4F0A374A0F0A3E0FF9008275AE0FAA3E0FB7D04120289
:2008A000376F9008275A7413F0A37440F0A3E0FF9008275AE0FAA3E0FBE4FD1202376FE449
:2008C0007F017E16FDFC900827561200842F90082756E0FCA3E0FDA3E0FEA3E044F0FFEE9B
:2008E0004401FEEC900827561200842F90082754E0FEA3E07803C333CE33CED8F92402FF45
:20090000EE3401FEC006C00790082756E0FCA3E0FDA3E0FEA3E0FF90082A711200842FD0ED
:2009200007D00612022DA990082754E0FEA3E07803C333CE33CED8F92401FFEE3401FE7BAB
:20094000097A277956120232F590082756E0FCA3E0FDA3E0FEA3E0FFEE44C0FEEC900827D4
:20096000561200842F90082756E0FCA3E0FDA3E0FEA3E0FFEE54DF210B739008275A740893
:20098000F0A3E4F0A3E0FF9008275AE0FAA3E0FBE4FD1202376F7F017E0012023105E47FB7
:2009A000017E16FDFC900827561200842F90082756E0FCA3E0FDA3E0FEA3E0540FFFEE54B6
:2009C000FEFEEC900827561200842F9008274FE0FBA3E0FAA3E0F9120081AE540F1460302B
:2009E00014604A14606414607E24046003210A899008275A7401F0A37440F090082756E076
:200A0000FCA3E0FDA3E0FEA3E0FFEE4401FE80709008275A7421F0A3E4F090082756E0FC30
:200A2000A3E0FDA3E0FEA3E04480FF80539008275A7420F0A3E4F090082756E0FCA3E0FD17
:200A4000A3E0FEA3E04440FF80369008275A7401F0A3E4F090082756E0FCA3E0FDA3E0FE72
:200A6000A3E04420FF8019E49008275AF0A3F090082756E0FCA3E0FDA3E0FEA3E04410FFAF
:200A8000EC900827561200842F90082754E07004A3E0641860159008275CE0FF9008275AA2
:200AA000E0FAA3E0FBE4FD1202376F90082754E07004A3E0641860619008274EE025E02505
:200AC000E02473F582E43406F583759308E0640170479008275CE0FF7B097A27795A7D1106
:200AE000120233379008275AE0A320E52CA3E0FF7B097A27795A7D1E120233379008275AFF
:200B0000E0F0A3E04480F0A3E0FF9008275AE0FAA3E0FB7D1E1202376F90082754E0FEA3F2
:200B2000E07803C333CE33CED8F92402FFEE3401FEC006C00790082756E0FCA3E0FDA3E0FD
:200B4000FEA3E0FF90082A711200842FD007D00612022DA9E4FFFEFDFC9008275612008401
:200B60002F90082756E0FCA3E0FDA3E0FEA3E0FFEE4420FEEC900827561200842F900827FD
:200B800056E0FCA3E0FDA3E0FEA3E054C0FFEE54F7FEEC900827561200842F9008274FE0A1
:200BA000FBA3E0FAA3E0F9120081AEE5F09008275630E012E0FCA3E0FDA3E0FEA3E04480D0
:200BC000FFEE44168010E0FCA3E0FDA3E0FEA3E0547FFFEE54E9FEEC900827561200842F1D
:200BE00090082754E0FAA3E0FB64184A7012A3E0FCA3E0FDA3E0FEA3E0FFEE4420FE804E22
:200C00009008274EE0FF25E025E02474F582E43406F583759308E0B4013DEF25E025E0243A
:200C200073F582E43406F583759308E090082756B4050EE0FCA3E0FDA3E0FEA3E044408004
:200C40000CE0FCA3E0FDA3E0FEA3E054BFFFEC900827561200842FEBAE027803C333CE3343
:200C6000CED8F92401FFEE3401FEC006C00790082756E0FCA3E0FDA3E0FEA3E0FF90082ACD
:200C8000711200842FD007D00612022DA92278A27C247D097B817A9079E27E007F061200AF
:200CA000805578A87C247D097B817A9079E87E007F0C1200805590080660E0FBA3E0FAA3C9
:200CC000E0F9120081AEFFAEF0E5F0600321126BEF24FE7003210E14147003210E142402D0
:200CE000600321126B900823FF7483F0A374A8F0A37464F090081976E0FBA3E0FAA3E0F93D
:200D00001200959290081A69EEF0A3EFF090081976E0FBA3E0FAA3E0F990081A69E0FEA388
:200D2000E0FFE92FF9EA3EFA900823FF7483F0A374A9F0A37425F01200959290081A6AE0EF
:200D40002FF090081A69E03EF012023CE1900824961200842F9008249EE4F0A304F09008A6
:200D60001976E0FBA3E0FAA3E0F990081A69E0FEA3E0FFE92FF9EA3EFAC001900823FF7473
:200D800083F0A374A9F0A37469F09008249FE075F008A4FFC374209FF990082496E0FCA3B5
:200DA000E0FDA3E0FEA3E0FFA8011200837FE490082402F0A3EFF0D0011200959290081AC6
:200DC0006AE02FF090081A69E03EF09008249FE004F070079008249EE004F0D39008249F7F
:200DE000E094049008249EE0648094805003210D5E90081A6AE024FEF090081A69E034FF2E
:200E0000F090080660E0FBA3E0FAA3E0F9E475F00221126590081976E0FBA3E0FAA3E0F932
:200E200090081A69E0FEA3E0FFE92FF9EA3EFA900823FF7481F0A37490F0A374B0F0A37400
:200E400083F0A374A9F0A374A3F01200959290081A6AE02FF090081A69E03EF012023CF107
:200E6000900824961200842FE47F01FEFDFC9008249A1200842FE49008249EF0A3F090088C
:200E8000249AE0FCA3E0FDA3E0FEA3E0FF90082496E0F8A3E0F9A3E0FAA3E05FFFEA5EFEEB
:200EA000E95DFDE85CFCE4FBFAF9F8C31200836E70087B837AA979B180067B837AA979B28A
:200EC000900824B4EBF0A3EAF0A3E9F090081976E0FBA3E0FAA3E0F990081A69E0FEA3E057
:200EE000FFE92FF9EA3EFAC003C002C001900823FF7481F0A37490F0A374F4F0A37483F0BF
:200F0000A374A9F0A374BAF09008249EE0FEA3E0FF90082405EEF0A3EFF0900824B4E0F93C
:200F2000A3E0FAA3E090082407C9F0A3EAF0A3E9F0900824A275F003EF1200843BEE75F063
:200F400003A42583F583759308E0F9A3E0FAA3E09008240AC9F0A3EAF0A3E9F0D001D002C6
:200F6000D0031200959290081A6AE02FF090081A69E03EF09008249AE0FCA3E0FDA3E0FEEE
:200F8000A3E0FF7801120083929008249A1200842F9008249FE004F070079008249EE00430
:200FA000F0C39008249FE094029008249EE0648094805003210E7E74FF900824A0F0A3F029
:200FC000E49008249EF0A3F0C390082484E09401FF90082483E09400FEC39008249FE09F8B
:200FE000EE6480F89008249EE0648098505AA3E0FF12023BF4900824B7EEF0A3EFF06402C9
:201000004E601A900824B7E0FEA3E0FF64044E600CEF64034E6006EF64054E70199008241E
:20102000A0E4F0A304F0E47F01FEFDFC9008249A1200842F80129008249FE004F070079067
:2010400008249EE004F08080C3900824A0E064809480500321121AA3E0FF74017E00A80737
:20106000088005C333CE33CED8F9FFEE3395E0FDFC9008249A1200842F90081976E0FBA3FF
:20108000E0FAA3E0F990081A69E0FEA3E0FFE92FF9EA3EFA900823FF7481F0A37490F0A373
:2010A00074B0F0A37483F0A374A9F0A374BEF01200959290081A6AE02FF090081A69E03E90
:2010C000F012023D01900824961200842F900824A0E0FFA3E09008249ECFF0A3EFF0C3900B
:2010E00008249FE094029008249EE064809480400321121A9008249AE0FCA3E0FDA3E0FEBA
:20110000A3E0FF90082496E0F8A3E0F9A3E0FAA3E05FFFEA5EFEE95DFDE85CFCE4FBFAF9AE
:20112000F8C31200836E70087B837AA979B180067B837AA979B2900824B4EBF0A3EAF0A3F1
:20114000E9F090081976E0FBA3E0FAA3E0F990081A69E0FEA3E0FFE92FF9EA3EFAC003C08A
:2011600002C001900823FF7481F0A37490F0A374F4F0A37483F0A374A9F0A374D3F09008CF
:20118000249EE0FEA3E0FF90082405EEF0A3EFF0900824B4E0F9A3E0FAA3E090082407C937
:2011A000F0A3EAF0A3E9F0900824A875F003EF1200843BEE75F003A42583F583759308E0B0
:2011C000F9A3E0FAA3E09008240AC9F0A3EAF0A3E9F0D001D002D0031200959290081A6AD3
:2011E000E02FF090081A69E03EF09008249AE0FCA3E0FDA3E0FEA3E0FF78011200839290E2
:2012000008249A1200842F9008249FE004F070079008249EE004F02110DE90081976E0FB5E
:20122000A3E0FAA3E0F990081A69E0FEA3E0FFE92FF9EA3EFA900823FF7483F0A374A9F0B6
:20124000A374D7F01200959290081A6AE02FF090081A69E03EF090080660E0FBA3E0FAA33A
:20126000E0F9E4F5F01200822880037F01227F002290081736EBF0A3EAF0A3E9F0E4900815
:201280001849F0A3F0FE7F51FD7B097A17793D120088517E007F517D007B097A17798E12F0
:2012A0000088517E007F047D007B097A177939120088519008264B7481F0A3748BF0A3748E
:2012C0006BF0A37481F0A3748AF0A37458F0A37409F0A37417F0743D1201E0A69008264BBA
:2012E0007481F0A3748BF0A37470F0A37481F0A3748AF0A37458F0A37409F0A37417F074E6
:201300008E1201E0A69008264B7481F0A3748BF0A37475F0A37481F0A3748AF0A37458F032
:20132000A37409F0A37417F0A374391201E0A77B097A17793D1201DAFD7B097A17793D1203
:2013400000A3BED3EF9414EE648094804010900823FF7481F0A3748BF0A3747C802D7B0997
:201360007A17798E1201DAFD7B097A17798E1200A3BED3EF9414EE648094804031900823E0
:20138000FF7481F0A3748BF0A374B7F0A3E4F0A37414F07B097A1779DF1200959290082920
:2013A0006A7409F0A37417F0A374DF2116CD7B097A1779391202000790081843EEF0A3EFF9
:2013C000F0C39403EE64809480400FD3E0941E90081843E06480948040119008296A7481ED
:2013E000F0A3748BF0A374DD2116CDE490081857F0A3F090081857E0FEA3E0FFD39402EE47
:2014000064809480400321165DEE7060EF14602414603E24027055900818617481F0A3740E
:201420008BF0A374F9F0A37481F0A3748BF0A374FDF08038900818617481F0A3748CF0A32F
:201440007410F0A37481F0A3748CF0A37414F0801B900818617481F0A3748CF0A37428F08F
:20146000A37481F0A3748CF0A3742CF0E490081845F0A3F090081861E0F9A3E0FAA3E09048
:20148000082832C9F0A3EAF0A3E9F090081736E0FBA3E0FAA3E0F9120207F590081736EB9F
:2014A000F0A3EAF0A3E9F0C002C00190081861E0F9A3E0FAA3E09008264BC9F0A3EAF0A3F4
:2014C000E9F0A37481F0A3748AF0A37458F0A37409F0A37418F0A37467F0D001D002120168
:2014E000E0B4E490081847F0A3F07B097A1879671200A3BEC390081848E09FEE6480F890FD
:20150000081847E06480985041A3E02467F582E43418F583759308E0FF12023D50401990D1
:20152000081864E0F9A3E0FAA3E09008296AC9F0A3EAF0A3E92116CD90081848E004F07021
:20154000A990081847E004F080A07B097A18796712020007AC06AD0790081846E025E0FFA6
:2015600090081845E033FE74592FF58274183EF583759308ECF0A3EDF090081737E475F015
:20158000011200818290081846E004F0700790081845E004F0C390081846E094049008184A
:2015A00045E064809480500321147490081857E0FEA3E0FF64014E7045EF7802C333CE33E3
:2015C000CED8F9244BF974183EFA900827A77409F0A3EAF0A3E9F07B097A1879591201A7D2
:2015E0004BEF4E706590081864E0F9A3E0FAA3E09008296AC9F0A3EAF0A3E92116CD900818
:201600001857E0FEA3E07802C333CE33CED8F9244BF974183EFA9008281A7409F0A3EAF0FA
:20162000A3E9F07B097A1879591201CDC9EF4E701990081864E0F9A3E0FAA3E09008296ABF
:20164000C9F0A3EAF0A3E92116CD90081858E004F0700790081857E004F02113F3900818BF
:201660004FE0FCA3E0FDA3E0FEA3E0FFA3E0F8A3E0F9A3E0FAA3E05FFFEA5EFEE95DFDE8F6
:201680005CFCC004C005C006AB079008184FE0FCA3E0FDA3E0FEA3E0FF9008184BE0F8A31D
:2016A000E0F9A3E0FAA3E05FFFEA5EFEE95DFDE85CFCD002D001D000C31200836E602990D8
:2016C00008296A7481F0A3748CF0A3743FF0A37481F0A3748BF0A374AFF07B817A8B79A0C7
:2016E00012021578E4FEFF2212023CB19008184BE0F8A3E0F9A3E0FAA3E0FBC31200836E35
:20170000601E9008184BE0FCA3E0FDA3E0FEA3E0FF900824751200842F900819847410F052
:2017200012023CC19008184FE0F8A3E0F9A3E0FAA3E0FBC31200836E60179008184FE0FC32
:20174000A3E0FDA3E0FEA3E0FF900824871200842F12023CD190081853E0F8A3E0F9A3E003
:20176000FAA3E0FBC31200836E601790081853E0FCA3E0FDA3E0FEA3E0FF9008247B120009
:20178000842FE4FFFEFDFC90082475E0F8A3E0F9A3E0FAA3E0FBC31200836E7034FFFEFDD8
:2017A000FC90082487E0F8A3E0F9A3E0FAA3E0FBC31200836E701AFFFEFDFC9008247BE03E
:2017C000F8A3E0F9A3E0FAA3E0FBC31200836E600D90082471E4F0A304F01201F4B7E4FF2E
:2017E000FE12023E6C7B097A17793D12023D977B097A17798E12023DA190081843E0FEA3F8
:20180000E0FF12023E5E90082494E07002A3E07004120234B112023CA1C004A905AA06ABE9
:201820000790081843E0FEA3E0FF7C027D5812008138EE3395E0FDFCD000EB2FFFEA3EFE92
:20184000E93DFDE83CFC900804061200842F7E007F012290080660E0FBA3E0FAA3E0F912DA
:201860000081AEFFAEF0E5F06003211D91EF24FE7003211A1E147003211BD7147003211D59
:201880003F24036003211D91900828D57409F0A37429F0A37404F0A37409F0A37429F0A390
:2018A0007405F07B097A297903E4FF12022B2A900823FF7483F0A3748AF0A374F4F090080B
:2018C0001976E0FBA3E0FAA3E0F91200959290081A69EEF0A3EFF0E490082909F0A3F09030
:2018E000082909E0FEA3E0FFD39403EE6480948040032119CE90082905E0FD7C00EFB505EB
:201900000CECB506087B837A8C792A80067B837A8C793390082906EBF0A3EAF0A3E9F09004
:20192000081976E0FBA3E0FAA3E0F990081A69E0FEA3E0FFE92FF9EA3EFAC003C002C00148
:20194000900823FF7483F0A3748CF0A37434F090082909E0FEA3E0FF90082402EEF0A3EFC0
:20196000F090082906E0F9A3E0FAA3E090082404C9F0A3EAF0A3E9F0900827FF75F003EF50
:201980001200843BEE75F003A42583F583759308E0F9A3E0FAA3E090082407C9F0A3EAF07A
:2019A000A3E9F0D001D002D0031200959290081A6AE02FF090081A69E03EF09008290AE00D
:2019C00004F0700790082909E004F02118DF90081976E0FBA3E0FAA3E0F990081A69E0FEF2
:2019E000A3E0FFE92FF9EA3EFA900823FF7483F0A3748CF0A3744FF01200959290081A6A53
:201A0000E02FF090081A69E03EF090080660E0FBA3E0FAA3E0F9E475F0021200822890082D
:201A200028D57409F0A37429F0A37404F0A37409F0A37429F0A37405F07B097A297903E42E
:201A4000FF12022B2A9008066BE0FBA3E0FAA3E0F9120081AEFFAEF09008290BEEF0A3EF27
:201A6000F0C390082484E09401FD90082483E09400FCD3EF9DEC6480F8EE6480984003215D
:201A80001B7490082905E0700EA37483F0A3748CF0A37433F08039C39008290CE09401FF7F
:201AA0009008290BE09400FE90082903E07C00B5070CECB506087B837A8C792A80067B8326
:201AC0007A8C793390082906EBF0A3EAF0A3E9F090081976E0FBA3E0FAA3E0F990081A69A3
:201AE000E0FEA3E0FFE92FF9EA3EFAC002C001900823FF7483F0A3748CF0A374B1F090084C
:201B0000290BE0FCA3E0FDC39401FEEC940090082402F0A3CEF090082906E0F9A3E0FAA390
:201B2000E090082404C9F0A3EAF0A3E9F0A3ECF0A3EDF0D001D0021200959290081A6AE07C
:201B40002FF090081A69E03EF09008066BE0FBA3E0FAA3E0F9E475F001120081FCC390082C
:201B60001A6AE094B090081A69E094045003211A457F002290081976E0FBA3E0FAA3E0F9BB
:201B800090081A69E0FEA3E0FFE92FF9EA3EFA900823FF7483F0A3748CF0A374CEF012007C
:201BA000959290081A6AE02FF090081A69E03EF090080660E0FBA3E0FAA3E0F9E475F0039C
:201BC000120082289008066BE0FBA3E0FAA3E0F9E475F001211D8A900828D57409F0A37441
:201BE00029F0A37404F0A37409F0A37429F0A37405F07B097A297903E4FF12022B2A9008EE
:201C0000066BE0FBA3E0FAA3E0F9120081AEFFAEF09008290BEEF0A3EFF0C390082484E092
:201C20009401FD90082483E09400FCD3EF9DEC6480F8EE6480984003211D2D90082905E07E
:201C4000700EA37483F0A3748CF0A37433F08039C39008290CE09401FF9008290BE09400B2
:201C6000FE90082904E07C00B5070CECB506087B837A8C792A80067B837A8C793390082930
:201C800006EBF0A3EAF0A3E9F090081976E0FBA3E0FAA3E0F990081A69E0FEA3E0FFE92FDC
:201CA000F9EA3EFAC002C001900823FF7483F0A3748CF0A374B1F09008290BE0FCA3E0FD72
:201CC000C39401FEEC940090082402F0A3CEF090082906E0F9A3E0FAA3E090082404C9F006
:201CE000A3EAF0A3E9F0A3ECF0A3EDF0D001D0021200959290081A6AE02FF090081A69E0FA
:201D00003EF09008066BE0FBA3E0FAA3E0F9E475F001120081FCC390081A6AE094B0900844
:201D20001A69E094045003211BFE7F002290080660E0FBA3E0FAA3E0F9E475F004804B9000
:201D4000081976E0FBA3E0FAA3E0F990081A69E0FEA3E0FFE92FF9EA3EFA900823FF7483B9
:201D6000F0A3748DF0A3742EF01200959290081A6AE02FF090081A69E03EF090080660E04F
:201D8000FBA3E0FAA3E0F9E4F5F0120082287F00227F0122900825491200842F9008254DB2
:201DA000EBF0A3EAF0A3E9F012023CD19008255B1200842F12023CC19008255F1200842F5F
:201DC0009008255FE0FCA3E0FDA3E0FEA3E0FF9008255BE0F8A3E0F9A3E0FAA3E05FFFEAD4
:201DE0005EFEE95DFDE85CFCC004C005C006AB07A3E0FCA3E0FDA3E0FEA3E0FF90082549FB
:201E0000E0F8A3E0F9A3E0FAA3E05FFFEA5EFEE95DFDE85CFCD002D001D000C31200836E0E
:201E200060179008255BE0FCA3E0FDA3E0FEA3E0FF900825491200842FE490082557F0A35E
:201E4000F090082557E0FEA3E0FFC39408EE648094804003211F1390081F6D75F00AEF12AF
:201E600000843BEE75F00AA42583F583759308E0FCA3E0FDA3E0FEA3E0FF90082549E0F835
:201E8000A3E0F9A3E0FAA3E0FBC31200836E707090082557E0FEA3E090081F6D75F00A120B
:201EA00000843BEE75F00AA42583F583759308E0FCA3E0FDA3E0FEA3E0FFE4FBFAF9F8C346
:201EC0001200836E603A90082557E0FEA3E0FF7C007D0A1200813874712FF9741F3EFA7BD0
:201EE00009C003C0029008254DE0FBA3E0FAA3E0F8AC02AD03D002D0037E007F0621225DD1
:201F000090082558E004F0700790082557E004F0211E4190081A69E0FEA3E0FF78007C0783
:201F20007D099008248FE0FBA3E0FAA3E0F91200805590081A69E0FFA3E090082559CFF0C3
:201F4000A3EFF090081FBFE4F0A3743CF090082557E4F0A304F09008197FE0FBA3E0FAA3C8
:201F6000E0F990082554EBF0A3EAF0A3E9F0E475F0011200822890082554E0FBA3E0FAA391
:201F8000E02402F9E43AFA740875F0001200822890082554E0FBA3E0FAA3E02404F9E43A62
:201FA000FA740675F0041200822890082554E0FBA3E0FAA3E02406F9E43AFAE475F0011205
:201FC00000822890082554E0FBA3E0FAA3E02408F9E43AFA1202384712023CB19008255489
:201FE000E0FBA3E0FAA3E0240EF9E43AFA120083C27E007F067D0090082554E0FBA3E0FA83
:20200000A3E02412F9E43AFA1200885190082549E0FCA3E0FDA3E0FEA3E0FF90082554E0B5
:20202000FBA3E0FAA3E02418F9E43AFA120083C290081973E0FBA3E0FAA3E0240CF9E43ABB
:20204000FA740875F006120082287E007F067DFF90081973E0FBA3E0FAA3E0F91200885181
:2020600090082554E0FBA3E0FAA3E02408F9E43AFAC003C002C00190081973E0FBA3E0FA75
:20208000A3E02406F9E43AA801FCAD03D001D002D0037E007F06120080559008248FE0FBA1
:2020A000A3E0FAA3E0F97D2A7C001201ADA112020B2B90082558E004F0700790082557E005
:2020C00004F0D390082558E0940390082557E0648094805003211F5612023CA1EF240AFFCB
:2020E000E43EFEE43DFDE43CFC900825501200842F12023CA190082550E0F8A3E0F9A3E0DF
:20210000FAA3E0FBD31200836E50032122657B097A1A79691201C7619008248FEBF0A3EA8E
:20212000F0A3E9F09008248FE0FBA3E0FAA3E04A4B60BE9008248FE0FBA3E0FAA3E0F990AB
:20214000081973EBF0A3EAF0A3E9F0240CF9E43AFA120081AE64067004E5F06408600321F2
:2021600021E390081973E0FBA3E0FAA3E0240EF9E43AFA90082554EBF0A3EAF0A3E9F01222
:20218000023CB190082554E0FBA3E0FAA3E02418F9E43AFA120083DDC31200836E7044909B
:2021A000082554E0FBA3E0FAA3E02406F9E43AFA120081AE640245F0702990082554A3E07F
:2021C000FAA3E0240EF9E43AFA120083A590082549E0F8A3E0F9A3E0FAA3E0FBC312008358
:2021E0006E6007120080232120F190082549E0FCA3E0FDA3E0FEA3E0FF90081973E0FBA31C
:20220000E0FAA3E02406F9E43AFA1201BEE090082559E0FFA3E090081A69CFF0A3EFF09011
:20222000081973E0FBA3E0FAA3E02406F9E43AFA78007C077D097E007F06120080559008F1
:202240001A69E0FEA3E0FF9008248FE0FBA3E0FAA3E0F8AC02AD037B097A0779001200800F
:2022600055E4FEFF227EFF7FFF229008223BEEF0A3EFF0A3E4F0A304F09008066BE0FBA3FF
:20228000E0FAA3E0F9120081AEC39401FFE5F09400FE90082241F0A3EFF0C39008247AE0A3
:2022A0009401FD90082479E09400FCEDB50709ECB506057E007F012290082242E0FF12027A
:2022C0003BF490082243EEF0A3EFF090082241E07002A3E0601A90082242E0C39401FF12E3
:2022E000023BF490082243E06E7003A3E06F602990082245E4F0A3740AF0E02402F0900802
:202300002245E03400F090082243E0FEA3E0FFA3E0FCA3E0FD12021F3A90081976E0FBA3E4
:20232000E0FAA3E0F990081A69E0FEA3E0FFE92FF9EA3EFA900823FF7483F0A37461F0A3ED
:2023400074D5F01200959290081A6AE02FF090081A69E03EF09008223FE4F0A304F09008CB
:20236000223FE0FEA3E0FFD39402EE940040032126FDEF64024E600321242F90082242E0D4
:2023800004F0700790082241E004F090082242E0FF12023BF490082243EEF0A3EFF0C39035
:2023A00008247AE09401FF90082479E09400FE90082241E06E7003A3E06F601A9008224238
:2023C000E0C39401FF12023BF490082243E06E7003A3E06F605990081976E0FBA3E0FAA3F8
:2023E000E0F990081A69E0FEA3E0FFE92FF9EA3EFA900823FF7483F0A37461F0A374DCF06A
:2024000090082245E0FEA3E0FF7C007D021200814A90082402EEF0A3EFF012009592900896
:202420001A6AE02FF090081A69E03EF021272190082242E0FF7B097A2279471201F03B90FE
:20244000082243E07004A3E06404703190082242E0FF120236D9EF4E70119008226B748357
:20246000F0A37461F0A374F4F0804390082247E0C4F854F0C8A3E0C4540F4880059008226C
:2024800048E0540F9008236975F0031200843BE475F003A42583F583759308E0F9A3E0FADE
:2024A000A3E09008226BC9F0A3EAF0A3E9F09008223BE07004A3E06401900819767043E0D7
:2024C000FBA3E0FAA3E0F990081A69E0FEA3E0FFE92FF9EA3EFA900823FF7483F0A3746240
:2024E000F0A37400F090082241E0FEA3E0FF90082402EEF0A3EFF02401FFE43EA3F0A3EF01
:20250000803CE0FBA3E0FAA3E0F990081A69E0FEA3E0FFE92FF9EA3EFA900823FF7483F0DC
:20252000A37462F0A37434F090082242E02401FE90082241E0340090082402F0A3CEF012C8
:2025400000959290081A6AE02FF090081A69E03EF090081976E0FBA3E0FAA3E0F990081A63
:2025600069E0FEA3E0FFE92FF9EA3EFAC003C002C001900823FF7483F0A37462F0A3744FA9
:20258000F09008226BE0F9A3E0FAA3E090082402C9F0A3EAF0A3E9F090082247E0FCA3E07D
:2025A000FDECC4F854F0C8EDC4540F48540F9008236975F0031200843BE475F003A42583B6
:2025C000F583759308E0F9A3E0FAA3E090082405C9F0A3EAF0A3E9F0EC54019008235D7559
:2025E000F0031200843BE475F003A42583F583759308E0F9A3E0FAA3E090082408C9F0A3FE
:20260000EAF0A3E9F090082247E0C31354019008236375F0031200843BE475F003A4258369
:20262000F583759308E0F9A3E0FAA3E09008240BC9F0A3EAF0A3E9F0D001D002D003120038
:20264000959290081A6AE02FF090081A69E03EF07B097A22794B120237C990081976E0FB15
:20266000A3E0FAA3E0F990081A69E0FEA3E0FFE92FF9EA3EFAC002C001900823FF7483F08F
:20268000A37462F0A37470F090082241E0FEA3E0244BF58274223EF583759308E075F00374
:2026A000A42457F582E43423F583759308E0F9A3E0FAA3E090082402C9F0A3EAF0A3E9F078
:2026C000D001D0021200959290081A6AE02FF090081A69E03EF09008066BE0FBA3E0FAA3D6
:2026E000E0F9E475F001120081FC90082240E004F070079008223FE004F021235E900822BA
:202700003EE004F070079008223DE004F0D39008223EE094049008223DE094005003212221
:2027200079E4FEFF229008261DEEF0A3EFF064014E701B74FFFFFEFDFC90081A66E0FBA3A5
:20274000E0FAA3E02404F9E43AFA120083C290081A66E0FBA3E0FAA3E02414F9E43AFA123E
:202760000080D314700321293824FB700321282224F5600321283C90081A66E0FBA3E0FA8F
:20278000A3E0F9120081AEFF9008197CE0FBA3E0FAA3E0F9E5F08FF01200822890081A6654
:2027A000E0FBA3E0FAA3E02402F9E43AFA120081AEFF9008197CE0FBA3E0FAA3E02402F9A0
:2027C000E43AFAE5F08FF01200822890081A6AE02408F090081A69E03400F0E0FEA3E0FF3A
:2027E0009008197CE0FBA3E0FAA3E02404F9E43AFAEE8FF0120082289008197CE0FBA3E0E4
:20280000FAA3E02406F9E43AFAE4F5F01200822890081A6AE02414F090081A69E03400F038
:20282000801D90081979E0FBA3E0FAA3E02410F9E43AFAE4F5F0120082288003212B73C327
:2028400090081A6AE09414FE90081A69E094009008262DF0A3CEF012023CB19008261F121B
:2028600000842F90081A66E0FBA3E0FAA3E02404F9E43AFA120083A5900826231200842F99
:20288000E490082627F090081A66E0FBA3E0FAA3E02414F9E43AFA120080D390082628F008
:2028A0009008262DE0FCA3E0FD90082629ECF0A3EDF09008197FE0FBA3E0FAA3E02414F952
:2028C000E43AFA1201D3E69008262BEEF0A3EFF07B097A26791F7D0E7C001201D3E6EFF459
:2028E000FFEEF49008262BF0A3EFF090081A66E0FBA3E0FAA3E02414F9E43AFA120080D3FB
:202900009008262BB41114E0FEA3E0FF9008197CE0FBA3E0FAA3E024068012E0FEA3E0FF71
:2029200090081979E0FBA3E0FAA3E02410F9E43AFAEE8FF01200822812023CB19008197FF3
:20294000E0FBA3E0FAA3E0240CF9E43AFA120083C290081A66E0FBA3E0FAA3E02404F9E40C
:202960003AFA120083A59008197FE0FBA3E0FAA3E02410F9E43AFA120083C290081A66E04A
:20298000FBA3E0FAA3E02414F9E43AFA120080D3FF9008197FE0FBA3E0FAA3E02409F9E47A
:2029A0003AFAEF120081249008197FE0FBA3E0FAA3E0F97445120081249008197FE0FBA31B
:2029C000E0FAA3E02401F9E43AFAE4120081249008197FE0FBA3E0FAA3E02406F9E43AFA83
:2029E000744075F000120082289008197FE0FBA3E0FAA3E02408F9E43AFA74FF1200812490
:202A000090081A69E0FEA3E0FF9008197FE0FBA3E0FAA3E02402F9E43AFAEE8FF0120082F8
:202A20002890081983E004F0700790081982E004F090081982E0FEA3E0FF9008197FE0FB4A
:202A4000A3E0FAA3E02404F9E43AFAEE8FF0120082289008197FE0FBA3E0FAA3E0240AF9E2
:202A6000E43AFAE4F5F0120082281201D3D6EFF4FFEEF4FE9008197FE0FBA3E0FAA3E0240C
:202A80000AF9E43AFAEE8FF01200822890081A6AE0240EF090081A69E03400F09008197391
:202AA000E0FBA3E0FAA3E0240CF9E43AFA740875F0001200822890081973E0FBA3E0FAA33E
:202AC000E02406F9E43AFA120238479008261DE07004A3E06401703090081973E0FBA3E00F
:202AE000FAA3E0F8AC02AD037B097A1979857E007F06120080559008248FE0FBA3E0FAA3BE
:202B0000E0F91202262A80709008261DE07004A3E064047033782D7C267D097B817A90797F
:202B200000FE7F061200805590081973E0FBA3E0FAA3E0F8AC02AD037B097A26792D7E008E
:202B40007F0612008055803090081A66E0FBA3E0FAA3E02404F9E43AFA120083A590081942
:202B600073E0FBA3E0FAA3E0F912011D94BEFF08BFFF057EFF7FFF221201F4B79008248F9C
:202B8000E0FBA3E0FAA3E0F990081A69E0FCA3E0FD1201ADA1E4FEFF22900827BFEBF0A38A
:202BA000EAF0A3E9F0EF25E024F3F582E43406F583759308E0900827C6F0EF25E024F4F541
:202BC00082E43406F583759308E0900827C7F07E007F047D007B097A2779C212008851901E
:202BE0000827BFE0FBA3E0FAA3E0F8AC02AD037B097A2779C27E007F04120087C7EF6003A3
:202C0000212D40900827C7E014605A147003212CAF147003212CF624036003212FDEE4FF0A
:202C2000FEFDFC900827C81200842F900827C8E0FCA3E0FDA3E0FEA3E0FF90082A71120026
:202C4000842F7F1F7E0012022DA97B097A2779C87F217E00120232F5900827C8A3A3A3E0AC
:202C6000FFE4FE8045E4FFFEFDFC900827C81200842F900827C8E0FCA3E0FDA3E0FEA3E0A1
:202C8000FF90082A711200842F7F207E0012022DA97B097A2779C87F217E00120232F590E7
:202CA0000827C8A3A3E0FEE4FFE4FDFC212E68E4FFFEFDFC900827C81200842F900827C8D5
:202CC000E0FCA3E0FDA3E0FEA3E0FF90082A711200842F7F227E0012022DA97B097A2779F6
:202CE000C87F247E00120232F5900827C8A3A3A3E0FFE4FE8045E4FFFEFDFC900827C81247
:202D000000842F900827C8E0FCA3E0FDA3E0FEA3E0FF90082A711200842F7F237E001202EE
:202D20002DA97B097A2779C87F247E00120232F5900827C8A3A3E0FEE4FFE4FDFC212F1030
:202D4000900827C7E0147003212DE5147003212E8C147003212F3424036003212FDE900896
:202D600027BFE0FBA3E0FAA3E02401F9E43AFA120080D3FE900827BFA3E0FAA3E0F9120070
:202D800080D3FDEDFFE4FCFD900827C81200842F900827C8E0FCA3E0FDA3E0FEA3E0FF9058
:202DA000082A711200842F7F1F7E0012022DA97B097A2779C87F217E00120232F590082727
:202DC000BFE0FBA3E0FAA3E02402F9E43AFA120080D3FA900827C8A3A3A3E0FFE4FDFCEAAD
:202DE000FEE4212E68900827BFE0FBA3E0FAA3E02401F9E43AFA120080D3FE900827BFA327
:202E0000E0FAA3E0F9120080D3FDEDFFE4FCFD900827C81200842F900827C8E0FCA3E0FD02
:202E2000A3E0FEA3E0FF90082A711200842F7F207E0012022DA97B097A2779C87F217E000C
:202E4000120232F5900827BFE0FBA3E0FAA3E02402F9E43AFA120080D3FB900827C8A3A37A
:202E6000E0FEE4FDFCEBFFE4900827C81200842F900827C8E0FCA3E0FDA3E0FEA3E0FF9007
:202E8000082A711200842F7F21212FD8900827BFE0FBA3E0FAA3E02401F9E43AFA120080E1
:202EA000D3FE900827BFA3E0FAA3E0F9120080D3FDEDFFE4FCFD900827C81200842F9008BB
:202EC00027C8E0FCA3E0FDA3E0FEA3E0FF90082A711200842F7F227E0012022DA97B097AA5
:202EE0002779C87F247E00120232F5900827BFE0FBA3E0FAA3E02402F9E43AFA120080D319
:202F0000FA900827C8A3A3A3E0FFE4FDFCEAFEE4900827C81200842F900827C8E0FCA3E08D
:202F2000FDA3E0FEA3E0FF90082A711200842F7F24212FD8900827BFE0FBA3E0FAA3E02451
:202F400001F9E43AFA120080D3FE900827BFA3E0FAA3E0F9120080D3FDEDFFE4FCFD9008C2
:202F600027C81200842F900827C8E0FCA3E0FDA3E0FEA3E0FF90082A711200842F7F237E9F
:202F80000012022DA97B097A2779C87F247E00120232F5900827BFE0FBA3E0FAA3E0240206
:202FA000F9E43AFA120080D3FB900827C8A3A3E0FEE4FDFCEBFFE4900827C81200842F906E
:202FC0000827C8E0FCA3E0FDA3E0FEA3E0FF90082A711200842F7F247E0012022DA92290E6
:202FE00008232CEEF0A3EFF09008066BE0FBA3E0FAA3E0F9120081AE45F060032130BA90C9
:20300000081976E0FBA3E0FAA3E0F990081A69E0FEA3E0FFE92FF9EA3EFA900823FF7483E6
:20302000F0A374AFF0A3745CF01200959290081A6AE02FF090081A69E03EF09008234EE41D
:20304000F0A304F090081976E0FBA3E0FAA3E0F990081A69E0FEA3E0FFE92FF9EA3EFA90B0
:203060000823FF7483F0A374AFF0A3748AF01200959290081A6AE02FF090081A69E03EF07B
:203080009008234FE004F070079008234EE004F0D39008234FE094049008234EE064809448
:2030A0008040A19008066BE0FBA3E0FAA3E0F9E475F0011200822821340C7B097A23792EA3
:2030C000120237C99008066BE0FBA3E0FAA3E0F9120081AEC39401FFE5F09400FE90082345
:2030E00050F0A3EFF0C39008247AE09401FD90082479E09400FCEDB50709ECB506057E0022
:203100007F012290082351E0FF12023BF490082352EEF0A3EFF090082350E07002A3E06032
:203120001A90082351E0C39401FF12023BF490082352E06E7003A3E06F601190082352E0D1
:20314000FEA3E0FF7D087C0012021F3A90081976E0FBA3E0FAA3E0F990081A69E0FEA3E00A
:20316000FFE92FF9EA3EFA900823FF7483F0A374AFF0A374B4F01200959290081A6AE02FA7
:20318000F090081A69E03EF0E49008234EF0A3F09008234EE0FEA3E0FFD39403EE6480946D
:2031A00080400321340CEF9400EE64809480500321324D90082351E004F07007900823502D
:2031C000E004F090082351E0FF12023BF490082352EEF0A3EFF0C39008247AE09401FF9083
:2031E000082479E09400FE90082350E06E7003A3E06F601A90082351E0C39401FF12023BEE
:20320000F490082352E06E7003A3E06F603F90081976E0FBA3E0FAA3E0F990081A69E0FE67
:20322000A3E0FFE92FF9EA3EFA900823FF7483F0A374AFF0A374C8F01200959290081A6A5E
:20324000E02FF090081A69E03EF021340C90082351E0242EF582E43423F583759308E0B4D9
:2032600001087B837AAF79DF80067B837AAF79E890082354EBF0A3EAF0A3E9F090081976AE
:20328000E0FBA3E0FAA3E0F990081A69E0FEA3E0FFE92FF9EA3EFA900823FF7483F0A374F4
:2032A000AFF0A374E9F090082351E02401FE90082350E0340090082402F0A3CEF01200959B
:2032C0009290081A6AE02FF090081A69E03EF09008232CE07004A3E064019008197660036B
:2032E00021336DE0FBA3E0FAA3E0F990081A69E0FEA3E0FFE92FF9EA3EFAC003C002C00145
:20330000900823FF7483F0A374AFF0A374FAF090082350E0FFA3E090082402CFF0A3EFF0E9
:2033200090082A8DE0F9A3E0FAA3E090082404C9F0A3EAF0A3E9F090082354E0F9A3E0FA8E
:20334000A3E090082407C9F0A3EAF0A3E9F090082A90E0F9A3E0FAA3E09008240AC9F0A328
:20336000EAF0A3E9F0D001D002D0038066E0FBA3E0FAA3E0F990081A69E0FEA3E0FFE92F34
:20338000F9EA3EFAC002C001900823FF7483F0A374B0F0A3744BF090082350E0FEA3E02455
:2033A0002EF58274233EF583759308E075F003A4248DF582E4342AF583759308E0F9A3E0D1
:2033C000FAA3E090082402C9F0A3EAF0A3E9F0D001D0021200959290081A6AE02FF0900871
:2033E0001A69E03EF09008066BE0FBA3E0FAA3E0F9E475F001120081FC9008234FE004F0A8
:2034000070079008234EE004F0213190E4FEFF229008197CE0FBA3E0FAA3E02408F9E43A28
:20342000FA90082893EBF0A3EAF0A3E9F0900829F17481F0A374A2F0A37402F0A3E4F0A308
:203440007410F0120221CFEF706F900827F67409F0A37428F0A37498F0A37409F0A37428E7
:20346000F0A3749AF0A37409F0A37428F0A3749CF07B097A28799612022B8B90082898E0A2
:203480007002A3E060032137C09008289AE07002A3E060032137C0D39008289DE0941E90C0
:2034A00008289CE06480948040032137C090082B54E4F0A304F02137F5900829F17481F0A7
:2034C000A374A2F0A3740BF0A3E4F0A37410F090082893E0FBA3E0FAA3E0F9120221CFEF89
:2034E00070032137F5900829F17481F0A374A2F0A37413F0A3E4F0A37409F090082893E0F8
:20350000FBA3E0FAA3E0F9120221CFEF705090082B54E07004A3E0640160032137C090089E
:203520002893E0FBA3E0FAA3E0240AF9E43AFA7D087C001201D3E6EFF47002EEF46003212E
:2035400037C090082893E0FBA3E0FAA3E0240AF9E43AFA12023C6E120234EC2137F5900830
:2035600029F17481F0A374A2F0A3741DF0A3E4F0A37409F090082893E0FBA3E0FAA3E0F9D1
:20358000120221CFEF701790082B54E07004A3E0640160032137C012023A042137F59008AC
:2035A00029F17481F0A374A2F0A37427F0A3E4F0A37407F090082893E0FBA3E0FAA3E0F989
:2035C000120221CFEF700A90082B54F0A3F02137F5900829F17481F0A374A2F0A3742FF021
:2035E000A3E4F0A37408F090082893E0FBA3E0FAA3E0F9120221CFEF705A900823FF7481B2
:20360000F0A374A2F0A37438F0A37481F0A374A2F0A3743BF090082893E0FBA3E0FAA3E031
:20362000F91200959290081A69EEF0A3EFF090082893E0FBA3E0FAA3E02FF9EA3EFA120251
:20364000384790081A6AE02406F090081A69E03400213828900829F17481F0A374A2F0A342
:20366000743FF0A3E4F0A3740AF090082893E0FBA3E0FAA3E0F9120221CFEF707390082367
:20368000FF7481F0A374A2F0A37438F0A37481F0A374A2F0A3744AF090082893E0FBA3E02B
:2036A000FAA3E0F91200959290081A69EEF0A3EFF090082893E0FBA3E0FAA3E02FF9EA3E62
:2036C000FA900823FF7481F0A374A2F0A37438F0A37481F0A374A2F0A37451F012009592A7
:2036E00090081A6AE02FF090081A69E03E213828900829F17481F0A374A2F0A3745BF0A3B0
:20370000E4F0A3740AF090082893E0FBA3E0FAA3E0F9120221CFEF7073900823FF7481F028
:20372000A374A2F0A37438F0A37481F0A374A2F0A37466F090082893E0FBA3E0FAA3E0F9DC
:203740001200959290081A69EEF0A3EFF090082893E0FBA3E0FAA3E02FF9EA3EFA90082382
:20376000FF7481F0A374A2F0A37438F0A37481F0A374A2F0A3746DF01200959290081A6A83
:20378000E02FF090081A69E03E213828900829F17481F0A374A2F0A3747AF0A3E4F0A37421
:2037A00005F090082893E0FBA3E0FAA3E0F9120221CFEF700B90082B56E07002A3E07035EC
:2037C000900823FF7481F0A374A2F0A37438F0A37481F0A374A2F0A37480F090082893E077
:2037E000FBA3E0FAA3E0F91200959290081A69EEF0A3EF8033900823FF7481F0A374A2F016
:20380000A37438F0A37481F0A374A2F0A37485F090082893E0FBA3E0FAA3E0F9120095924C
:2038200090081A69EEF0A3EFF07F027E001201272522E4900826BFF0A3F0900815DAE0FE44
:20384000A3E0FFC3900826C0E09F900826BFE09E4003213C457B097A19798F90081A66EB24
:20386000F0A3EAF0A3E9F02414F9E43AFA74111200812412023CE190081A66E0FBA3E0FA39
:20388000A3E02404F9E43AFA120083C290081A66E0FBA3E0FAA3E0F974FC75F003120082BD
:2038A0002890081A66E0FBA3E0FAA3E02402F9E43AFA74FC75F0021200822812020B2B12C7
:2038C000023DF0EF4E700E12023DDDAC06AD077F01120235269008197CE0FBA3E0FAA3E073
:2038E0002408F9E43AFA900826B9EBF0A3EAF0A3E9F02428F9E43AFAA3EBF0A3EAF0A3E95C
:20390000F012023CB1900826BCE0FBA3E0FAA3E0F9120083C2900826BDE475F004120081B6
:2039200082900826BCE0FBA3E0FAA3E0F8AC02AD037B817AA079D61200869312023D789071
:203940000826BDEE8FF012008182900826BCE0FBA3E475F00112008198A9F0FA7420120054
:203960008124900826BFE475F00112008198FEE5F025E0FFEE33FE74D22FF58274133EF514
:2039800083759308E0FFA3E0900826C1CFF0A3EFF0900823FF7481F0A374A1F0A37427F0FD
:2039A000900826C1E0FFA3E090082402CFF0A3EFF0900826BCE0FBA3E0FAA3E0F912009532
:2039C00092900826C3EEF0A3EFF0900826BDEE8FF012008182900826C1E0FEA3E0FFC39441
:2039E000D0EE648094874003213B31EF64EA7003EE64036003213AEC900826C0E025E0FF29
:203A0000900826BFE033FE74D22FF58274133EF583759308E0FCA3E0FDA3E0FEA3E0FF90F0
:203A20000826C71200842F900826C0E02402F0900826BFE03400F0C3900826C2E094E8FF39
:203A4000900826C1E09403CFC39401CF9400FE900814BA75F003EF1200843BEE75F003A460
:203A60002583F583759308E0F9A3E0FAA3E0900823FFC9F0A3EAF0A3E9F0900826C7E0FC70
:203A8000A3E0FDA3E0FEA3E0FF78181200837FE490082402F0A3EFF0900826C7E0FCA3E007
:203AA000FDA3E0FEA3E0FF78101200837FE490082404F0A3EFF0900826C7E0FCA3E0FDA3D0
:203AC000E0FEA3E0FF78081200837FE490082406F0A3EFF0900826C7E0FCA3E0FDA3A3E0D3
:203AE000FEE490082408F0A3CE213BCBC3900826C2E094E8FF900826C1E09403CFC39401DD
:203B0000CF9400FE900814BA75F003EF1200843BEE75F003A42583F583759308E0F9A3E030
:203B2000FAA3E0900823FFC9F0A3EAF0A3E9213BCB900826C1E0FEA3E0FFC394B8EE6480A5
:203B4000948B5016C3EF94D0FFEE9407CFC39401CF9400FE900815C2801CC3900826C2E08C
:203B600094B8FF900826C1E0940BCFC39401CF9400FE900815D475F003EF1200843BEE7568
:203B8000F003A42583F583759308E0F9A3E0FAA3E0900823FFC9F0A3EAF0A3E9F09008265B
:203BA000BFE475F00112008198FEE5F025E0FFEE33FE74D22FF58274133EF583759308E0C2
:203BC000FFA3E090082402CFF0A3EFF0900826BCE0FBA3E0FAA3E0F912009592900826C35C
:203BE000EEF0A3EFF0900826C3E0FEA3E0FF900826BDEE8FF012008182900826B9A3E0FA93
:203C0000A3E0AE02FFA3A3E0FAA3E0C39FFFEA9E90081A69F0A3EFF0900826B9E0FBA3E084
:203C2000FAA3E0F91202161A7F027E0012012725900826C5EEF0A3EFF0F47002EEF46003DE
:203C400021383A8000900826C5E0FEA3E0FF2290080660E0FBA3E0FAA3E0F9120081AEFF3A
:203C6000AEF0E5F06003214061EF24FE7003213D25147003214010240260032140619008CA
:203C800023FF7483F0A3749DF0A37425F090081976E0FBA3E0FAA3E0F91200959290081A65
:203CA00069EEF0A3EFF090082595E4F0A304F090081976E0FBA3E0FAA3E0F990081A69E088
:203CC000FEA3E0FFE92FF9EA3EFA900823FF7483F0A3749FF0A37411F01200959290081AE7
:203CE0006AE02FF090081A69E03EF090082596E004F0700790082595E004F0D39008259648
:203D0000E0940290082595E06480948040A190080660E0FBA3E0FAA3E0F9E475F0021200F3
:203D200082287F002290082595E4F0A304F09008066BE0FBA3E0FAA3E0F9120081AEC39406
:203D400001FFE5F09400FE90082599F0A3EFF0C39008247AE09401FD90082479E09400FC24
:203D6000EDB5071BECB5061790080660E0FBA3E0FAA3E0F9E475F0031200822821401090E6
:203D800008259AE0FF12023BF49008259BEEF0A3EFF090082599E07002A3E0601A90082520
:203DA0009AE0C39401FF12023BF49008259BE06E7003A3E06F60119008259BE0FEA3E0FFBB
:203DC0007D0A7C0012021F3A90081976E0FBA3E0FAA3E0F990081A69E0FEA3E0FFE92FF9EC
:203DE000EA3EFA900823FF7483F0A3749FF0A37488F01200959290081A6AE02FF090081AC5
:203E000069E03EF090082597E4F0A304F090082597E0FEA3E0FFD39402EE64809480400326
:203E2000213FE7EF64024E6003213EC69008259AE004F0700790082599E004F09008259AED
:203E4000E0FF12023BF49008259BEEF0A3EFF0C39008247AE09401FF90082479E09400FE74
:203E600090082599E06E7003A3E06F601A9008259AE0C39401FF12023BF49008259BE06E48
:203E80007003A3E06F603F90081976E0FBA3E0FAA3E0F990081A69E0FEA3E0FFE92FF9EAAD
:203EA0003EFA900823FF7483F0A3749FF0A3748FF01200959290081A6AE02FF090081A697E
:203EC000E03EF07F002290082599E0FEA3E0FF90081C807409F0A37425F0A374A1F0A374F1
:203EE00009F0A37425F0A374A5F0A37409F0A37425F0A374A9F07B097A25799D1201A2F126
:203F000090081976E0FBA3E0FAA3E0F990081A69E0FEA3E0FFE92FF9EA3EFAC003C002C0B3
:203F200001900823FF7483F0A3749FF0A374A6F090082599E0FEA3E0FF90082402EEF0A397
:203F4000EFF02401FFE43EA3F0A3EFF0900825A1E0FCA3E0FDA3E0FEA3E0FF900824061296
:203F600000842F900825A9E0FCA3E0FDA3E0FEA3E0FF9008240A1200842F9008259DE0FC08
:203F8000A3E0FDA3E0FEA3E0FF9008240E1200842F900825A5E0FCA3E0FDA3E0FEA3E0FF4E
:203FA000900824121200842FD001D002D0031200959290081A6AE02FF090081A69E03EF07B
:203FC0009008066BE0FBA3E0FAA3E0F9E475F001120081FC90082598E004F07007900825CE
:203FE00097E004F0213E0D90082596E004F0700790082595E004F0D390082596E0940490F8
:20400000082595E0648094805003213D2E7F002290081976E0FBA3E0FAA3E0F990081A6970
:20402000E0FEA3E0FFE92FF9EA3EFA900823FF7483F0A3749FF0A374FFF0120095929008CF
:204040001A6AE02FF090081A69E03EF090080660E0FBA3E0FAA3E0F9E4F5F01200822880DD
:20406000037F01227F0022E490081A6BF0A3F0C39008247AE09401FF90082479E09400FE62
:20408000C390081A6CE09FEE6480F890081A6BE06480984003214445A3E0FF12023BF4EFDC
:2040A0004E6006EF64014E705C12023D1190081B0D1200842FE4FFFEFDFC90081B0DE0F885
:2040C000A3E0F9A3E0FAA3E0FBC31200836E7003214432E47F01FEFDFC90081B15120084E0
:2040E0002FE47F02FEFDFC90081B111200842FE47FB97E0BFDFC90081B1D1200842FE47F16
:20410000BA7E0B805A12023D0190081B0D1200842FE4FFFEFDFC90081B0DE0F8A3E0F9A31A
:20412000E0FAA3E0FBC31200836E7003214432E47F04FEFDFC90081B151200842FE47F0801
:20414000FEFDFC90081B111200842FE47FD57E07FDFC90081B1D1200842FE47FD67E07FDD9
:20416000FC90081B191200842F90081A6CE0FF7B097A1A7971E490082ACAF012023D5F9013
:20418000081A6CE0FF7B097A1A797190082ACA7402F012023D5F90081A6CE0FF7B097A1AF9
:2041A000797190082ACA7406F012023D5F90081B15E0FCA3E0FDA3E0FEA3E0FF90081B0D88
:2041C000E0F8A3E0F9A3E0FAA3E05FFFEA5EFEE95DFDE85C4D4E4F700321431590081A8553
:2041E000E0FCA3E0FDA3E0FEA3E0FF90081A81E0F8A3E0F9A3E0FAA3E02FFFEA3EFEE93D5F
:20420000FDE83CFC90081A89E0F8A3E0F9A3E0FAA3E02FFFEA3EFEE93DFDE83CFC90081AA9
:20422000C1E0F8A3E0F9A3E0FAA3E02FFFEA3EFEE93DFDE83CFCA3E0F8A3E0F9A3E0FAA3BB
:20424000E02FFFEA3EFEE93DFDE83CFC90081A6D1200842F90081A6BE0FEA3E07802C33315
:20426000CE33CED8F924C2F58274143EF583759308E0F8A3E0F9A3E0FAA3E0FB90081A6D85
:20428000E0FCA3E0FDA3E0FEA3E0C39BFFEE9AFEED99FDEC98FCE47B32FAF9F8C312008304
:2042A0006E503290081B1FE0FEA3E0FFC006C00790081A6CE02401FF90081A6BE03400FEFE
:2042C0003395E0FDFC90082AB31200842FD007D00612020CA790081A6DE0FCA3E0FDA3E091
:2042E000FEA3E0FFC004C005C006C00790081A6BE0FEA3E07802C333CE33CED8F924C2F5BF
:204300008274143EF583759308D007D006D005D0041200842F90081B11E0FCA3E0FDA3E00F
:20432000FEA3E0FF90081B0DE0F8A3E0F9A3E0FAA3E05FFFEA5EFEE95DFDE85C4D4E4F7064
:204340000321443290081B05E0FCA3E0FDA3E0FEA3E0FFA3E0F8A3E0F9A3E0FAA3E02FFF87
:20436000EA3EFEE93DFDE83CFC90081A6D1200842F90081A6BE0FEA3E07802C333CE33CE33
:20438000D8F92442F58274153EF583759308E0F8A3E0F9A3E0FAA3E0FB90081A6DE0FCA333
:2043A000E0FDA3E0FEA3E0C39BFFEE9AFEED99FDEC98FCE47B32FAF9F8C31200836E503272
:2043C00090081B1BE0FEA3E0FFC006C00790081A6CE02401FF90081A6BE03400FE3395E029
:2043E000FDFC90082AB31200842FD007D00612020CA790081A6DE0FCA3E0FDA3E0FEA3E097
:20440000FFC004C005C006C00790081A6BE0FEA3E07802C333CE33CED8F92442F582741593
:204420003EF583759308D007D006D005D0041200842F90081A6CE004F0700790081A6BE035
:2044400004F021406F22900826EDEEF0A3EFF0A3EBF0A3EAF0A3E9F0E4FFFEFDFC9008265C
:20446000F61200842FE4FFFEFDFC900826FA1200842F900826EDE0FEA3E0FF900829B37437
:2044800009F0A37426F0A374F4F07B097A2679F21202285DC39008247AE09401FF900824AA
:2044A00079E09400FEC3900826EEE09FEE6480F8900826EDE0648098400321477C9008266D
:2044C000F5E0900826EF30E003214589E0FBA3E0FAA3E02401F9E43AFA120080D3FE90084C
:2044E00026EFA3E0FAA3E0F9120080D3FDEDFFE4FCFD900826F61200842F900826F4E0A2D6
:20450000E713FEA3E013FF7C007D0312008138EF2427FFE43EFEC006C007A3E0FCA3E0FD62
:20452000A3E0FEA3E0FF90082A711200842FD007D00612022DA9900826F4E0A2E713FEA31A
:20454000E013FF7C007D0312008138EF2427FFE43ECF2402CF3400FE7B097A2679F61202AA
:2045600032F5900826EFE0FBA3E0FAA3E02402F9E43AFA120080D3FA900826F6A3A3A3E079
:20458000FFE4FDFCEAFE214648E0FBA3E0FAA3E02401F9E43AFA120080D3FE900826EFA3E4
:2045A000E0FAA3E0F9120080D3FDEDFFE4FCFD900826F61200842F900826F4E0A2E713FED5
:2045C000A3E013FF7C007D0312008138EF2427FFE43ECF2401CF3400FEC006C007A3E0FC23
:2045E000A3E0FDA3E0FEA3E0FF90082A711200842FD007D00612022DA9900826F4E0A2E78E
:2046000013FEA3E013FF7C007D0312008138EF2427FFE43ECF2402CF3400FE7B097A26793F
:20462000F6120232F5900826EFE0FBA3E0FAA3E02402F9E43AFA120080D3FB900826F6A3D3
:20464000A3E0FEE4FDFCEBFFE4900826F61200842F900826F4E0A2E713FEA3E013FF7C0078
:204660007D0312008138EF2427FFE43ECF2402CF3400FEC006C007A3E0FCA3E0FDA3E0FE91
:20468000A3E0FF90082A711200842FD007D00612022DA9900826EFE0FBA3E0FAA3E024035A
:2046A000F9E43AFA120080D330E019E47F01FEFDFC900826F5E0F9F812008392900826FA9D
:2046C0001200842F7B097A2679F67F4B7E00120232F5900826F6E0F8A3E0F9A3E0FAA3E0F7
:2046E000FBC000A3E0FCA3E0FDA3E0FEA3E0FF78101200837FD000EB4FFFEA4EFEE9FDE854
:20470000FC900826F61200842F900826F6E0FCA3E0FDA3E0FEA3E0FF90082A711200842F19
:204720007F4B7E0012022DA97B097A2679F67F4C7E00120232F5900826F6E0F8A3E0F9A385
:20474000E0FAA3E0FB900826FCE0FEA3E0FFEB4FFFEA4EFEE9FDE8FC900826F61200842F35
:20476000900826F6E0FCA3E0FDA3E0FEA3E0FF90082A711200842F7F4C21481D900826EF30
:20478000E0FBA3E0FAA3E02403F9E43AFA120080D3FE900826EFA3E0FAA3E02402F9E43AB9
:2047A000FA120080D3FDEDFFE4FCFD900826F61200842F900826F6E0FCA3E0FDA3E0FEA327
:2047C000E0FF90082A711200842F7F4D7E0012022DA9900826EFE0FBA3E0FAA3E02401F928
:2047E000E43AFA120080D3FE900826EFA3E0FAA3E0F9120080D3FDEDFFE4FCFD900826F6B9
:204800001200842F900826F6E0FCA3E0FDA3E0FEA3E0FF90082A711200842F7F4E7E00126B
:20482000022DA922900829CEEBF0A3EAF0A3E9F090080403E0FBA3E0FAA3E0F9120080D343
:2048400014700321497B14700321497B24026003214B7CE49008246FF0A3F0900828327417
:2048600083F0A37489F0A374D1F0900829CEE0FBA3E0FAA3E0F9120207F5900829D1EBF07D
:20488000A3EAF0A3E9F0900829D1E0FBA3E0FAA3E04A4B7003FEFF22900828327483F0A30F
:2048A0007489F0A374E5F0900829D1E0FBA3E0FAA3E0F9120207F5900829D1EBF0A3EAF0BF
:2048C000A3E9F0900829D1E0FBA3E0FAA3E04A4B7003FEFF227B837A8979E51200A3BE9066
:2048E0000829D2EE8FF0801B900829D1E0FBA3E0FAA3E0F9120080D3B42D0E900829D2E47C
:2049000075F0011200818280DFC3E99401F9EA9400FA9008264B7483F0A37489F0A374EF85
:20492000F0A37483F0A37489F0A374F1F0A37409F0A37424F0A3744DF01201E0B49008297E
:20494000A07483F0A37489F0A374F4F07B097A24794D1202253D7B097A24794D1200A3BE8C
:204960009008246DEEF0A3EFF090080403E0FBA3E0FAA3E0F974011200812490080403E090
:20498000FBA3E0FAA3E0F9120080D364016003214A83900828327483F0A37489F0A374F98F
:2049A000F0900829CEE0FBA3E0FAA3E0F9120207F5900829D1EBF0A3EAF0A3E9F09008296D
:2049C000D1E0FBA3E0FAA3E04A4B7037D390082470E094059008246FE06480948040129092
:2049E0000829D17483F0A3748AF0A3740AF0214AB290082470E004F070609008246FE00430
:204A0000F080577B837A8979F91200A3BE900829D2EE8FF012008182E49008244BF0A3F066
:204A200090080403E0FBA3E0FAA3E0F9740212008124900829CEA3E0FAA3E0AE02FFA3A352
:204A4000E0FAA3E0C39FFFEA9EFE90081A69E0FCA3E0FDB50708ECB50604E4FEFF22C3ED79
:204A60009FFFEC9E90081A69F0A3EFF0900829D1E0F9A3E0FAA3E0900829CEC9F0A3EAF051
:204A8000A3E9F090081A69E0FEA3E0FF9008244CE02FFF9008244BE03EFED3EF94A8EE9466
:204AA000064051900829D17483F0A3748AF0A3741CF0900829D1E0F9A3E0FAA3E090082906
:204AC0006AC9F0A3EAF0A3E9F0A37483F0A3748AF0A3743DF07B837A8A792E120215789081
:204AE000080403E0FBA3E0FAA3E0F9E412008124FE7F012290081A69E0FEA3E0FF90082461
:204B00004BE0FCA3E02400F974073CA801FC7D09900829CEE0FBA3E0FAA3E0F912008055A2
:204B200090081A69E0FEA3E0FF9008244CE02FF09008244BE03EF09008246DE0FCA3E0FD59
:204B40009008244BE0FAA3E02400F974073AFA7B09C3E99DF9EA9CFAC3E9940AF9EA94001E
:204B6000FA900828327409F0A37424F0A3744DF0120207F5E94A4B7003FEFF221202269E65
:204B8000900829D4EEF0A3EFF064014E7012900829D17483F0A3748AF0A37448F0214AB275
:204BA000900829D4E0FEA3E0FF64024E7012900829D17483F0A3748AF0A37465F0214AB237
:204BC000EF64034E7012900829D17483F0A3748AF0A3747CF0214AB290082492E4F0A3043C
:204BE000F090080403E0FBA3E0FAA3E0F9E412008124900819847410F07E007F0122900856
:204C0000275DEBF0A3EAF0A3E9F09008066BE0FBA3E0FAA3E0F9120081AEFF90082765E516
:204C2000F0F0A3EFF090081976E0FBA3E0FAA3E0F990081A69E0FEA3E0FFE92FF9EA3EFA69
:204C4000900823FF7483F0A374A4F0A374ECF01200959290081A6AE02FF090081A69E03E88
:204C6000F0E490082763F0A3F090082763E0FEA3E0FFC3940CEE648094804003214D6A9045
:204C8000082766E02FFF90082765E03EFE90082767F0A3EFF0C390082484E09401FD90088C
:204CA0002483E09400FCD3EF9DEC6480F8EE648098405790081976E0FBA3E0FAA3E0F9902A
:204CC000081A69E0FEA3E0FFE92FF9EA3EFA900823FF7483F0A374A5F0A37401F0900827A2
:204CE00063E0FEA3E0FFC3740C9F90082403F0E49E90082402F01200959290081A6AE02FCC
:204D0000F090081A69E03EF0806090081976E0FBA3E0FAA3E0F990081A69E0FEA3E0FFE93B
:204D20002FF9EA3EFA900823FF7483F0A374A5F0A37419F090082767E0FFA3E09008240276
:204D4000CFF0A3EFF01200959290081A6AE02FF090081A69E03EF090082764E004F0700727
:204D600090082763E004F0214C6990081976E0FBA3E0FAA3E0F990081A69E0FEA3E0FFE908
:204D80002FF9EA3EFA900823FF7483F0A374A4F0A374ECF01200959290081A6AE02FF090A6
:204DA000081A69E03EF0E490082763F0A3F090082763E0FEA3E0FFC3940CEE6480948040C6
:204DC00003214F5D90082766E02FFF90082765E03EFE90082767F0A3EFF0C390082484E015
:204DE0009401FD90082483E09400FCD3EF9DEC6480F8EE648098405890081976E0FBA3E0C4
:204E0000FAA3E0F990081A69E0FEA3E0FFE92FF9EA3EFA900823FF7483F0A374A5F0A3740A
:204E200001F090082763E0FEA3E0FFC3740C9F90082403F0E49E90082402F0120095929075
:204E4000081A6AE02FF090081A69E03EF0214F5D90082768E024FFF090082767E034FFF08E
:204E6000E0FEA3E07803CEA2E713CE13D8F8FF9008275DE0FBA3E0FAA3E02FF9EA3EFA12E9
:204E80000080D3FD7C0090082768E05407FF74017E00A807088005C333CE33CED8F9FFEE33
:204EA0005CFEEF5D4E90082769600D7483F0A374A5F0A37428F0800B7483F0A374A5F0A3E6
:204EC0007430F090081976E0FBA3E0FAA3E0F990081A69E0FEA3E0FFE92FF9EA3EFAC003D2
:204EE000C002C001900823FF7483F0A374A5F0A37431F090082760E0F9A3E0FAA3E090081A
:204F00002402C9F0A3EAF0A3E9F090082767E0FFA3E090082405CFF0A3EFF090082769E027
:204F2000F9A3E0FAA3E090082407C9F0A3EAF0A3E9F0D001D002D0031200959290081A6A38
:204F4000E02FF090081A69E03EF090082764E004F0700790082763E004F0214DAE9008060B
:204F60006BE0FBA3E0FAA3E0F9E475F00C120081FC9008066BE0FBA3E0FAA3E0F91200819E
:204F8000AEFFC390082484E09401FD90082483E09400FCD3EF9DE5F09C40057E007F01220B
:204FA000E4FEFF2290082424EBF0A3EAF0A3E9F0E490082433F0A3F0900828327481F0A36A
:204FC000748BF0A374F9F090082424E0FBA3E0FAA3E0F9120207F590082424EBF0A3EAF0E6
:204FE000A3E9F09008264B7481F0A3748BF0A374F9F0A37481F0A3748AF0A37458F0A37426
:2050000009F0A37424F0A37441F01201E0B4E490082435F0A3F07B097A2479411200A3BED6
:20502000C390082436E09FEE6480F890082435E0648098502BA3E02441F582E43424F58397
:20504000759308E0FF12023D50400321510790082436E004F070BF90082435E004F080B614
:205060007B097A24794112020007AC06AD0790082434E025E0FF90082433E033FE742B2F31
:20508000F58274243EF583759308ECF0A3EDF090082425E475F0011200818290082434E0CF
:2050A00004F0700790082433E004F0C390082434E0940490082433E0648094805003214F0D
:2050C000B8E4FFFEFDFC9008242BE0F8A3E0F9A3E0FAA3E0FBC31200836E700EFFFEFDFCCE
:2050E000900824271200842F80469008281A7409F0A37424F0A37427F07B097A24792B12CA
:2051000001CDC9EF4E70299008296A7481F0A3748DF0A374B9F0A37481F0A3748DF0A3748B
:20512000C9F07B817A8D79AC12021578E4FEFF2290082427E0FCA3E0FDA3E0FEA3E0FF1296
:20514000023E2290082433E4F0A304F090082433E0FEA3E0FFD39403EE6480948040032190
:205160005337EF64014E70119008243E7481F0A3748BF0A3746BF0802FEF64024E7011903C
:2051800008243E7481F0A3748DF0A374D2F08018EF64034E60032153379008243E7481F02A
:2051A000A3748DF0A374D7F0E4FFFEFDFC900824371200842F9008243EE0F9A3E0FAA3E018
:2051C00090082832C9F0A3EAF0A3E9F090082424E0FBA3E0FAA3E0F9120207F59008243B70
:2051E000EBF0A3EAF0A3E9F09008243BE0FBA3E0FAA3E04A4B70032152C0900823FF74811F
:20520000F0A3748DF0A374DCF09008243EE0F9A3E0FAA3E090082402C9F0A3EAF0A3E9F0E4
:205220007B097A24794112009592900823017409F0A37424F0A37441F0A37409F0A3742472
:20524000F0A37449F09008243BE0FBA3E0FAA3E0F91200997190082437E0F8A3E0F9A3E05D
:20526000FAA3E0FBC000C001E47F01FEFDFC9008244AE0F9F812008392D001D000EB4FFF02
:20528000EA4EFEE94DFDE84CFC900824371200842F9008243EE0FBA3E0FAA3E0F91200A33A
:2052A000BE9008243BE0FBA3E0FAA3E02FF9EA3EFA90082424EBF0A3EAF0A3E9F02151B539
:2052C00090082433E07004A3E06401701590082437E0FCA3E0FDA3E0FEA3E0FF12023E2A50
:2052E000804290082433E07004A3E06402701590082437E0FCA3E0FDA3E0FEA3E0FF1202D5
:205300003E32802090082433E07004A3E06403701390082437E0FCA3E0FDA3E0FEA3E0FF7B
:2053200012023E3A90082434E004F0700790082433E004F021514C120234B17E007F01220C
:205340009008298BE0FBA3E0FAA3E02428F9E43AFA90082B97EBF0A3EAF0A3E9F0E475F052
:20536000011200822890082B98E475F0021200818212023D78EF2404FFE43EF990082B9761
:20538000E0FBA3E0FAA3E0C98FF01200822890082B98E475F00212008182900823FF7481C4
:2053A000F0A374A2F0A374DFF0A37481F0A374A2F0A374E2F090082B97E0FBA3E0FAA3E01F
:2053C000F91200959212023D7890082B98EE8FF01200818290082B97E0FBA3E0FAA3E0F9C7
:2053E000E475F0021200822890082B98E475F0021200818290082B97E0FBA3E0FAA3E0F9BD
:20540000E475F0181200822890082B98E475F0021200818212023E73C003C00290082B9710
:20542000E0FBA3E0FAA3E0F8AC02AD03D002D0037E007F141200805590082B98E475F014E6
:205440001200818290082B97E0FBA3E0FAA3E0F9E475F0031200822890082B98E475F0025B
:205460001200818290082B97E0FBA3E0FAA3E0F9E475F0181200822890082B98E475F00226
:205480001200818212023E7AC003C00290082B97E0FBA3E0FAA3E0F8AC02AD03D002D00376
:2054A0007E007F141200805590082B98E475F0141200818290082B97E0FBA3E0FAA3E0F9F9
:2054C000E475F0041200822890082B98E475F0021200818290082B97E0FBA3E0FAA3E0F9DA
:2054E000E475F0081200822890082B98E475F0021200818212023CB190082B97E0FBA3E02B
:20550000FAA3E0F9120083C290082B98E475F0041200818290082B97E0FBA3E0FAA3E0F9D3
:20552000E475F0051200822890082B98E475F0021200818290082B97E0FBA3E0FAA3E0F978
:20554000E475F0081200822890082B98E475F0021200818212023CC190082B97E0FBA3E0BA
:20556000FAA3E0F9120083C290082B98E475F0041200818290082B97E0FBA3E0FAA3E0F973
:20558000E475F0061200822890082B98E475F0021200818290082B97E0FBA3E0FAA3E0F917
:2055A000E475F0081200822890082B98E475F0021200818212023CD190082B97E0FBA3E04A
:2055C000FAA3E0F9120083C290082B98E475F0041200818290082B97E0FBA3E0FAA3E0F913
:2055E000E475F0071200822890082B98E475F0021200818290082B97E0FBA3E0FAA3E0F9B6
:20560000E475F0081200822890082B98E475F0021200818212023CE190082B97E0FBA3E0D9
:20562000FAA3E0F9120083C290082B98E475F0041200818290082B97E0FBA3E0FAA3E0F9B2
:20564000E475F0151200822890082B98E475F0021200818290082B97E0FBA3E0FAA3E0F947
:20566000E475F0061200822890082B98E475F0021200818212023DAB90082B97E0FBA3E0B0
:20568000FAA3E0F9EE8FF01200822890082B98E475F002120081829008298BA3E0FAA3E064
:2056A000AE02FF90082B97A3E0FAA3E0C39FFFEA9E90081A69F0A3EFF02290080660E0FB70
:2056C000A3E0FAA3E0F9120081AEFFAEF0E5F06003215A1FEF24FE700321579014700321ED
:2056E00059CE24026003215A1F900823FF7483F0A37497F0A37431F090081976E0FBA3E064
:20570000FAA3E0F91200959290081A69EEF0A3EFF090082A43E4F0A304F090081976E0FBED
:20572000A3E0FAA3E0F990081A69E0FEA3E0FFE92FF9EA3EFA900823FF7483F0A37498F082
:20574000A3742FF01200959290081A6AE02FF090081A69E03EF090082A44E004F0700790B5
:20576000082A43E004F0D390082A44E0940290082A43E06480948040A190080660E0FBA357
:20578000E0FAA3E0F9E475F002120082287F002290082A43E4F0A304F09008066BE0FBA314
:2057A000E0FAA3E0F9120081AEC39401FFE5F09400FE90082A47F0A3EFF0C39008247AE040
:2057C0009401FD90082479E09400FCEDB5071BECB5061790080660E0FBA3E0FAA3E0F9E45A
:2057E00075F003120082282159CE90081976E0FBA3E0FAA3E0F990081A69E0FEA3E0FFE9DE
:205800002FF9EA3EFA900823FF7483F0A37498F0A37467F01200959290081A6AE02FF090AC
:20582000081A69E03EF090082A45E4F0A304F090082A45E0FEA3E0FFD39402EE64809480A7
:2058400040032159A5EF64024E703190082A48E004F0700790082A47E004F0C39008247A77
:20586000E09401FF90082479E09400FE90082A47E0B50608A3E0B507037F002290082A4874
:20588000E0FF12023BF4EF64024E6012EF64044E600CEF64034E6006EF64054E70449008C4
:2058A0001976E0FBA3E0FAA3E0F990081A69E0FEA3E0FFE92FF9EA3EFA900823FF7483F036
:2058C000A37498F0A3746EF090082A48E02401FE90082A47E0340090082402F0A3CEF0215A
:2058E000596C90082A48E0FF7B097A2A79491202359790081976E0FBA3E0FAA3E0F990089D
:205900001A69E0FEA3E0FFE92FF9EA3EFAC003C002C001900823FF7483F0A37498F0A374D4
:2059200096F090082A47E0FEA3E0FF90082402EEF0A3EFF02401FFE43EA3F0A3EFF0900867
:205940002A49E075F003A42482F582E43429F583759308E0F9A3E0FAA3E090082406C9F0AE
:20596000A3EAF0A3E9F0D001D002D0031200959290081A6AE02FF090081A69E03EF09008A3
:20598000066BE0FBA3E0FAA3E0F9E475F001120081FC90082A46E004F0700790082A45E0AF
:2059A00004F021582F90082A44E004F0700790082A43E004F0D390082A44E0940490082A0E
:2059C00043E06480948050032157997F002290081976E0FBA3E0FAA3E0F990081A69E0FEB3
:2059E000A3E0FFE92FF9EA3EFA900823FF7483F0A37498F0A374E8F01200959290081A6A6E
:205A0000E02FF090081A69E03EF090080660E0FBA3E0FAA3E0F9E4F5F01200822880037F05
:205A200001227F002290080660E0FBA3E0FAA3E0F9120081AEFFAEF0E5F06003215D8BEFC2
:205A400024FE602E147003215B80147003215D4D24036003215D8B7F017E0012020D5D9022
:205A6000080660E0FBA3E0FAA3E0F9E475F002215D84900823FF7483F0A37474F0A3742A3A
:205A8000F090081976E0FBA3E0FAA3E0F91200959290081A69EEF0A3EFF0900829DEE4F0F4
:205AA000A304F0C390082484E09401FF90082483E09400FE900829DEE0FCA3E0FDD39FEECC
:205AC0006480F8EC648098505490081976E0FBA3E0FAA3E0F990081A69E0FEA3E0FFE92F50
:205AE000F9EA3EFA900823FF7483F0A37470F0A374F1F0A3ECF0A3EDF01200959290081A91
:205B00006AE02FF090081A69E03EF0900829DFE004F0708F900829DEE004F0808690081956
:205B200076E0FBA3E0FAA3E0F990081A69E0FEA3E0FFE92FF9EA3EFA900823FF7483F0A329
:205B40007470F0A374FFF01200959290081A6AE02FF090081A69E03EF09008066BE0FBA367
:205B6000E0FAA3E0F9E475F0011200822890080660E0FBA3E0FAA3E0F9E475F003215D84A9
:205B80009008066BE0FBA3E0FAA3E0F9120081AEFFC390082484E09401FD90082483E094C0
:205BA00000FCD3EF9DE5F09C402B90080660E0FBA3E0FAA3E0F9E475F00412008228D39070
:205BC000081A6AE0940090081A69E094005003215D4D7F002290081976E0FBA3E0FAA3E075
:205BE000F990081A69E0FEA3E0FFE92FF9EA3EFA900823FF7483F0A37471F0A37447F01285
:205C000000959290081A6AE02FF090081A69E03EF0900829DEE4F0A37402F0900829DEE01E
:205C2000FEA3E0FFC3EE648094805003215D22EF4E701AA37483F0A37471F0A3744FF0A386
:205C40007483F0A37470F0A37406F0801B900829E07483F0A37470F0A37406F0A37483F0A8
:205C6000A37471F0A37457F090081976E0FBA3E0FAA3E0F990081A69E0FEA3E0FFE92FF9C7
:205C8000EA3EFAC003C002C001900823FF7483F0A37471F0A3745CF09008066BE0FBA3E0B9
:205CA000FAA3E0F9120081AEC39401FEE5F0940090082402F0A3CEF0900829DEE0FFA3E05E
:205CC00090082404CFF0A3EFF0900829E0E0F9A3E0FAA3E090082406C9F0A3EAF0A3E9F0D5
:205CE000900829E3E0F9A3E0FAA3E090082409C9F0A3EAF0A3E9F0D001D002D00312009593
:205D00009290081A6AE02FF090081A69E03EF0900829DFE024FFF0900829DEE034FFF02157
:205D20005C1B9008066BE0FBA3E0FAA3E0F9E475F001120081FCC390081A6AE094B090089B
:205D40001A69E094045003215B807F0022900823FF7483F0A37475F0A3747EF0900819768F
:205D6000E0FBA3E0FAA3E0F91200959290081A69EEF0A3EFF090080660E0FBA3E0FAA3E0C2
:205D8000F9E4F5F0120082287F00227F01227B097A19798F90081A66EBF0A3EAF0A3E9F037
:205DA0002414F9E43AFA74111200812474FFFFFEFDFC90081A66E0FBA3E0FAA3E02404F9E1
:205DC000E43AFA120083C290081A66E0FBA3E0FAA3E0F9E475F0441200822890081A66E027
:205DE000FBA3E0FAA3E02402F9E43AFAE475F0431200822812020B2B12023DF0EF4E700EE3
:205E000012023DC9AC06AD077F01120235269008197CE0FBA3E0FAA3E02408F9E43AFA903E
:205E2000082A99EBF0A3EAF0A3E9F024ECF9E43AFAA3EBF0A3EAF0A3E9F090082A99E0FBF5
:205E4000A3E0FAA3E0F974011200812490082A99E0FBA3E0FAA3E02401F9E43AFA7401122A
:205E600000812490082A99E0FBA3E0FAA3E02402F9E43AFA740612008124900822ECE0FC5D
:205E8000A3E0FDA3E0FEA3E0FF90082A99E0FBA3E0FAA3E02404F9E43AFA120083C2900821
:205EA0002A99E0FBA3E0FAA3E0241CF9E43AA801FCAD037B097A2279F47E007F0612008076
:205EC000557F637E537D827C6390082A9CE0FBA3E0FAA3E0F9120083C290082A9DE475F0AB
:205EE000041200818290082A9CE0FBA3E475F00112008198A9F0FA74351200812490082A83
:205F00009CE0FBA3E475F00112008198A9F0FA74011200812490082A9CE0FBA3E475F0010D
:205F200012008198A9F0FA74031200812490082A9CE0FBA3E475F00112008198A9F0FA741D
:205F40003D1200812490082A9CE0FBA3E475F00112008198A9F0FA74071200812490082A75
:205F60009CE0FBA3E475F00112008198A9F0FA74011200812490082A9CE0FBA3E0FAA3E09A
:205F8000F8AC02AD037B097A2279F47E007F061200805590082A9DE475F0061200818290E1
:205FA000082A9CE0FBA3E475F00112008198A9F0FA74321200812490082A9CE0FBA3E475FB
:205FC000F00112008198A9F0FA740412008124900822E8E0FCA3E0FDA3E0FEA3E0FF90084A
:205FE0002A9CE0FBA3E0FAA3E0F9120083C290082A9DE475F0041200818290082A9CE0FBB6
:20600000A3E475F00112008198A9F0FA74361200812490082A9CE0FBA3E475F001120081BB
:2060200098A9F0FA740412008124900822E0E0FCA3E0FDA3E0FEA3E0FF90082A9CE0FBA331
:20604000E0FAA3E0F9120083C290082A9DE475F0041200818290082A9CE0FBA3E475F001AC
:2060600012008198A9F0FA74371200812490082A9CE0FBA3E475F00112008198A9F0FA74A8
:20608000021200812490082A9CE0FBA3E475F00112008198A9F0FA74011200812490082A75
:2060A0009CE0FBA3E475F00112008198A9F0FA74031200812490082A9CE0FBA3E0FAA3E057
:2060C000F974FF1200812490081A697401F0A3742CF07F017E000201272590080660E0FBC4
:2060E000A3E0FAA3E0F9120081AEFFAEF0E5F0600321640FEF24FE70032161AD14700321A2
:20610000637F2402600321640F900823FF7483F0A3745BF0A37457F090081976E0FBA3E09A
:20612000FAA3E0F91200959290081A69EEF0A3EFF09008287FE4F0A304F090081976E0FB89
:20614000A3E0FAA3E0F990081A69E0FEA3E0FFE92FF9EA3EFA900823FF7483F0A3745CF094
:20616000A37438F01200959290081A6AE02FF090081A69E03EF090082880E004F070079048
:2061800008287FE004F0D390082880E094029008287FE06480948040A190080660E0FBA37F
:2061A000E0FAA3E0F9E475F002120082289008066BE0FBA3E0FAA3E0F9120081AEC394010C
:2061C000FFE5F09400FE9008287DF0A3EFF0900828EA7409F0A37428F0A37481F07B097ADE
:2061E00028798412021232EF4E707E90080660E0FBA3E0FAA3E0F9E475F00312008228908D
:2062000008287DE0FEA3E0FF7C007D021200814AED64014C703C90081976E0FBA3E0FAA32D
:20622000E0F990081A69E0FEA3E0FFE92FF9EA3EFA900823FF7483F0A3745CF0A37485F047
:206240001200959290081A6AE02FF090081A69E03EF0D390081A6AE0940090081A69E094CF
:2062600000500321637F7F00229008287DE0FEA3E0FF7C007D021200814AED4C703C900835
:206280001976E0FBA3E0FAA3E0F990081A69E0FEA3E0FFE92FF9EA3EFA900823FF7483F04C
:2062A000A3745CF0A3749CF01200959290081A6AE02FF090081A69E03EF090082881E0FB3F
:2062C000A3E0FAA3E0F91200A3BEEF4E700F900828817483F0A37453F0A37474F0900819E8
:2062E00076E0FBA3E0FAA3E0F990081A69E0FEA3E0FFE92FF9EA3EFAC002C001900823FF69
:206300007483F0A3745CF0A374B0F09008287DE0FEA3E0FF90082402EEF0A3EFF02401FF9D
:20632000E43EA3F0A3EFF090082881E0F9A3E0FAA3E090082406C9F0A3EAF0A3E9F0D001C7
:20634000D0021200959290081A6AE02FF090081A69E03EF09008066BE0FBA3E0FAA3E0F911
:20636000E475F001120081FCC390081A6AE094B090081A69E0940450032161AD7F002290FB
:2063800008066BE0FBA3E0FAA3E0F9120081AEC39401FFE5F09400FEEF64014E900823FF55
:2063A000700C7483F0A3745CF0A374F3802B7483F0A3745EF0A3749AF09008066BE0FBA3EE
:2063C000E0FAA3E0F9120081AEC39401FFE5F09400FE90082402F0A3EFF0A3EEF0A3EFF035
:2063E00090081976E0FBA3E0FAA3E0F91200959290081A69EEF0A3EFF090080660E0FBA372
:20640000E0FAA3E0F9E4F5F0120082287F00227F0122900823D3EBF0A3EAF0A3E9F0E4A375
:20642000F0A3F0900828327481F0A3748EF0A3747BF0120207F5900823D3EBF0A3EAF0A352
:20644000E9F09008264B7481F0A3748EF0A3747BF0A37481F0A3748AF0A37458F0A37409C6
:20646000F0A37423F0A374E8F01201E0B4E4900823D8F0A3F07B097A2379E81200A3BEC3BA
:20648000900823D9E09FEE6480F8900823D8E06480985039A3E024E8F582E43423F5837579
:2064A0009308E0FF12023D5040119008296A7481F0A3748EF0A3748C21654E900823D9E0E0
:2064C00004F070B1900823D8E004F080A87B097A2379E812020007900823DCEEF0A3EFF084
:2064E000C3900823D7E09401900823D6E06480948040109008296A7481F0A3748EF0A3745D
:20650000BC804B900823D6E0FEA3E0FF7B097A2379DE120228C5EF4E7010900823DCE0FF57
:20652000A3E0A3CFF0A3EFF08052900823DEE0FEA3E0FF900823DCE0B5062EA3E0B5072961
:206540009008296A7481F0A3748EF0A374D5F0A37481F0A3748EF0A374B1F07B817A8E7968
:206560008012021578E4FEFF22900823D7E004F07007900823D6E004F02164E07E007F044F
:206580007D007B097A2379E0120088517E007F047D007B097A2379E412008851E490082393
:2065A000D8F0A3F0C390082484E09401FF90082483E09400FEC3900823D9E09FEE6480F8B8
:2065C000900823D8E06480984003216722900823FF7481F0A3748EF0A374F3F0900823D81E
:2065E000E0FFA3E090082402CFF0A3EFF07B097A2379E812009592900828327409F0A37409
:2066000023F0A374E8F0900823D3E0FBA3E0FAA3E0F9120207F5900823D3EBF0A3EAF0A37D
:20662000E9F0900829A07481F0A3748EF0A374F8F07B097A2379E81202253D90082301747F
:2066400009F0A37423F0A374E8F0A37409F0A37423F0A374DCF0900823D3E0FBA3E0FAA382
:20666000E0F912009971900823D8E0FCA3E0FDAE047803CEA2E713CE13D8F8FF900823DA5A
:20668000EEF0A3EFF07E00ED5407FFD3900823DDE09400900823DCE064809480406590084A
:2066A00023DBE024E0F582E43423F583C083C082759308E0FDAC077401A804088002C33308
:2066C000D8FC4D759308D082D083F0900823DCE07004A3E06402702B900823DBE024E4F512
:2066E00082E43423F583C083C082759308E0FD7401A807088002C333D8FC4D759308D082CC
:20670000D083F0900823D4E475F00112008182900823D9E004F07007900823D8E004F021E1
:2067200065A4900823D6E0FEA3E0FF7B097A2379DE1200FFFB120234B17E007F012290082A
:206740001A6AE024E4F090081A69E034FFF0C3A3E09428FE90081A69E0940090081F66F023
:20676000A3CEF09008298BE0FBA3E0FAA3E02428F9E43AFA90081F09EBF0A3EAF0A3E9F0A0
:20678000D390081F67E0940090081F66E0648094805003216A6090081F09E0FBA3E0FAA3A6
:2067A000E0F9120081AE90081F6AF0E92402F9E43AFA120081AEFFAEF090081F68EEF0A310
:2067C000EFF0C39404FFEE9400FE90081F09A3E0FAA3E02404F9E43AFA780C7C1F7D091250
:2067E000008055C390081F69E09404FF90081F68E09400FE740C2FF582741F3EF583759362
:2068000008E4F090082471E07002A3E060032168A690081F6AE06409600321678012023EDD
:2068200057780C7C1F7D09120085E9EF705490082471F0A304F090081F68E0FEA3E0FF9066
:20684000081F0AEE8FF012008182C390081F67E09FF090081F66E09EF09008298BE0FBA3E0
:20686000E0FAA3E0240CF9E43AFA120081AE640A45F0600321678090082485F0A304F02142
:2068800067809008298BE0FBA3E0FAA3E0240EF9E43AFAE475F00212008228E490081F669F
:2068A000F0A3F021678090081F68E0FEA3E0FF90081F0AEE8FF012008182C390081F67E0CA
:2068C0009FF090081F66E09EF090081F6AE0120084B867800168F402690103690E04694078
:2068E0000569720669A90769BF0869CC0A6A211500006A447B097A1F790C12023D972167CA
:20690000807B097A1F790C12023DA121678012023CB190081F0CE0F8A3E0F9A3E0FAA3E043
:20692000FBC31200836E700321678090081F0CE0FCA3E0FDA3E0FEA3E0FF900824758062E6
:2069400012023CC190081F0CE0F8A3E0F9A3E0FAA3E0FBC31200836E700321678090081F1C
:206960000CE0FCA3E0FDA3E0FEA3E0FF90082487803012023CD190081F0CE0F8A3E0F9A3DE
:20698000E0FAA3E0FBC31200836E700321678090081F0CE0FCA3E0FDA3E0FEA3E0FF9008A4
:2069A000247B1200842F21678090081F0CE0FCA3E0FDA3E0FEA3E0FF12023E222167807B52
:2069C000097A1F790C12023D8D21678090081F0CE090081F6B7005F0A3F08005E4F0A304ED
:2069E000F012023DF9AC06AD0790081F6BE0FEA3E0FF6D7002EE6C7003216780EF64014E1F
:206A000070089008247FF0A304F012023E6C120080231201797B12020B2B1201534021674A
:206A20008012023DAB90081F0CE0FCA3E0FD6F7002EC6E700321678090082494ECF0A3ED49
:206A4000F02167809008298BE0FBA3E0FAA3E0240EF9E43AFAE475F00412008228216780C3
:206A6000229008265CEEF0A3EFF0A3EBF0A3EAF0A3E9F07E007F047D007B097A26796B126B
:206A8000008851786B7C267D099008265EE0FBA3E0FAA3E0F97E007F04120087C7EF700A58
:206AA00090082666F0A3F0216B349008265DE024CEF582E4340FF583759308E0FF7E00906F
:206AC000082666EEF0A3EFF0F4706990082666F0A3F090082666E0FEA3E0FFC39418EE6409
:206AE0008094805036EF7802C333CE33CED8F92444F9740E3EFA7B09786B7C267D097E0055
:206B00007F04120087C7EF601290082667E004F070C090082666E004F080B790082667E0D4
:206B2000FF9008265DE024CEF582E4340FF583759308EFF07E007F807D007B097A18797368
:206B40001200885190082666E0FEA3E07802C333CE33CED8F92444F9740E3EA801FC7D0969
:206B60009008265EE0FBA3E0FAA3E0F97E007F0412008055E490082664F090082664E0FF46
:206B8000C394184003216C36EF75F004A42444F9740E35F0FA900826687409F0A3EAF0A3CF
:206BA000E9F0E490082665F090082665E0FFD390082484E09F7480F890082483E0648098EA
:206BC000406A90082665E0131313541FFE90082668E0FBA3E0FAA3E02EF9E43AFA1200808C
:206BE000D3FEEF5407FF7401A807088002C333D8FC5E602E90082665E075F004A42473F977
:206C0000741835F0FA90082A1C7409F0A3EAF0A3E9F090082668E0FBA3E0FAA3E0F9120277
:206C2000099A90082665E004F0216BA890082664E004F0216B7AE490082664F09008266472
:206C4000E0FFFDD390082484E09D7480F890082483E06480985003216D08EF75F004A42438
:206C6000F3F9741835F0FA900826687409F0A3EAF0A3E9F0E490082665F090082665E0FFF8
:206C8000D390082484E09F7480F890082483E0648098406A90082665E0131313541FFE90F4
:206CA000082668E0FBA3E0FAA3E02EF9E43AFA120080D3FEEF5407FF7401A807088002C307
:206CC00033D8FC5E602E90082665E075F004A42473F9741835F0FA90082A1C7409F0A3EA9E
:206CE000F0A3E9F090082668E0FBA3E0FAA3E0F91202099A90082665E004F0216C7A9008E1
:206D00002664E004F0216C3CE490082664F090082664E0FFFDD390082484E09D7480F8904C
:206D2000082483E06480984023EF75F004A42473F9741835F0FA7B0990082664E07E001298
:206D400001444690082664E004F080C290082666E0FEA3E0FF7C007D091200813874B32FC9
:206D6000F9740E3EA801FC7D0990082661E0FBA3E0FAA3E0F90200869390081BD0EBF0A320
:206D8000EAF0A3E9F0900828327481F0A3748AF0A3743EF0120207F590081BD0EBF0A3EAF5
:206DA000F0A3E9F0900823017481F0A3748AF0A37447F0A37409F0A3741BF0A374D6F012C6
:206DC0000099719008264B7481F0A3748AF0A37452F0A37481F0A3748AF0A37458F0A37442
:206DE00009F0A3741BF0A374D8F090081BD01201E0AC90081BD6E0FEA3E0FF7C007D09127A
:206E000000813874B32FF9740E3EFA7B09900829F17409F0A3741BF0A374D8F0A3E4F0A3F2
:206E20007421F0120221CFEF7003216EB3E490081C79F0A3F090081C79E0FEA3E0FFC394AD
:206E400018EE64809480506B7C007D091200813874B32FF9740E3EFA7B09900829F17409F0
:206E6000F0A3741BF0A374D8F0A3E4F0A37421F0120221CFEF702A900823FF7481F0A3743F
:206E80008AF0A3745AF07B097A1C795D120095929008296A7481F0A3748AF0A37470217035
:206EA0004890081C7AE004F0708B90081C79E004F080827B097A1B79D81201DAFD7B097A38
:206EC0001B79D81200A3BED3EF9408EE64809480403D900823FF7481F0A3748AF0A374903B
:206EE000F0A3E4F0A37408F07B097A1B79F9120095929008296A7409F0A3741BF0A374F98E
:206F0000F0A37481F0A3748AF0A3745A2170547E007F047D007B097A1C7975120088519011
:206F20000828327481F0A3748AF0A374B2F090081BD0E0FBA3E0FAA3E0F9120207F59008C1
:206F40001BD3EBF0A3EAF0A3E9F090081BD3E0FBA3E0FAA3E04A4B7003216FF990082301C1
:206F60007481F0A3748AF0A374B7F0A37409F0A3741CF0A37473F090081BD3E0FBA3E0FA52
:206F8000A3E0F91200997190081BD3E0FBA3E0FAA3E02404F9E43AFA90081BD0EBF0A3EAD4
:206FA000F0A3E9F090081C73E0FAA3E0FB7C007D08FFAE021200814A90081C71EEF0A3EFC4
:206FC000F07C007D08AF03AE021200814AE02475F582E4341CF583C083C082759308E0FF71
:206FE000AE057401A806088002C333D8FC4F759308D082D083F0216F1F90081BD6E0FEA3BA
:20700000E0FF7B097A1C797512019973EF4E7053900823FF7481F0A3748AF0A374C0F090E3
:20702000081BD6E0FFA3E090082402CFF0A3EFF07B097A1C795D120095929008296A7481AD
:20704000F0A3748AF0A374CFF0A37409F0A3741CF0A3745DF07B817A8A796312021578E4E1
:20706000FEFF2290081BD6E0FEA3E0FF900826617409F0A3741BF0A374D8F07B097A1C79E8
:207080007512016A61120234B17E007F012212023DF9EF4E700321739F900822DEE070046B
:2070A000A3E06404600321739F12023CA1900822F0E0F8A3E0F9A3E0FAA3E0FBD3120083FD
:2070C0006E400321739F7B097A19798F90081A66EBF0A3EAF0A3E9F02414F9E43AFA7411F3
:2070E00012008124900822E0E0FCA3E0FDA3E0FEA3E0FF90081A66E0FBA3E0FAA3E02404C5
:20710000F9E43AFA120083C290081A66E0FBA3E0FAA3E0F9E475F0441200822890081A66BA
:20712000E0FBA3E0FAA3E02402F9E43AFAE475F0431200822812020B2B12023DF0EF4E70BD
:207140000E12023DC9AC06AD077F01120235269008197CE0FBA3E0FAA3E02408F9E43AFA6D
:2071600090082A9FEBF0A3EAF0A3E9F024ECF9E43AFAA3EBF0A3EAF0A3E9F012023CA190C1
:207180000822EC1200842F90082A9FE0FBA3E0FAA3E0F974011200812490082A9FE0FBA3D4
:2071A000E0FAA3E02401F9E43AFA74011200812490082A9FE0FBA3E0FAA3E02402F9E43A97
:2071C000FA740612008124900822ECE0FCA3E0FDA3E0FEA3E0FF90082A9FE0FBA3E0FAA323
:2071E000E02404F9E43AFA120083C290082A9FE0FBA3E0FAA3E0241CF9E43AA801FCAD0337
:207200007B097A2279F47E007F06120080557F637E537D827C6390082AA2E0FBA3E0FAA307
:20722000E0F9120083C290082AA3E475F0041200818290082AA2E0FBA3E475F00112008198
:2072400098A9F0FA74351200812490082AA2E0FBA3E475F00112008198A9F0FA7401120032
:20726000812490082AA2E0FBA3E475F00112008198A9F0FA74031200812490082AA2E0FB12
:20728000A3E475F00112008198A9F0FA743D1200812490082AA2E0FBA3E475F0011200811C
:2072A00098A9F0FA74071200812490082AA2E0FBA3E475F00112008198A9F0FA7401120000
:2072C000812490082AA2E0FBA3E0FAA3E0F8AC02AD037B097A2279F47E007F0612008055FD
:2072E00090082AA3E475F0061200818290082AA2E0FBA3E475F00112008198A9F0FA743235
:207300001200812490082AA2E0FBA3E475F00112008198A9F0FA740412008124900822E8FB
:20732000E0FCA3E0FDA3E0FEA3E0FF90082AA2E0FBA3E0FAA3E0F9120083C290082AA3E416
:2073400075F0041200818290082AA2E0FBA3E0FAA3E0F974FF1200812490081A697401F0CD
:20736000A3742CF0900822E0E0FCA3E0FDA3E0FEA3E0FF7B097A2279D01201BEE07F027EC8
:20738000001201272512023CA1EF24A0FFEE348CFEE43DFDE43CFC900822F01200842F2274
:2073A000900827E6EEF0A3EFF09008066BE0FBA3E0FAA3E0F9120081AE45F0705090081904
:2073C00076E0FBA3E0FAA3E0F990081A69E0FEA3E0FFE92FF9EA3EFA900823FF7483F0A371
:2073E0007453F0A37405F01200959290081A6AE02FF090081A69E03EF09008066BE0FBA3C6
:20740000E0FAA3E0F9E475F001120082289008066BE0FBA3E0FAA3E0F9120081AEC394019A
:20742000FFE5F09400FE900827EEF0A3EFF0900828EA7409F0A37427F0A374F0F07B097A8D
:207440002779E812021232EF4E7019D390081A6AE0940090081A69E09400400321768C7EB0
:20746000007F0122900827F0E0FBA3E0FAA3E0F91200A3BEEF4E700F900827F07483F0A37F
:207480007453F0A37474F090081976E0FBA3E0FAA3E0F990081A69E0FEA3E0FFE92FF9EA49
:2074A0003EFA900823FF7483F0A37453F0A3747BF01200959290081A6AE02FF090081A69A8
:2074C000E03EF0900827E6E07004A3E06401704D90081976E0FBA3E0FAA3E0F990081A69EA
:2074E000E0FEA3E0FFE92FF9EA3EFA900823FF7483F0A37453F0A37495F0900827EEE0FFD6
:20750000A3E090082402CFF0A3EFF01200959290081A6AE02FF090081A69E03EF0900819BB
:2075200076E0FBA3E0FAA3E0F990081A69E0FEA3E0FFE92FF9EA3EFAC002C001900823FF16
:207540007483F0A37453F0A374ADF0900827EFE02401FE900827EEE0340090082402F0A373
:20756000CEF0900827F0E0F9A3E0FAA3E090082404C9F0A3EAF0A3E9F0D001D00212009509
:207580009290081A6AE02FF090081A69E03EF0E4900827ECF0A3F0C390082484E09401FF8C
:2075A00090082483E09400FE900827ECE0FCA3E0FDC39FEE6480F8EC648098400321766441
:2075C000EDAE047803CEA2E713CE13D8F824E8F58274273EF583759308E0FD7C009008277A
:2075E000EDE05407FF74017E00A807088005C333CE33CED8F9FFEE5CFEEF5D4E6053900873
:207600001976E0FBA3E0FAA3E0F990081A69E0FEA3E0FFE92FF9EA3EFA900823FF7483F0B8
:20762000A37453F0A374C3F0900827EDE02401FE900827ECE0340090082402F0A3CEF01297
:2076400000959290081A6AE02FF090081A69E03EF0900827EDE004F07007900827ECE00439
:20766000F02175979008066BE0FBA3E0FAA3E0F9E475F001120081FCC390081A6AE094B034
:2076800090081A69E09404500321740DE4FEFF2290081DAAEBF0A3EAF0A3E9F0900828323A
:2076A0007481F0A3748EF0A374FBF0120207F590081DAAEBF0A3EAF0A3E9F09008230174DB
:2076C00081F0A3748FF0A37403F0A37409F0A3741DF0A374ADF01200997190081DAEE0242E
:2076E000FFF090081DADE034FFF0E0FEA3E0FF7B097A1D79B7120228C57E007F047D007B91
:20770000097A1D79B9120088517E007F047D007B097A1D79BD12008851E490081DB1F0A315
:20772000F0C390082484E09401FF90082483E09400FEC390081DB2E09FEE6480F890081D09
:20774000B1E0648098400321795F900823FF7481F0A3748EF0A374F3F090081DB1E0FFA3CA
:20776000E090082402CFF0A3EFF07B097A1E791112009592900828327409F0A3741EF0A324
:207780007411F090081DAAE0FBA3E0FAA3E0F9120207F590081DAAEBF0A3EAF0A3E9F0906E
:2077A0000829A07481F0A3748EF0A374F8F07B097A1E79111202253D900823017409F0A397
:2077C000741EF0A37411F0A37409F0A3741DF0A374AFF090081DAAE0FBA3E0FAA3E0F912E0
:2077E00000997190081DB1E0FCA3E0FDAE047803CEA2E713CE13D8F8FF90081DB3EEF0A38D
:20780000EFF07E00ED5407FFD390081DB0E0940090081DAFE064809480406B90081DB4E0E8
:2078200024B9F582E4341DF583C083C082759308E0FDAC077401A804088002C333D8FC4D60
:20784000759308D082D083F090081DAFE07004A3E06402600321794090081DB4E024BDF586
:2078600082E4341DF583C083C082759308E0FD7401A807088002C333D8FC4D759308D08240
:20788000D083F021794090081DB1E0FEA3E0FF7B097A1D79B51202347490081DB5E0540F53
:2078A000FCA3E0FDA3E06C7003A3E06D6003217940900823FF7481F0A3748FF0A3740DF074
:2078C00090081DB2E02401FE90081DB1E0340090082402F0A3CEF0A3ECF0A3EDF07B097AB8
:2078E0001D79C112009592900823FF7481F0A3748FF0A3744EF090081DAEE02401FE900870
:207900001DADE0340090082402F0A3CEF07B097A1E7911120095929008296A7409F0A374EC
:207920001DF0A374C1F0A37409F0A3741EF0A37411F07B817A8E798012021578E4FEFF2284
:2079400090081DABE475F0041200818290081DB2E004F0700790081DB1E004F02177219030
:20796000081DADE0FEA3E0FF7B097A1D79B71200FFFB120234B17E007F01227B097A2279CC
:20798000F412023847E4FFFEFDFC1202370BE4FFFEFDFC12023E12E4FFFEFDFC12023E1AAC
:2079A000E4FFFEFDFC900822F01200842FE4FFFEFDFC900822DA1200842F12023CA1EF2447
:2079C00032FFE43EFEE43DFDE43CFC900822D61200842F900822DEE4F0A37402F012023C02
:2079E000A1900822D6E0F8A3E0F9A3E0FAA3E0FBC31200836E5003217C3712023CA1900891
:207A000022DAE0F8A3E0F9A3E0FAA3E0FBC31200836E503D900822DEE07004A3E064027083
:207A20000612018A6E8011900822DEE07004A3E0640370A912015D8E12023CA1EF240AFFAA
:207A4000E43EFEE43DFDE43CFC900822DA1200842F7B097A1A79691201C7619008248FEB08
:207A6000F0A3EAF0A3E9F09008248FE0FBA3E0FAA3E04A4B70032179DD9008248FE0FBA3AF
:207A8000E0FAA3E0F990081A69E0FEA3E0FFE92FF9EA3EFAE4120081249008248FE0FBA37E
:207AA000E0FAA3E0F990081973EBF0A3EAF0A3E9F0240CF9E43AFA120081AEB40041E5F02C
:207AC000B4813C9008248FA3E0FAA3E02410F9E43AFA120081AEFF90081973E0FBA3E0FAE9
:207AE000A3E0240CF9E43AFAE5F08FF0120082289008248FE0FBA3E0FAA3E02412800D9039
:207B0000081973E0FBA3E0FAA3E0240EF9E43AFA9008197FEBF0A3EAF0A3E9F09008197F7F
:207B2000E0FBA3E0FAA3E02414F9E43AFA90081979EBF0A3EAF0A3E9F09008197FA3E0FA76
:207B4000A3E02414F9E43AFA9008197CEBF0A3EAF0A3E9F09008197FA3E0FAA3E0F97D149E
:207B60007C001201D3E6EFF47002EEF46003217C3090081973E0FBA3E0FAA3E0240CF9E44A
:207B80003AFA120081AEB40044E5F0B4083F9008197FE0FBA3E0FAA3E02409F9E43AFA124D
:207BA0000080D3B411279008197CE0FBA3E0FAA3E0F9120081AE644345F07011E92402F9DF
:207BC000E43AFA120081AE644445F060028061120184F1EF64014E7057900822E8E0FCA31A
:207BE000E0FDA3E0FEA3E0FF1202370B900822FAE0FCA3E0FDA3E0FEA3E0FF12023E129048
:207C00000822E4E0FCA3E0FDA3E0FEA3E0FF12023E1A12023CA1EF24A0FFEE348CFEE43D1B
:207C2000FDE43CFC900822F01200842F02008023120080232179DD7F017E007DA87CC0127A
:207C400002370B74FF7F00FEFDFC12023E127FFE7E007DA87CC012023E1A2290081D25EBE4
:207C6000F0A3EAF0A3E9F0E4A3F0A3F0900828327481F0A3748DF0A374E2F090081D25E003
:207C8000FBA3E0FAA3E0F9120207F590081D25EBF0A3EAF0A3E9F09008264B7481F0A3742D
:207CA0008DF0A374E2F0A37481F0A3748AF0A37458F0A37409F0A3741DF0A37432F0120166
:207CC000E0B4E490081D2AF0A3F07B097A1D79321200A3BEC390081D2BE09FEE6480F89015
:207CE000081D2AE06480985039A3E02432F582E4341DF583759308E0FF12023D50401190E2
:207D000008296A7481F0A3748DF0A374F5217DD690081D2BE004F070B190081D2AE004F047
:207D200080A87B097A1D79321202000790081D2CEEF0A3EFF0900828327481F0A3748EF08D
:207D4000A37410F090081D25E0FBA3E0FAA3E0F9120207F590081D25EBF0A3EAF0A3E9F0A0
:207D60009008264B7481F0A3748EF0A37410F0A37481F0A3748AF0A37458F0A37409F0A33E
:207D8000741DF0A37432F01201E0B4E490081D2AF0A3F07B097A1D79321200A3BEC39008A8
:207DA0001D2BE09FEE6480F890081D2AE06480985045A3E02432F582E4341DF58375930855
:207DC000E0FF12023D50401D9008296A7481F0A3748EF0A37416F0A37481F0A3748EF0A344
:207DE0007407217F0390081D2BE004F070A590081D2AE004F0809C7B097A1D7932120200F3
:207E00000790081D2EEEF0A3EFF090081D25E0FBA3E0FAA3E04A4B7003217F3190081D2CA9
:207E2000E0FCA3E0FDEC540FFEAF0590081D30E054F04EFE90081D30EEF0FAA3EFF0FB90C6
:207E4000081D2FE05407C454F0FEEA548F4EFEEBFFA3EEF0A3EFF0EE547F90081D30F0A34E
:207E6000EFF090081D28E0FEA3E0FF12020A6BEF601690081D28E0FEA3E0FF7B097A1D7927
:207E80003012022CFC217F12900823FF7481F0A3748EF0A3742DF090081D2CE0FCA3E0FD1F
:207EA00090082402ECF0A3EDF090081D29E02401FE90081D28E0340090082404F0A3CEF0C5
:207EC000A3ECF0A3EDF07B097A1D794612009592900823FF7481F0A3748EF0A37470F07B6A
:207EE000097A1D7996120095929008296A7409F0A3741DF0A37446F0A37409F0A3741DF05D
:207F0000A37496F07B817A8D79E812021578E4FEFF2290081D26E475F005120081829008E6
:207F20001D29E004F0700790081D28E004F0217C6C120234B17E007F0122E49008266FF0DC
:207F4000A3F0E490082671F0A3F090082671E0FCA3E0FDC39402EC6480948040032180DE6E
:207F60009008266FE0FEA3E07802C333CE33CED8F92DFFEC3EFE90082673F0A3EFF09008D4
:207F800022A075F0031200843BEE75F003A42583F583759308E0F9A3E0FAA3E09008267BAA
:207FA000C9F0A3EAF0A3E9F07E007F04C006C0077D0090082673E0FEA3E07802C333CE3301
:207FC000CED8F924C3F974213EFA7B09D007D00612008851900828327483F0A374ACF0A30A
:207FE00074EBF09008267BE0FBA3E0FAA3E0F9120207F59008267BEBF0A3EAF0A3E9F09078
:2080000008267BE0FBA3E0FAA3E04A4B70032180C8900823017483F0A374ACF0A374EDF021
:20802000A37409F0A37426F0A37475F09008267BE0FBA3E0FAA3E0F912009971900826762A
:20804000E024FFF090082675E034FFF0E0FAA3E0FB7C007D08FFAE021200814AA3EEF0A3EE
:20806000EFF07C007D08AF03AE021200814AA3ECF0A3EDF090082678E0FF90082674E02596
:20808000E025E024C3F582E43421F583E5822FF582E43583F583C083C082759308E0FF90C7
:2080A00008267AE0FE7401A806088002C333D8FC4F759308D082D083F09008267CE475F04C
:2080C0000112008182217FD490082672E004F06003217F4A90082671E004F0217F4A900840
:2080E000266FE0FEA3E07802C333CE33CED8F9FF90082673EEF0A3EFF090082671E0700269
:20810000A3E070032181F1E490082671F0A3F0C39008247AE09401FF90082479E09400FE2C
:20812000C390082672E09FEE6480F890082671E064809840032181BEE0FAA3E0FB7C007D84
:2081400008FFAE021200814A90082677EEF0A3EFF07C007D08AF03AE021200814AA3ECF037
:20816000A3EDF090082678E0FF90082674E025E025E024C3F582E43421F583E5822FF58232
:20818000E43583F583759308E0FD7C009008267AE0FF74017E00A807088005C333CE33CE57
:2081A000D8F9FFEE5CFEEF5D4E701390082672E004F0700790082671E004F021810F9008C3
:2081C0002671E0FEA3E0FF900829B37409F0A37426F0A37480F07B097A26797E1202285D5F
:2081E00090082670E0FBFF9008267FE0FD120238C290082670E004F070079008266FE004C5
:20820000F0C390082670E094039008266FE0648094805003217F422290080660E0FBA3E04E
:20822000FAA3E0F9120081AEFFAEF0E5F060032184EBEF24FE60491470032184AE24026008
:20824000032184EB900823FF7483F0A374ACF0A374F3F090081976E0FBA3E0FAA3E0F91230
:2082600000959290081A69EEF0A3EFF090080660E0FBA3E0FAA3E0F9E475F0021200822883
:208280009008066BE0FBA3E0FAA3E0F9120081AEC39401FFE5F09400FE900827E4F0A3EFDD
:2082A000F0C39403EE64809480401790080660E0FBA3E0FAA3E0F9E475F003120082287FDE
:2082C0000022900827E5E0FF7B097A2779D91202343690081976E0FBA3E0FAA3E0F9900871
:2082E0001A69E0FEA3E0FFE92FF9EA3EFA900823FF7483F0A374AEF0A37435F0900827E433
:20830000E0FCA3E0FD2401FEE43C90082402F0A3CEF0A3ECF0A3EDF01200959290081A6A5B
:20832000E02FF090081A69E03EF0E4900827E0F0A3F0900827E0E0FCA3E0FDC39402EC646B
:208340008094804003218497900827E4E0FEA3E07802C333CE33CED8F92DFFEC3EFE90080A
:2083600027E2F0A3EFF0900822A075F0031200843BEE75F003A42583F583759308E0FBA347
:20838000E0FAA3E0F91200A3BEC3EF9406EE648094805003218484900827E2E0FEA3E078EC
:2083A00002C333CE33CED8F924C3F974213EFA7B0978D97C277D097E007F04120087C7EF2A
:2083C000900827DD700D7483F0A374AEF0A37488F0800B7483F0A374AEF0A37491F0900802
:2083E0001976E0FBA3E0FAA3E0F990081A69E0FEA3E0FFE92FF9EA3EFAC003C002C0019096
:208400000823FF7483F0A374AEF0A37492F0900827E2E0FCA3E0FD2401FEE43C90082402FF
:20842000F0A3CEF0900827DDE0F9A3E0FAA3E090082404C9F0A3EAF0A3E9F0900822A07535
:20844000F003ED1200843BEC75F003A42583F583759308E0FBA3E0FAA3E02401F9E43AFA32
:2084600090082407EBF0A3EAF0A3E9F0D001D002D0031200959290081A6AE02FF090081AE9
:2084800069E03EF0900827E1E004F07007900827E0E004F02183329008066BE0FBA3E0FAD0
:2084A000A3E0F9E475F001120081FC218280900823FF7483F0A374AEF0A374AEF090081988
:2084C00076E0FBA3E0FAA3E0F91200959290081A69EEF0A3EFF090080660E0FBA3E0FAA3A5
:2084E000E0F9E4F5F01200822880037F01227F00229008197CE0FBA3E0FAA3E02408F9E447
:208500003AFA900829E6EBF0A3EAF0A3E9F0A3EBF0A3EAF0A3E9F0900829E6E0FBA3E0FA36
:20852000A3E0F9120080D36402706BE92404F9E43AFA120083A5900822ECE0F8A3E0F9A320
:20854000E0FAA3E0FBC31200836E706F900829E6E0FBA3E0FAA3E024ECF9E43AFA120083E6
:20856000A57B637A5379827863C31200836E704B900829E6E0FBA3E0FAA3E0241CF9E43A7B
:20858000A801FCAD037B097A2279F47E007F06120087C7EF60032187BC900829E6E0FBA3BB
:2085A000E0FAA3E024F0F9E43AFAA3EBF0A3EAF0A3E9F0120080D3643560032187BC900865
:2085C00029EAE475F00212008182900822DEE0FEA3E0FFEE60032187BCEF24FD7003218651
:2085E000A70460032187BC900829E9E0FBA3E0FAA3E0F9120080D3640260032187BC900861
:2086000029E6E0FBA3E0FAA3E02410F9E43AFA120083A5900822E81200842F900829EAE4FB
:2086200075F0018062900829E9E0FBA3E0FAA3E0F9120080D3FFF46054EF24CA701DE924F1
:2086400002F9E43AFA120083A5900822E01200842F900829EAE475F006802C900829E9E03E
:20866000FBA3E0FAA3E02401F9E43AFA120080D3FF7E00900829ECEEF0A3EFF02402FFEEC7
:2086800033900829EA8FF0120081828098900822DEE4F0A37403F0E4FFFEFDFC900822DA6C
:2086A0001200842F2187BC900829E9E0FBA3E0FAA3E0F9120080D3640560032187BC9008E6
:2086C00029E6E0FBA3E0FAA3E02410F9E43AFA120083A5900822E8E0F8A3E0F9A3E0FAA31B
:2086E000E0FBC31200836E60032187BC90081973E0FBA3E0FAA3E02406F9E43AFA78D07C14
:20870000227D097E007F0612008055900829EAE475F0012187A6900829E9E0FBA3E0FAA3DF
:20872000E0F9120080D3FFF470032187ADEF24FD602124027044E92402F9E43AFA12008320
:20874000A5900822FA1200842F900829EAE475F0068053900829E9E0FBA3E0FAA3E0240283
:20876000F9E43AFA120083A5900822E41200842F900829EAE475F006802C900829E9E0FB20
:20878000A3E0FAA3E02401F9E43AFA120080D3FF7E00900829ECEEF0A3EFF02402FFEE336E
:2087A000900829EA8FF012008182218716900822DEE4F0A37404F07E007F0122E4FEFF2222
:2087C00090082979EEF0A3EFF09008066BE0FBA3E0FAA3E0F9120081AE45F0600321889B05
:2087E00090081976E0FBA3E0FAA3E0F990081A69E0FEA3E0FFE92FF9EA3EFA900823FF74A2
:2088000083F0A3746BF0A3749CF01200959290081A6AE02FF090081A69E03EF09008297B17
:20882000E4F0A304F090081976E0FBA3E0FAA3E0F990081A69E0FEA3E0FFE92FF9EA3EFA24
:20884000900823FF7483F0A3746BF0A374CAF01200959290081A6AE02FF090081A69E03EA7
:20886000F09008297CE004F070079008297BE004F0D39008297CE094049008297BE06480E8
:20888000948040A19008066BE0FBA3E0FAA3E0F9E475F00112008228218A6A9008066BE002
:2088A000FBA3E0FAA3E0F9120081AEFFC390082484E09401FD90082483E09400FCD3EF9D01
:2088C000E5F09C40057E007F012290081976E0FBA3E0FAA3E0F990081A69E0FEA3E0FFE963
:2088E0002FF9EA3EFA900823FF7483F0A3746CF0A37411F01200959290081A6AE02FF0901E
:20890000081A69E03EF090082979E07004A3E064019008297F700D7483F0A3746CF0A3741A
:2089200025F0800B7483F0A3746CF0A374ADF0E49008297BF0A3F09008066BE0FBA3E0FA85
:20894000A3E0F9120081AEFFAEF0C390082484E09401FD90082483E09400FCD3EF9DEE9CB0
:2089600040032189F4C3EF9401FFEE9400FE7B097A29797D1202347490081976E0FBA3E0F2
:20898000FAA3E0F990081A69E0FEA3E0FFE92FF9EA3EFAC003C002C0019008297FE0F9A3B1
:2089A000E0FAA3E0900823FFC9F0A3EAF0A3E9F09008066BE0FBA3E0FAA3E0F9120081AED0
:2089C000FF90082402E5F0F0A3EFF09008297DE0FCA3E0FDEC540FAF0590082404F0A3EFB4
:2089E000F0ECC45407FFA3E4F0A3EFF0D001D002D003802A90081976E0FBA3E0FAA3E0F969
:208A000090081A69E0FEA3E0FFE92FF9EA3EFA900823FF7483F0A3746CF0A374CBF01200B0
:208A2000959290081A6AE02FF090081A69E03EF09008066BE0FBA3E0FAA3E0F9E475F001A4
:208A4000120081FC9008297CE004F070079008297BE004F0D39008297CE094039008297B2C
:208A6000E0648094805003218937E4FEFF227B097A19798F90081A66EBF0A3EAF0A3E9F0DC
:208A80002414F9E43AFA74111200812474FFFFFEFDFC90081A66E0FBA3E0FAA3E02404F9D4
:208AA000E43AFA120083C290081A66E0FBA3E0FAA3E0F9E475F0441200822890081A66E01A
:208AC000FBA3E0FAA3E02402F9E43AFAE475F0431200822812020B2B12023DF0EF4E700ED6
:208AE00012023DC9AC06AD077F01120235269008197CE0FBA3E0FAA3E02408F9E43AFA9032
:208B0000082A93EBF0A3EAF0A3E9F024ECF9E43AFAA3EBF0A3EAF0A3E9F012023CA190089B
:208B200022EC1200842F90082A93E0FBA3E0FAA3E0F974011200812490082A93E0FBA3E05A
:208B4000FAA3E02401F9E43AFA74011200812490082A93E0FBA3E0FAA3E02402F9E43AFACF
:208B6000740612008124900822ECE0FCA3E0FDA3E0FEA3E0FF90082A93E0FBA3E0FAA3E08F
:208B80002404F9E43AFA120083C290082A93E0FBA3E0FAA3E0241CF9E43AA801FCAD037BEE
:208BA000097A2279F47E007F06120080557F637E537D827C6390082A96E0FBA3E0FAA3E0F5
:208BC000F9120083C290082A97E475F0041200818290082A96E0FBA3E475F001120081983F
:208BE000A9F0FA74351200812490082A96E0FBA3E475F00112008198A9F0FA74011200819C
:208C00002490082A96E0FBA3E475F00112008198A9F0FA74011200812490082A96E0FBA350
:208C2000E475F00112008198A9F0FA743D1200812490082A96E0FBA3E475F0011200819879
:208C4000A9F0FA74071200812490082A96E0FBA3E475F00112008198A9F0FA740112008169
:208C60002490082A96E0FBA3E0FAA3E0F8AC02AD037B097A2279F47E007F06120080559040
:208C8000082A97E475F0061200818290082A96E0FBA3E475F00112008198A9F0FA7437120C
:208CA00000812490082A96E0FBA3E475F00112008198A9F0FA74021200812490082A96E0CC
:208CC000FBA3E475F00112008198A9F0FA74011200812490082A96E0FBA3E475F001120090
:208CE0008198A9F0FA74031200812490082A96E0FBA3E0FAA3E0F974FF1200812490081A92
:208D0000697401F0A3742CF07F017E00020127259008252FEEF0A3EFF0900825487401F04F
:208D2000E490082547F090082547E0FBFFD39008248CE09F7480F89008248BE06480984014
:208D40003DE4FFFEFDFCEB25E025E0243AF582E43425F5837593081200842FE4FFFEFDFCCE
:208D6000EB25E025E0243EF582E43425F5837593081200842F90082547E004F080A8E49027
:208D8000082539F07F01FEFDFC218EF790082539E0FFD390082484E09F7480F890082483CE
:208DA000E06480985003218F0290082539E025E025E02472F582E43406F583759308E0904F
:208DC000082546F0EF25E025E02471F582E43406F583759308E090082547F090082542E0D2
:208DE000FCA3E0FDA3E0FEA3E0FF90082531E0F8A3E0F9A3E0FAA3E05FFFEA5EFEE95DFDCB
:208E0000E85C4D4E4F605490082547E025E025E0243AF582E43425F583C083C08275930863
:208E2000E0F8A3E0F9A3E0FAA3E0FBC000C001E47F01FEFDFC90082546E0F9F8120083920C
:208E4000D001D000EB4FFFEA4EFEE94DFDE84CFC759308D082D0831200842F90082542E046
:208E6000FCA3E0FDA3E0FEA3E0FF90082535E0F8A3E0F9A3E0FAA3E05FFFEA5EFEE95DFD46
:208E8000E85C4D4E4F605490082547E025E025E0243EF582E43425F583C083C082759308DF
:208EA000E0F8A3E0F9A3E0FAA3E0FBC000C001E47F01FEFDFC90082546E0F9F8120083928C
:208EC000D001D000EB4FFFEA4EFEE94DFDE84CFC759308D082D0831200842F90082539E0CF
:208EE00004F090082542E0FCA3E0FDA3E0FEA3E0FF780112008392900825421200842F219B
:208F00008D8CE490082547F090082547E0FBFFD39008248CE09F7480F89008248BE06480F1
:208F200098407190082547E0C00725E025E0243AF582E43425F583759308E0FCA3E0FDA39A
:208F4000E0FEA3E0FF900827011200842FEB25E025E0243EF582E43425F583759308E0FCBD
:208F6000A3E0FDA3E0FEA3E0FF900827051200842F90082548E090082709F09008252FE07C
:208F8000FCA3E0FDD0071201F27F90082547E004F0218F08229008197CE0FBA3E0FAA3E040
:208FA0002408F9E43AFA9008298BEBF0A3EAF0A3E9F02410F9E43AFA120083A57BD87A5AAE
:208FC00079947801C31200836E600321919C9008298BE0FBA3E0FAA3E02402F9E43AFA1224
:208FE0000081AEFFAEF090082BB4EEF0A3EFF064014E601590082BB4E0FEA3E0FF4E600918
:20900000EF64024E600321919C7B097A29798E120238479008298BE0FBA3E0FAA3E0240EE2
:20902000F9E43AFAE4F5F0120082289008298BE0FBA3E0FAA3E0240CF9E43AFA120081AEF1
:20904000FFAEF0E5F0600321919CEF24FD603724FE70032190EA24FE700321910624FD7038
:20906000032191392409600321919C120153409008298BE0FBA3E0FAA3E0240CF9E43AFA16
:20908000E475F00280549008298BE0FBA3E0FAA3E02404F9E43AFA788E7C297D097E007F23
:2090A00006120087C7EF70169008298BE0FBA3E0FAA3E0F9120081AE640245F060032191C4
:2090C0009C1201673E9008298BE0FBA3E0FAA3E0240CF9E43AFAE475F00412008228900833
:2090E0002BB4E4F0A304F02191A0120153409008298BE0FBA3E0FAA3E0240CF9E43AFAE4E2
:2091000075F00621918C9008298BE0FBA3E0FAA3E0F9120081AE640245F06002807E120137
:20912000673E9008298BE0FBA3E0FAA3E0240CF9E43AFAE475F00880539008298BE0FBA334
:20914000E0FAA3E02404F9E43AFA788E7C297D097E007F06120087C7EF70169008298BE044
:20916000FBA3E0FAA3E0F9120081AE640245F0600280291201673E9008298BE0FBA3E0FAB8
:20918000A3E0240CF9E43AFAE475F00B1200822890082BB4E4F0A37402F08004020080237E
:2091A0009008298BE0FBA3E0FAA3E02404F9E43AA801FCAD037B097A29798E7E007F0612B1
:2091C0000080559008298BE0FBA3E0FAA3E0F9E475F002120082289008298BE0FBA3E0FAEF
:2091E000A3E02402F9E43AFAE475F001120082289008298BE0FBA3E0FAA3E0240AF9E43A43
:20920000FAE475F0011200822890082BB4E0FEA3E0FF1201272522900824F8EEF0A3EFF0E2
:20922000E490082513F0A3F0FE7F04FD7B097A2579051200885112023DF0EF64014E6003A7
:2092400021935F900824FAF0A3F0900824FAE0FEA3E0FFC39418EE648094804003219484DB
:20926000900828EA7409F0A37424F0A374FEF07B097A25790112021232EF4E7003219484C9
:20928000E4900824FCF0A3F0900824FDE02401F582E43425F583C083C082759308E0FD90C3
:2092A0000824F8E0FEA3E07802C333CE33CED8F924C3F58274213EF583C083C0829008242F
